:100000000C948E0E0C9496170C94C7170C94F8173A
:100010000C9429180C945A180C948B180C94BC1836
:100020000C94ED180C94BB0E0C94BB0E0C94BB0EF0
:100030000C94BB0E0C94D9960C94BB0E0C94BB0E76
:100040000C94BB0E0C947A6B0C94BB0E0C94BB0EF0
:100050000C94BB0E0C94BB0E0C9472740C9485140F
:100060000C94BB0E0C9407410C94BB0E0C94BB0E6D
:100070000C94BB0E0C94BB0E0C94BB0E0C94BB0EDC
:100080000C94BB0E0C94BB0E0C94BB0E0C94BB0ECC
:100090000C94BB0E0C94BB0E0C94BB0E0C94BB0EBC
:1000A0000C94BB0E0C94BB0E0C94BB0E0C94BB0EAC
:1000B0000C94BB0E0C94BB0E0C94BB0E0C94BB0E9C
:1000C0000C94BB0E0C94BB0E0C94BB0E0C94BB0E8C
:1000D0000C94BB0E0C94BB0E0C94BB0E0C94BB0E7C
:1000E0000C94BB0E084AD73B3BCE016E84BCBFFDCF
:1000F000C12F3D6C74319ABD56833DDA3D00C77FF8
:1001000011BED9E4BB4C3E916BAAAABE0000008090
:100110003F05A84CCDB2D44EB93836A9020C50B91F
:10012000918688083CA6AAAA2ABE000000803F004B
:10013000002100240027002A002D00300033000198
:10014000010000040107010A010000220025002827
:10015000002B002E003100340002010000050108D0
:10016000010B01000020002300260029002C002F95
:100170000032000001000003010601090105050528
:1001800005070508080808020202020A0A0808040E
:10019000040404010101010101010103030303033C
:1001A000030303040707070C0C0C0C0C0C0C0C02CB
:1001B00002020206060606060606060B0B0B0B0BD2
:1001C0000B0B0B01021020200808102040102040CB
:1001D000800201020108040201010204081020400B
:1001E0008080402010080402018004020180402029
:1001F0001008040201080402010102040810204052
:100200008001020408102040800000090A02080B47
:100210000C0D0706030401000000000000000000B0
:1002200000000000000000000000000000000000CE
:10023000000000000011100F00000000000000008E
:100240000000000000000000000000000000006549
:1002500063686F3A004572726F723A0053544F50A0
:100260005045442E20005072696E7465722073747C
:100270006F707065642064756520746F206572729C
:100280006F72732E204669782074686520657272DB
:100290006F7220616E6420757365204D3939392085
:1002A000746F20726573746172742E202854656DAA
:1002B000706572617475726520697320726573650B
:1002C000742E2053657420697420616674657220F1
:1002D00072657374617274696E6729004B494C4C86
:1002E00045442E20005072696E7465722068616CFE
:1002F0007465642E206B696C6C28292063616C6CBA
:10030000656421006F6B00526573656E643A20006E
:100310002200556E6B6E6F776E20636F6D6D616E30
:10032000643A2022004368616E67652066696C61EB
:100330006D656E74005A204F6666736574203A20AE
:10034000007A5F6D61783A20007A5F6D696E3A20BD
:10035000005A204F6666736574005A204F666673B4
:100360006574206F6B00486F74656E64206F6666FD
:10037000736574733A007A5F6D696E3A2000795F35
:100380006D696E3A2000785F6D696E3A2000205AE0
:100390003A0020593A0020436F756E7420583A2075
:1003A0000020453A00205A3A0020593A00583A00B5
:1003B0004649524D574152455F4E414D453A4D6178
:1003C000726C696E2056313B20537072696E746591
:1003D000722F6772626C206D617368757020666F32
:1003E000722067656E36204649524D574152455F2F
:1003F00055524C3A687474703A2F2F6669726D7753
:100400006172652E756C74696D616B65722E636FB8
:100410006D2050524F544F434F4C5F5645525349F5
:100420004F4E3A312E30204D414348494E455F549E
:100430005950453A556C74696D616B657220455829
:100440005452554445525F434F554E543A3220550D
:100450005549443A30303030303030302D30303043
:10046000302D303030302D303030302D3030303095
:1004700030303030303030300A00556C74696D6186
:100480006B6572204F66662E0042656420646F6E55
:10049000652E0020423A0020453A00543A00426559
:1004A000642048656174696E672E004865617469EF
:1004B0006E6720646F6E652E0020573A0020453A23
:1004C00000543A0048656174696E672E2E2E002034
:1004D00042403A0020403A00202F003A00205400C9
:1004E000202F0020423A00202F006F6B20543A004A
:1004F0002569206D696E2C20256920736563004590
:100500006E642066696C65206C697374004265676F
:10051000696E2066696C65206C697374004E6F208B
:100520006D6F76652E00526573756D696E6720700C
:1005300072696E74005761697420666F72207573FA
:1005400065722E2E2E00536C6565702E2E2E00FFC8
:10055000FFFF0000524300005243000052430000DE
:10056000000000000000000000000000000000008B
:100570000000000000000000524300005243000051
:1005800052430000A0400000A04000000040256948
:1005900020686F757273202569206D696E757465AA
:1005A0007300446F6E65207072696E74696E6720A7
:1005B00066696C650053544F505045442E200050DE
:1005C00072696E7465722073746F707065642064F4
:1005D000756520746F206572726F72732E20466984
:1005E0007820746865206572726F7220616E642075
:1005F000757365204D39393920746F2072657374B5
:100600006172742E202854656D7065726174757204
:10061000652069732072657365742E20536574209C
:100620006974206166746572207265737461727496
:10063000696E6729006F6B004E6F204C696E6520F4
:100640004E756D62657220776974682063686563B2
:100650006B73756D2C204C617374204C696E653A18
:1006600020004E6F20436865636B73756D2077695A
:100670007468206C696E65206E756D6265722C20E1
:100680004C617374204C696E653A20006368656341
:100690006B73756D206D69736D617463682C204C8C
:1006A000617374204C696E653A20004C696E652058
:1006B0004E756D626572206973206E6F74204C6197
:1006C0007374204C696E65204E756D6265722B31B6
:1006D0002C204C617374204C696E653A20004D31BA
:1006E000313000446F6E6520736176696E672066F5
:1006F000696C652E006F6B004D3239002020506C04
:10070000616E6E6572427566666572427974657374
:100710003A20002046726565204D656D6F72793A0A
:100720002000536570203139203230313400436F5E
:100730006D70696C65643A200028446176696420B4
:10074000427261616D2900207C20417574686F726E
:100750003A20005365702031392032303134203155
:10076000303A32323A353500204C6173742055707E
:1007700064617465643A2000312E302E30004D6182
:10078000726C696E0020536F6674776172652052D7
:100790006573657400205761746368646F672052E5
:1007A00065736574002042726F776E206F757420D8
:1007B0005265736574002045787465726E616C20B3
:1007C000526573657400506F77657255700073746D
:1007D000617274002200656E717565696E67202212
:1007E000002200656E717565696E672022007C3C91
:1007F0003E5E2B3D3F2F5B5D3B2C2A225C006563F8
:10080000686F3A0020746F6F206C6F6E6720657898
:1008100074727573696F6E2070726576656E74653B
:10082000640020636F6C6420657874727573696FFF
:100830006E2070726576656E7465640045303A208E
:10084000005A3A2000593A2000583A20004D5331BE
:100850002C4D53322050696E730A0024F404D920C1
:100860001BC40C5C0E9804C4095F0265077101F497
:1008700005F900FB04B30048048700C10369005870
:1008800003550003034500BE023A008402310053C1
:10089000022A002902250004022000E4011C00C8ED
:1008A000011900AF011700980114008401130071B1
:1008B0000110006101100051010E0043010D0036CE
:1008C000010B002B010B0020010B00150109000C8E
:1008D00001090003010800FB000800F3000800EB19
:1008E000000700E4000600DE000600D8000600D283
:1008F000000600CC000500C7000500C2000500BDD1
:10090000000400B9000400B5000400B1000400AD0B
:10091000000400A9000400A5000300A20003009F3A
:100920000004009B00030098000300950002009360
:10093000000300900003008D0002008B000300887C
:100940000002008600020084000300810002007F94
:100950000002007D0002007B0002007900020077A7
:1009600000010076000200740002007200010071B4
:100970000002006F0002006D0001006C0002006ABE
:1009800000010069000200670001006600010065C7
:1009900000010064000200620001006100010060CB
:1009A0000001005F0002005D0001005C0001005BCF
:1009B0000001005A000100590001005800010057D1
:1009C00000010056000100550001005400010053D1
:1009D00000000053000100520001005100010050CE
:1009E0000001004F0001004E0000004E0001004DCC
:1009F0000001004C0001004B0000004B0001004AC8
:100A000000010049000100480000004800010047C3
:100A100000010046000000460001004500000045BE
:100A200000010044000100430000004300010042B7
:100A300000000042000100410000004100010040B0
:100A40000001003F0000003F0001003E0000003EAA
:100A50000001003D0000003D0001003C0000003CA2
:100A60000000003C0001003B0000003B0001003A98
:100A70000000003A00010039000000390001003890
:100A80000000003800000038000100370000003787
:100A9000000100360000003600000036000100357D
:100AA0000000003500000035000100340000003473
:100AB0000000003400010033000000330000003368
:100AC000000100320000003200000032000100315D
:100AD0000000003100000031000100300000003053
:100AE000000000300001002F0000002F0000002F48
:100AF0000000002F0001002E0000002E0000002E3C
:100B00000001002D0000002D0000002D0000002D30
:100B10000001002C0000002C0000002C0000002C24
:100B20000001002B0000002B0000002B0000002B18
:100B30000001002A0000002A0000002A0000002A0C
:100B40000001002900000029000000290000002900
:100B500000000029000100280000002800000028F3
:100B600000000028000000280001002700000027E6
:100B700000000027000000270000002700010026D9
:100B800000000026000000260000002600000026CD
:100B900000010025000000250000002500000025C0
:100BA00000000025000000250001002400000024B2
:100BB00000000024000000240000002400010023A5
:100BC0000000002300000023000000230000002399
:100BD000000000230000002300010022000000228A
:100BE000000000220000002200000022000000227D
:100BF0000001002100000021000000210000002170
:100C00000000002100000021000000210001002060
:100C10000000002000000020000000200000002054
:100C20000000002000000020000000200001001F44
:100C30000000001F0000001F0000001F0000001F38
:100C40000000001F0000001F0001001E0000001E29
:100C50000000001E0000001E00000024F4D43050EC
:100C6000C38E20C2A24017828B7011127A910D811F
:100C70006CD90AA861E108C7586607615143061E8E
:100C80004B5D05C145A7041A411104093D98037144
:100C90003931034036DB0265339102D4305402808F
:100CA0002E1D02632CEE01752AC501B028A001108B
:100CB0002781018F2564012B244B01E0223401ACF4
:100CC000211F018D200D01801FFC00841EED009767
:100CD0001DDF00B81CD200E61BC600201BBC006450
:100CE0001AB200B219A8000A19A0006A189900D116
:100CF00017910040178B00B516840031167E00B3A3
:100D00001579003A157300C7146F0058146A00EE85
:100D10001366008813630025135E00C7125B006C26
:100D200012570015125400C111510070114F0021CB
:100D3000114B00D61049008D1047004610440002A8
:100D4000104200C00F4000800F3E00420F3C0006E2
:100D50000F3B00CB0E3800930E37005C0E3500279A
:100D60000E3400F30D3200C10D3100900D300060E3
:100D70000D2E00320D2D00050D2C00D90C2B00AED0
:100D80000C2900850C29005C0C2700350C27000E6F
:100D90000C2600E80B2400C40B2400A00B23007DCC
:100DA0000B23005A0B2100390B2100180B2000F8EF
:100DB0000A1F00D90A1E00BB0A1E009D0A1D0080E2
:100DC0000A1D00630A1C00470A1B002C0A1B0011A5
:100DD0000A1A00F7091A00DD091900C4091900AB45
:100DE000091900920917007B091800630917004CC4
:100DF00009160036091600200916000A091500F523
:100E0000081500E0081400CC081400B8081400A469
:100E1000081400900813007D0812006B0813005896
:100E200008120046081200340811002308110012AD
:100E300008110001081100F0071000E0071000D0B1
:100E4000071000C0071000B0070F00A107100091A5
:100E5000070E0083070F0074070F0065070E005789
:100E6000070E0049070E003B070D002E070E00205D
:100E7000070D0013070D0006070D00F9060C00ED25
:100E8000060D00E0060C00D4060C00C8060C00BCE1
:100E9000060C00B0060C00A4060B0099060C008D91
:100EA000060B0082060B0077060B006C060B006138
:100EB000060A0057060B004C060A0042060A0038D4
:100EC000060A002E060A0024060A001A060A001066
:100ED00006090007060A00FD050900F4050900EBF4
:100EE000050900E2050900D9050900D0050900C778
:100EF000050900BE050900B5050800AD050800A5F7
:100F00000509009C050800940508008C050800846C
:100F10000508007C050800740508006C05070065DD
:100F20000508005D050700560508004E0507004747
:100F30000507004005080038050700310507002AAD
:100F4000050700230507001C050600160507000F0E
:100F50000507000805060002050700FB040600F56A
:100F6000040700EE040600E8040600E2040700DBC4
:100F7000040600D5040600CF040600C9040600C319
:100F8000040600BD040600B7040600B1040500AC69
:100F9000040600A6040600A00405009B04060095B4
:100FA000040500900406008A0405008504050080FD
:100FB0000406007A04050075040500700405006B42
:100FC00004050066040500610405005C0405005783
:100FD000040500520405004D0405004804050043C3
:100FE0000405003E0404003A040500350405003001
:100FF0000404002C04050027040400230405001E3B
:101000000404001A04040016040500110404000D71
:10101000040400090405000404040000040400FCA6
:10102000030400F8030400F4030400F0030400ECDC
:10103000030400E8030400E4030400E0030400DC0C
:10104000030400D8030400D4030400D0030400CC3C
:10105000030400C8030300C50303006563686F3A17
:1010600000656E6473746F7073206869743A205AF7
:1010700000205A3A00656E6473746F70732068695B
:10108000743A20590020593A00656E6473746F7089
:1010900073206869743A20580020583A00656E64DD
:1010A00073746F7073206869743A20004572726FB0
:1010B000723A004572723A204D415854454D5020C5
:1010C0004245440054656D706572617475726520A7
:1010D0006865617465642062656420737769746310
:1010E000686564206F66662E204D415854454D500A
:1010F00020747269676765726564202121004572FA
:10110000723A204D494E54454D50003A204578746E
:101110007275646572207377697463686564206FA3
:1011200066662E204D494E54454D502074726967B5
:1011300067657265642021004572723A204D4158FE
:1011400054454D50003A204578747275646572209C
:101150007377697463686564206F66662E204D41FD
:101160005854454D502074726967676572656420F4
:101170002100202D20496E76616C696420657874A9
:101180007275646572206E756D6265722021000053
:10119000000000300E0100C00E0A00500F1400D0F5
:1011A0000F1E0060102800E010320070113C00F0AB
:1011B0001146007012500000135A008013640000A2
:1011C000146E00901478001015820090158C001099
:1011D0001696009016A0001017AA009017B40010E1
:1011E00018BE009018C8001019D2009019DC001029
:1011F0001AE600801AF000001BFA00801B0401F0C0
:101200001B0E01701C1801F01C2201601D2C01E056
:101210001D3601501E4001D01E4A01401F5401B02E
:101220001F5E0130206801A020720110217C019016
:10123000218601002290016026F401902A58028044
:101240002EBC0250322003E03584035039E803807D
:101250003C4C046563686F3A0048656174696E6769
:10126000206661696C656400504944204175746F63
:1012700074756E652066696E6973686564212050B7
:10128000757420746865206C617374204B702C2019
:101290004B6920616E64204B6420636F6E737461D0
:1012A0006E74732066726F6D2061626F766520695F
:1012B0006E746F20436F6E66696775726174696FD3
:1012C0006E2E6800504944204175746F74756E65C8
:1012D000206661696C6564212074696D656F757441
:1012E0000020403A006F6B20543A006F6B20423A66
:1012F00000504944204175746F74756E65206661B5
:10130000696C6564212054656D70657261747572D5
:101310006520746F6F206869676800204B643A200D
:1013200000204B693A2000204B703A200020436C8B
:1013300061737369632050494420002054753A203A
:1013400000204B753A2000206D61783A2000206D16
:10135000696E3A200020643A200020626961733A85
:1013600020004D383420582059205A20450065630C
:10137000686F3A0043616E6E6F7420656E746572BB
:10138000207375626469723A20004D3234004D3228
:1013900033202573006175746F25692E67004572CF
:1013A000726F723A006572726F7220777269746937
:1013B0006E6720746F2066696C65004E6F742053F1
:1013C00044207072696E74696E67002F0053442068
:1013D0007072696E74696E67206279746520002E80
:1013E0000044656C6574696F6E206661696C656444
:1013F0002C2046696C653A200046696C652064655E
:101400006C657465643A002E006F70656E206661CD
:10141000696C65642C2046696C653A2000577269D6
:1014200074696E6720746F2066696C653A20002EBF
:10143000006F70656E206661696C65642C2046697A
:101440006C653A20002E006F70656E206661696CD5
:1014500065642C2046696C653A200046696C6520FD
:1014600073656C6563746564002053697A653A201E
:101470000046696C65206F70656E65643A20002EC9
:10148000006F70656E206661696C65642C2046692A
:101490006C653A20004E6F7720667265736820662F
:1014A000696C653A20004E6F7720646F696E672023
:1014B00066696C653A20002220706F7300222070EC
:1014C0006172656E743A2200535542524F55544929
:1014D0004E452043414C4C207461726765743A223A
:1014E00000747279696E6720746F2063616C6C2080
:1014F0007375622D67636F64652066696C65732020
:101500007769746820746F6F206D616E79206C65E7
:1015100076656C732E204D4158206C6576656C2085
:1015200069733A0053442063617264206F6B006FEB
:1015300070656E526F6F74206661696C65640076C9
:101540006F6C756D652E696E6974206661696C6576
:101550006400534420696E6974206661696C00659B
:1015600063686F3A0048617264636F646564204425
:10157000656661756C742053657474696E67732059
:101580004C6F616465640053746F726564207365A9
:101590007474696E677320726574726965766564C8
:1015A000002044002049002020204D3330312050BD
:1015B000005049442073657474696E67733A002063
:1015C0005A0020590020204D323036205800486FF4
:1015D0006D65206F666673657420286D6D293A000D
:1015E000204500205A0020580020420020540020AE
:1015F000204D323035205300416476616E6365645E
:10160000207661726961626C65733A20533D4D6961
:101610006E20666565647261746520286D6D2F7338
:10162000292C20543D4D696E2074726176656C20C2
:10163000666565647261746520286D6D2F73292C51
:1016400020423D6D696E696D756D207365676D65CE
:101650006E742074696D6520286D73292C20583DA7
:101660006D6178696D756D205859206A65726B20BF
:10167000286D6D2F73292C20205A3D6D6178696D7E
:10168000756D205A206A65726B20286D6D2F732945
:101690002C2020453D6D6178696D756D2045206A6F
:1016A00065726B20286D6D2F732900205400202057
:1016B0004D323034205300416363656C6572617450
:1016C000696F6E3A20533D616363656C6572617446
:1016D000696F6E2C20543D72657472616374206171
:1016E0006363656C65726174696F6E0020450020EC
:1016F0005A0020590020204D3230312058004D61D1
:1017000078696D756D20416363656C65726174699C
:101710006F6E20286D6D2F7332293A00204500200E
:101720005A0020590020204D3230332058004D619E
:1017300078696D756D206665656472617465732086
:10174000286D6D2F73293A00204500205A0020593A
:101750000020204D3932205800537465707320707A
:10176000657220756E69743A0053657474696E67AA
:10177000732053746F72656400022D2D3A2D2D0075
:101780002D2D2D00534400012000012000012000D8
:101790004E6F2053442063617264005072696E740E
:1017A0002066726F6D2053440053746F7020707206
:1017B000696E7400526573756D65207072696E7420
:1017C000005061757365207072696E7400436F6EAE
:1017D00074726F6C00507265706172650054756E42
:1017E0006500496E666F2073637265656E00052E35
:1017F0002E004D61696E004D3234004D323320258C
:1018000073004D383420582059205A20450046692D
:10181000726D776172652076657273696F6E0052C2
:101820006573746F7265206661696C7361666500CB
:101830004C6F6164206D656D6F72790053746F72C7
:1018400065206D656D6F7279004D6F74696F6E0004
:1018500054656D7065726174757265004D61696E75
:101860000053657020313920323031342031303A24
:1018700032333A3031003131353230305F647561A6
:101880006C00556C74696D616B65723A2031342E51
:101890003038004669726D776172652076657273C3
:1018A000696F6E004573746570732F6D6D004573BD
:1018B000746570732F6D6D005A73746570732F6D3E
:1018C0006D005A73746570732F6D6D005973746574
:1018D00070732F6D6D005973746570732F6D6D008B
:1018E0005873746570732F6D6D00587374657073E1
:1018F0002F6D6D00412D7265747261637400412D0E
:101900007265747261637400416D61782065004195
:101910006D6178206500416D6178207A00416D61CC
:1019200078207A00416D6178207900416D617820DE
:101930007900416D6178207800416D6178207800F0
:101940005654726176206D696E005654726176202D
:101950006D696E00566D696E00566D696E00566D4C
:101960006178206500566D6178206500566D61785C
:10197000207A00566D6178207A00566D6178207962
:1019800000566D6178207900566D61782078005698
:101990006D617820780056652D6A65726B0056651A
:1019A0002D6A65726B00567A2D6A65726B00567AE5
:1019B0002D6A65726B005678792D6A65726B0056D8
:1019C00078792D6A65726B00416363656C004163D1
:1019D00063656C00436F6E74726F6C005072656863
:1019E0006561742041425320636F6E6600507265DA
:1019F0006865617420504C4120636F6E66005049E9
:101A0000442D43005049442D43005049442D440087
:101A10005049442D44005049442D49005049442D1B
:101A200049005049442D50005049442D5000466112
:101A30006E2073706565640046616E207370656525
:101A4000640042656400426564004E6F7A7A6C659A
:101A500032004E6F7A7A6C6532004E6F7A7A6C651E
:101A6000004E6F7A7A6C6500436F6E74726F6C0013
:101A700053746F7265206D656D6F72790042656495
:101A800000426564004E6F7A7A6C65004E6F7A7A18
:101A90006C650046616E2073706565640046616E1A
:101AA0002073706565640054656D7065726174754E
:101AB00072650053746F7265206D656D6F72790089
:101AC00042656400426564004E6F7A7A6C65004E30
:101AD0006F7A7A6C650046616E207370656564008C
:101AE00046616E2073706565640054656D70657243
:101AF0006174757265004D6F766520617869730059
:101B0000436F6F6C646F776E0050726568656174C7
:101B100020414253005072656865617420504C4109
:101B2000004D6F7665205A004175746F20686F6DA7
:101B300065004D38340044697361626C65207374CC
:101B4000657070657273004D61696E004D6F7665EA
:101B500020302E316D6D004D6F766520316D6D003A
:101B60004D6F76652031306D6D0050726570617219
:101B700065004578747275646572004D6F766520F6
:101B80005A004D6F76652059004D6F7665205800DC
:101B90004D6F76652061786973004578747275645D
:101BA0006572005A0059005800507265686561748A
:101BB000204142532042656400507265686561743B
:101BC0002041425320416C6C00507265686561741D
:101BD0002041425320320050726568656174204193
:101BE0004253203100507265706172650050726519
:101BF0006865617420504C412042656400507265F4
:101C00006865617420504C4120416C6C00507265D5
:101C10006865617420504C412032005072656865DF
:101C2000617420504C4120310050726570617265C2
:101C3000005A004D3834205830205930004732388F
:101C4000004D363030004368616E67652066696C10
:101C5000616D656E7400466C6F77203100466C6F65
:101C600077203100466C6F77203000466C6F77200C
:101C7000300046616E2073706565640046616E20B9
:101C800073706565640042656400426564004E6F70
:101C90007A7A6C6532004E6F7A7A6C6532004E6FDC
:101CA0007A7A6C65004E6F7A7A6C65005370656560
:101CB00064005370656564004D61696E0043617234
:101CC000642072656D6F766564004361726420699B
:101CD0006E73657274656400494E46494E495459A5
:101CE0004E414ECDCCCC3D0AD7233C17B7D13877E7
:101CF000CC2B329595E6241FB14F0A0000204100FD
:101D000000C84200401C4620BCBE4CCA1B0E5AAE46
:101D1000C59D7400A11A9B4144CF9A1A11241FBE7D
:101D2000CFEFD1E2DEBFCDBF00E00CBF14E0A0E0FA
:101D3000B2E0EEE9F0EC01E00BBF02C007900D92BB
:101D4000A03CB107D9F71BBE12E1A0ECB4E001C082
:101D50001D92A83AB107E1F71DE1CAE1DDE104C037
:101D60002297FE010E94F4DFC431D107C9F70E9417
:101D7000D4DA0C9442E00C940000A0E0B0E0E3EC74
:101D8000FEE00C9411E0EC015B016115710519F0A6
:101D9000FB0191838083F9908F2D90E00E94F8DF02
:101DA000892BC9F7FDE2FF1621F4F990EE24E394A4
:101DB00005C02BE2F21609F4F990EE248E010150D1
:101DC0001040C80168ED7CE143E050E00E945311EF
:101DD000892B01F58E010E5F1F4FC8016BED7CE171
:101DE00045E050E00E945311892B19F48E01095FE0
:101DF0001F4FA114B10419F0F50111830083E0FC19
:101E000004C070E090E080E814C070E090E080E8EA
:101E10006FEF08C1C80160EE7CE143E050E00E9432
:101E20005311892B69F4A114B10429F470E090E0F6
:101E300080EC6FE7F7C02296F501D183C083F6CF1F
:101E40008824992440E050E060E070E0EF2DE053FA
:101E5000EA30A0F5F2E0EF2A8E2D90E09C01287088
:101E60003070E2FE06C0232B79F50894811C911C8A
:101E70002BC0232B19F0089481089108DB01CA01BB
:101E800012E0880F991FAA1FBB1F1A95D1F7480FA0
:101E9000591F6A1F7B1F440F551F661F771F4E0F68
:101EA000511D611D711D483929E9520729E9620751
:101EB00029E1720748F084E0E82A06C0EE3F31F4D9
:101EC000E3FC39C098E0E92AF990C0CFE53311F07E
:101ED000E53189F529912D3219F4E0E1EE2A05C0AA
:101EE0002B3219F081E090E003C0299182E090E06C
:101EF000E22FE053EA3018F0C81BD90B1CC020E0D9
:101F000030E0FCE020383F075CF4C901880F991FDE
:101F1000880F991F280F391F220F331F2E0F311DD5
:101F2000E991E053EA3068F3E4FE03C0309521956F
:101F30003F4F820E931ECE2CDD24E1FE07C0A1147C
:101F4000B10421F02197F501D183C083CB01BA01FF
:101F50000E945DDC7B018C01F3E0CF22DD2423E0D5
:101F6000C216D10421F417FB109517F910955701EB
:101F70006801C801B70120E030E040E050E00E9475
:101F8000BDDB882309F44AC097FE0DC027EFE22E7F
:101F90002CE1F22E9094819491089394C0E2D0E0C9
:101FA00000E010E012C09FE0E92E9DE1F92EF6CF8F
:101FB000F7012591359145915491C601B5010E94D3
:101FC0009DDE5B016C018C1A9D0A8C169D0684F7C0
:101FD000D595C7950F5F1F4F0630110529F08CEF7F
:101FE0009FEFE80EF91EF1CFC501D6017C018D01EE
:101FF0008C2D880F8D2D881F8F3F51F0C601B501A4
:1020000020E030E040E050E00E94BDDB882331F466
:1020100082E290E09093A7128093A6127E2D9F2DCE
:10202000802F612F272F392F482F562FB901CA0132
:10203000CDB7DEB7ECE00C942DE02F923F925F928B
:102040006F927F928F929F92AF92BF92CF92DF92C8
:10205000EF92FF920F931F93CF93DF938C011B019D
:10206000EA016115710519F0FB01918380832097C6
:1020700049F0CE010297839728F020E030E040E05D
:1020800050E0F6C0F801A1908F018A2D90E00E94E7
:10209000F8DF892BB9F7FDE2AF1631F4F801A19012
:1020A0008F015524539407C0FBE2AF1619F4F801D1
:1020B000A1908F015524209719F0C031D105C1F4AA
:1020C000F0E3AF1679F4F8018081883711F0883594
:1020D00049F4F801A1800E5F1F4FF2E05F2AC0E1D2
:1020E000D0E006C0209721F480E3A816E9F427C0C9
:1020F000C830D10531F1C930D10524F4C230D10541
:1021000031F50CC0CA30D10589F0C031D105F9F4E0
:10211000C12CD12CE12CB8E0FB2E28C0C12CD12C35
:10212000E12CA0E4FA2E22C0CAE0D0E0FCECCF2ED5
:10213000FCECDF2EFCECEF2EFCE0FF2E17C0C8E01D
:10214000D0E0C12CD12CE12CE0E1FE2E0FC09E018D
:10215000442737FD4095542F60E070E080E090E820
:102160000E94B5DFC901DA016C017D0120E030E099
:1021700040E050E060E03E01882477FC8094982C99
:1021800070EDB72EBA0CE9E0EB1570F48A2D81548E
:102190008A3118F499ECB92E06C08A2D81568A31FD
:1021A00050F589EAB82EBA0C8B2D90E08C179D075C
:1021B00014F56F3FE1F0C216D306E406F506B0F061
:1021C000CA01B901A40193010E946FDF9B01AC0118
:1021D0002B0D311D411D511D2130F0E03F07F0E076
:1021E0004F07F0E85F0710F461E001C06FEFF801FE
:1021F000A1908F01C5CF2114310481F0662331F005
:1022000001501040F1011183008308C051FE1AC033
:1022100002501040F1011183008314C067FF12C007
:1022200050FC05C02FEF3FEF4FEF5FE704C020E009
:1022300030E040E050E882E290E09093A712809373
:10224000A61216C050FE08C05095409530952195B5
:102250003F4F4F4F5F4F0CC057FF0AC082E290E0E4
:102260009093A7128093A6122FEF3FEF4FEF5FE7F7
:10227000B901CA01DF91CF911F910F91FF90EF90AB
:10228000DF90CF90BF90AF909F908F907F906F9096
:102290005F903F902F900895FB01DC0105900D9217
:1022A0000020E1F70895FB01DC014150504088F027
:1022B0008D9181341CF08B350CF4805E6591613416
:1022C0001CF06B350CF4605E861B611171F3990B89
:1022D0000895881BFCCFFB01DC014150504048F0C1
:1022E00005900D920020C9F701C01D924150504049
:1022F000E0F70895FB0155915523A9F0BF01DC01DA
:102300004D9145174111E1F759F4CD010590002099
:1023100049F04D9140154111C9F3FB014111EFCF37
:1023200081E090E001970895FB01DC0104C08D91EC
:102330000190801921F441505040C8F7881B990B37
:102340000895FB01DC0102C001900D924150504004
:10235000D8F70895FB01DC010D900020E9F71197F3
:1023600001900D920020E1F70895FC0181918617FC
:1023700021F08823D9F7992708953197CF0108953F
:10238000FB01DC0101900D920020E1F70895FB01B3
:10239000DC014150504030F08D910190801919F4CA
:1023A0000020B9F7881B990B0895FB01DC0141500F
:1023B000504048F001900D920020C9F701C01D92D5
:1023C00041505040E0F70895AEE0B0E0EAEEF1E1B0
:1023D0000C9419E00E891F898EE08C831A8309837F
:1023E0008FEF9FE79E838D839E01265E3F4FCE0138
:1023F0000196688D798DA9010E9408122F81388578
:10240000020F131FF80110822E96E4E00C9435E0C1
:10241000ABE0B0E0EEE0F2E10C940BE03C012B010C
:102420005A01FC0117821682838181FD03C06FEF80
:102430007FEFC6C19AE0892E1E010894211C311C31
:10244000F3012381F20123FD859123FF81912F0167
:10245000882309F4B2C1853239F423FD859123FF25
:1024600081912F01853229F490E0B3010E94FB1382
:10247000E7CF982FFF24EE249924FFE1FF15D0F039
:102480009B3269F09C3228F4903259F0933291F4E7
:102490000EC09D3249F0903369F441E024C052E00F
:1024A000F52A84E0F82A28C098E0F92A25C0E0E15E
:1024B000FE2A22C0F7FC29C0892F80538A3070F48D
:1024C000F6FE05C0989C902C1124980E15C0E89C2F
:1024D000E02C1124E80EF0E2FF2A0EC09E3229F40F
:1024E000F6FC6BC140E4F42A07C09C3619F450E8AE
:1024F000F52A02C0983649F4F20123FD959123FF95
:1025000091912F01992309F0B8CF892F85548330F9
:1025100018F08052833038F444E050E0A40EB51E29
:102520005FE359830FC0933631F0933779F09335D9
:1025300009F056C020C0F5018081898342E050E057
:10254000A40EB51E610101E010E012C0F501C080CB
:10255000D180F6FC03C06FEF7FEF02C0692D70E001
:1025600042E050E0A40EB51EC6010E94F0138C019B
:102570005FE7F52214C0F501C080D180F6FC03C0EE
:102580006FEF7FEF02C0692D70E042E050E0A40ED3
:10259000B51EC6010E94E5138C0150E8F52AF3FE32
:1025A00007C01AC080E290E0B3010E94FB13EA94D6
:1025B0008E2D90E008171907A8F30EC0F601F7FC5E
:1025C0008591F7FE81916F0190E0B3010E94FB13AA
:1025D000E110EA94015010400115110579F7EAC0A5
:1025E000943611F0993669F5F7FE08C0F50120819F
:1025F00031814281538184E090E00AC0F5018081FD
:1026000091819C01442737FD4095542F82E090E052
:10261000A80EB91E9FE6F92257FF09C050954095B4
:10262000309521953F4F4F4F5F4FE0E8FE2ACA019A
:10263000B901A1012AE030E00E942714D82ED21857
:1026400040C0953729F41F2D1F7E2AE030E01DC0C1
:102650001F2D197F9F3661F0903720F4983509F0CF
:10266000ACC00FC0903739F0983709F0A6C004C04D
:1026700028E030E00AC0106114FD146020E130E071
:1026800004C014FD166020E132E017FF08C0F50118
:10269000608171818281938144E050E008C0F5013E
:1026A00080819181BC0180E090E042E050E0A40E86
:1026B000B51EA1010E942714D82ED2188FE7F82E3C
:1026C000F122F6FE0BC05EEFF522D91438F4F4FEC9
:1026D00007C0F2FC05C08FEEF82202C01D2D01C01C
:1026E000192DF4FE0DC0FE01ED0DF11D808180332A
:1026F00019F499EEF92208C01F5FF2FE05C003C06D
:102700008F2D867809F01F5F0F2DF3FC14C0F0FEAB
:102710000FC01E1510F09D2C0BC09D2C9E0C911A05
:102720001E2D06C080E290E0B3010E94FB131F5FE4
:102730001E15C0F304C01E1510F4E11A01C0EE24EA
:1027400004FF0FC080E390E0B3010E94FB1302FF7F
:102750001DC001FD03C088E790E00EC088E590E051
:102760000BC0802F867891F001FF02C08BE201C080
:1027700080E2F7FC8DE290E0B3010E94FB1306C0FB
:1027800080E390E0B3010E94FB139A94D914C0F344
:10279000DA94F101ED0DF11D808190E0B3010E940A
:1027A000FB13DD20A9F706C080E290E0B3010E9490
:1027B000FB13EA94EE20C1F743CEF30166817781E3
:1027C000CB012B96E2E10C9427E0FC0105906150CF
:1027D00070400110D8F7809590958E0F9F1F089537
:1027E000FC016150704001900110D8F780959095E0
:1027F0008E0F9F1F08950F931F93CF93DF938C012C
:10280000EB018B8181FF1BC082FF0DC02E813F81B8
:102810008C819D812817390764F4E881F98101933F
:10282000F983E88306C0E885F985802F1995892BFF
:1028300031F48E819F8101969F838E8302C00FEFBA
:102840001FEFC801DF91CF911F910F910895FA01F9
:10285000AA27283051F1203181F1E8946F936E7FDF
:102860006E5F7F4F8F4F9F4FAF4FB1E03ED0B4E0D0
:102870003CD0670F781F891F9A1FA11D680F791F11
:102880008A1F911DA11D6A0F711D811D911DA11D22
:1028900020D009F468943F912AE0269F1124301932
:1028A000305D3193DEF6CF010895462F4770405DCD
:1028B0004193B3E00FD0C9F7F6CF462F4F70405D7C
:1028C0004A3318F0495D31FD4052419302D0A9F7D7
:1028D000EACFB4E0A6959795879577956795BA95D1
:1028E000C9F700976105710508959B01AC010A2E97
:1028F00006945795479537952795BA95C9F7620F6E
:10290000731F841F951FA01D08951F920F920FB66D
:102910000F9211242F933F938F939F93AF93BF9365
:102920008091C4049091C504A091C604B091C704DD
:102930003091C8040196A11DB11D232F2D5F2D37A5
:1029400020F02D570196A11DB11D2093C80480933E
:10295000C4049093C504A093C604B093C7048091A7
:10296000C0049091C104A091C204B091C304019627
:10297000A11DB11D8093C0049093C104A093C20413
:10298000B093C304BF91AF919F918F913F912F91CD
:102990000F900FBE0F901F9018958FB7F89420914D
:1029A000C4043091C5044091C6045091C7048FBF40
:1029B000B901CA0108959B01AC017FB7F8948091D9
:1029C000C0049091C104A091C204B091C30466B543
:1029D000A89B05C06F3F19F00196A11DB11D7FBFD7
:1029E000BA2FA92F982F8827860F911DA11DB11DE1
:1029F00062E0880F991FAA1FBB1F6A95D1F7BC011F
:102A00002DC0FFB7F8948091C0049091C104A091AB
:102A1000C204B091C304E6B5A89B05C0EF3F19F00E
:102A20000196A11DB11DFFBFBA2FA92F982F88278E
:102A30008E0F911DA11DB11DE2E0880F991FAA1FE5
:102A4000BB1FEA95D1F7861B970B885E9340C8F2AF
:102A5000215030404040504068517C4F2115310595
:102A60004105510571F60895019739F0880F991FB6
:102A7000880F991F02970197F1F70895789484B50C
:102A8000826084BD84B5816084BD85B5826085BD6A
:102A900085B5816085BDEEE6F0E080818160808350
:102AA000E1E8F0E010828081826080838081816033
:102AB0008083E0E8F0E0808181608083E1EBF0E0FA
:102AC000808184608083E0EBF0E08081816080839E
:102AD000E1E9F0E080818260808380818160808391
:102AE000E0E9F0E0808181608083E1EAF0E08081CC
:102AF00082608083808181608083E0EAF0E0808171
:102B000081608083E1E2F1E0808182608083808166
:102B100081608083E0E2F1E0808181608083EAE788
:102B2000F0E0808184608083808182608083808106
:102B3000816080838081806880831092C1000895C5
:102B40001F93CF93DF93182FEB0161E00E94801653
:102B5000209709F4CAC0CF3FD10509F4C9C0E12FBD
:102B6000F0E0E75FFD4F8491893009F466C08A3058
:102B7000B0F48430F1F1853040F4823059F1833083
:102B800070F5813009F0AEC020C0873009F443C031
:102B9000883008F048C0863009F0A4C034C08D30B9
:102BA00009F478C08E3038F48B3009F45AC08C3078
:102BB00008F066C04CC0803109F480C0813109F44E
:102BC00087C08F3009F08EC06FC084B5806884BD27
:102BD000C7BD92C084B5806284BDC8BD8DC08091E0
:102BE0008000806880938000D0938900C093880023
:102BF00083C080918000806280938000D0938B009E
:102C0000C0938A0079C08091B00080688093B00042
:102C1000C093B30071C08091B00080628093B00017
:102C2000C093B40069C08091900080688093900048
:102C3000D0939900C09398005FC08091900080620B
:102C400080939000D0939B00C0939A0055C08091D0
:102C50009000886080939000D0939D00C0939C006A
:102C60004BC08091A00080688093A0008091A0005C
:102C70008F7B8093A000D093A900C093A8003CC094
:102C80008091A00080628093A000D093AB00C0939D
:102C9000AA0032C08091A00088608093A000D093E9
:102CA000AD00C093AC0028C0809120018068809363
:102CB0002001D0932901C09328011EC080912001DA
:102CC000806280932001D0932B01C0932A0114C00D
:102CD00080912001886080932001D0932D01C093C2
:102CE0002C010AC0C038D1051CF4812F60E002C05D
:102CF000812F61E00E943317DF91CF911F910895DA
:102D0000CF93DF93482F50E0CA018D539E4FFC01B3
:102D1000349143585E4FFA018491882369F190E021
:102D2000880F991FFC01E15DFE4FA591B491FC0154
:102D3000E75BFE4FC591D491662351F42FB7F89409
:102D40008C91932F909589238C93888189230BC034
:102D5000623061F42FB7F8948C91932F909589236A
:102D60008C938881832B88832FBF06C09FB7F894EC
:102D70008C91832B8C939FBFDF91CF9108958930E5
:102D800009F449C08A30A0F4843051F1853040F410
:102D9000823079F1833000F5813009F063C026C0BC
:102DA000873079F1883098F5863009F05BC025C00E
:102DB0008D3009F442C08E3028F48B30B1F18C3064
:102DC000C0F52DC0803109F442C0813109F445C0FD
:102DD0008F3009F047C037C0809180008F7703C0E3
:102DE000809180008F7D80938000089584B58F77D7
:102DF00002C084B58F7D84BD08958091B0008F7727
:102E000003C08091B0008F7D8093B00008958091C1
:102E100090008F7707C0809190008F7D03C08091D4
:102E20009000877F8093900008958091A0008F7715
:102E300007C08091A0008F7D03C08091A000877F94
:102E40008093A0000895809120018F7703C0809126
:102E500020018F7D80932001089580912001877F3C
:102E6000809320010895FF920F931F93F62E482F11
:102E700050E0CA01875F9D4FFC012491CA018D5328
:102E80009E4FFC01149143585E4FFA0104910023B8
:102E9000C9F0222319F0822F0E94BF16E02FF0E024
:102EA000EE0FFF1FE75BFE4FA591B4919FB7F8941B
:102EB000FF2021F48C911095812302C08C91812BED
:102EC0008C939FBF1F910F91FF9008950F931F93B5
:102ED000482F50E0CA01875F9D4FFC012491CA0131
:102EE0008D539E4FFC01049143585E4FFA0114919B
:102EF000112319F420E030E015C0222319F0822FAD
:102F00000E94BF16812F90E0880F991F8D599E4F08
:102F1000FC01A591B4918C9120E030E0802311F068
:102F200021E030E0C9011F910F9108951F920F9287
:102F30000FB60F920BB60F9211242F933F934F931E
:102F40005F936F937F938F939F93AF93BF93EF9311
:102F5000FF938091CD049091CE04892B29F0E091CC
:102F6000CD04F091CE041995FF91EF91BF91AF91EF
:102F70009F918F917F916F915F914F913F912F9191
:102F80000F900BBE0F900FBE0F901F9018951F92C1
:102F90000F920FB60F920BB60F9211242F933F93FF
:102FA0004F935F936F937F938F939F93AF93BF9351
:102FB000EF93FF938091CF049091D004892B29F057
:102FC000E091CF04F091D0041995FF91EF91BF915A
:102FD000AF919F918F917F916F915F914F913F91B1
:102FE0002F910F900BBE0F900FBE0F901F90189552
:102FF0001F920F920FB60F920BB60F9211242F93C0
:103000003F934F935F936F937F938F939F93AF9370
:10301000BF93EF93FF938091D1049091D204892BB9
:1030200029F0E091D104F091D2041995FF91EF912C
:10303000BF91AF919F918F917F916F915F914F91D0
:103040003F912F910F900BBE0F900FBE0F901F90CE
:1030500018951F920F920FB60F920BB60F92112474
:103060002F933F934F935F936F937F938F939F9390
:10307000AF93BF93EF93FF938091D3049091D404C7
:10308000892B29F0E091D304F091D4041995FF9194
:10309000EF91BF91AF919F918F917F916F915F91D0
:1030A0004F913F912F910F900BBE0F900FBE0F903D
:1030B0001F9018951F920F920FB60F920BB60F929A
:1030C00011242F933F934F935F936F937F938F932D
:1030D0009F93AF93BF93EF93FF938091C904909117
:1030E000CA04892B29F0E091C904F091CA0419950A
:1030F000FF91EF91BF91AF919F918F917F916F91D0
:103100005F914F913F912F910F900BBE0F900FBE8B
:103110000F901F9018951F920F920FB60F920BB63B
:103120000F9211242F933F934F935F936F937F934D
:103130008F939F93AF93BF93EF93FF938091CB04B3
:103140009091CC04892B29F0E091CB04F091CC0430
:103150001995FF91EF91BF91AF919F918F917F91C1
:103160006F915F914F913F912F910F900BBE0F90F8
:103170000FBE0F901F9018951F920F920FB60F92CF
:103180000BB60F9211242F933F934F935F936F933E
:103190007F938F939F93AF93BF93EF93FF93809110
:1031A000D5049091D604892B29F0E091D504F091B3
:1031B000D6041995FF91EF91BF91AF919F918F9197
:1031C0007F916F915F914F913F912F910F900BBE27
:1031D0000F900FBE0F901F9018951F920F920FB671
:1031E0000F920BB60F9211242F933F934F935F933F
:1031F0006F937F938F939F93AF93BF93EF93FF93BF
:103200008091D7049091D804892B29F0E091D704BC
:10321000F091D8041995FF91EF91BF91AF919F91D3
:103220008F917F916F915F914F913F912F910F906F
:103230000BBE0F900FBE0F901F901895CF92DF928C
:10324000EF92FF920F931F93CF93DF937C016B015B
:103250008A01C0E0D0E00FC0D6016D916D01D701A9
:10326000ED91FC910190F081E02DC7011995C80FF7
:10327000D91F015010400115110571F7CE01DF91E2
:10328000CF911F910F91FF90EF90DF90CF90089515
:10329000DC01ED91FC910190F081E02D19950895EC
:1032A000CF93DF93EC016115710519F420E030E054
:1032B0000FC0DB010D900020E9F71197A61BB70B9B
:1032C000E881F9810280F381E02DAD0119959C011F
:1032D000C901DF91CF9108950E9450190895EF928E
:1032E000FF920F931F93CF93DF93EC01E090880739
:1032F000F090890700918A0710918B076881798186
:103300008A819B81A80197010E94BDDB882324F458
:10331000E882F9820A831B83E0908C07F0908D0786
:1033200000918E0710918F076C817D818E819F8126
:10333000A80197010E94BDDB882324F4EC82FD8262
:103340000E831F83E0909007F09091070091920701
:1033500010919307688579858A859B85A8019701D7
:103360000E94BDDB882324F4E886F9860A871B8740
:10337000E0909303F09094030091950310919603CD
:10338000688179818A819B81A80197010E94CBDDA8
:10339000181624F4E882F9820A831B83E0909703CD
:1033A000F09098030091990310919A036C817D81AC
:1033B0008E819F81A80197010E94CBDD181624F40D
:1033C000EC82FD820E831F83E0909B03F0909C03B0
:1033D00000919D0310919E03688579858A859B8560
:1033E000A80197010E94CBDD181624F4E886F9861F
:1033F0000A871B87DF91CF911F910F91FF90EF906C
:1034000008958091B607089567707070E82FF0E016
:10341000E75FFD4F84918B3028F48830A0F486302C
:1034200090F106C08E30D0F08F50833060F521C00F
:103430008091B100887F8093B1008091B100862B8C
:103440008093B100089580919100887F80939100CE
:1034500080919100862B8093910008958091A10026
:10346000887F8093A1008091A100862B8093A1008A
:10347000089580912101887F80932101809121010D
:10348000862B8093210108950F931F93CF93DF9391
:103490008130910549F46F5F7F4F09F046C089ED97
:1034A00094E00E94C38C41C0892B09F03EC06F5F3D
:1034B0007F4FD9F586E394E09093A4068093A3060A
:1034C0008091AA06882321F087EA96E00E9480472F
:1034D000CFE5D6E006E314E005C06F9785E0C9327A
:1034E000D80751F0198308838F818823B1F3CE0167
:1034F00004960E948047F1CF86E394E09983888305
:103500008F81882321F0CE0104960E94804786E3B4
:1035100094E0909309058093080580910F05882316
:1035200021F08CE095E00E948047DF91CF911F91C0
:103530000F91089580E090E06FEF7FEF0E94441AB2
:10354000089581E090E06FEF7FEF0E94441A0895A4
:103550000E948B738091B607882309F03AC081E0FE
:103560008093B6078091B9079091BA07A091BB07E5
:10357000B091BC078093BD079093BE07A093BF078F
:10358000B093C007E5E5F2E0949108C08091C000D7
:1035900085FFFCCF9093C600319694919923B1F7A3
:1035A000E6E6F2E0949108C08091C00085FFFCCF70
:1035B0009093C600319694919923B1F78091C00001
:1035C00085FFFCCF8AE08093C6008CE592E00E94E4
:1035D00081CF0895F8940E948B73159A10929407E6
:1035E000469A10929507439A10929607409A8FB781
:1035F000F89490910B01926090930B018FBFE5E5D9
:10360000F2E0949108C08091C00085FFFCCF9093B8
:10361000C600319694919923B1F7E5EEF2E09491CA
:1036200008C08091C00085FFFCCF9093C600319602
:1036300094919923B1F78091C00085FFFCCF8AE077
:103640008093C6008CED92E00E9490CFFFCF0E9445
:10365000CD146093C1077093C2078093C307909302
:10366000C407E091EA07F091EB07E451F84F80813D
:103670008823A9F4E4E0F3E0949108C08091C000AD
:1036800085FFFCCF9093C600319694919923B1F7B2
:103690008091C00085FFFCCF8AE08093C60008952A
:1036A0000E94CD146093C1077093C2078093C30733
:1036B0009093C4070895EF92FF920F931F930E9477
:1036C000CD14E090C507F090C6070091C707109190
:1036D000C8072091C1073091C2074091C30750919C
:1036E000C407621B730B840B950BE616F7060807DD
:1036F000190738F4E114F1040105110511F00E94D5
:10370000EA1A8091A1039091A203A091A303B09122
:10371000A4030097A105B10599F10E94CD14209151
:10372000C1073091C2074091C3075091C407621B83
:10373000730B840B950B2091A1033091A203409150
:10374000A3035091A4032617370748075907C0F46D
:103750009091551180915611981791F4159A1092E5
:103760009407469A10929507439A10929607409AAA
:103770009FB7F89480910B01826080930B019FBFEB
:103780000E94615A1F910F91FF90EF9008956F92E0
:103790007F928F929F92AF92BF92CF92DF92EF92E1
:1037A000FF920F931F93F82E6091C9077091CA077B
:1037B0008091CB079091CC072091CD073091CE0717
:1037C0004091CF075091D0070E94D8DD3B014C01BA
:1037D00000D000D00DB71EB70F5F1F4F609183035D
:1037E00070918403882777FD8095982F0E945FDC75
:1037F0002091A5033091A6034091A7035091A803FF
:103800000E949DDE20E030E040E752E40E94C4DBED
:1038100020E030E048EC52E40E94C4DB5B016C0124
:10382000F8016082718282829382F4828091AB0778
:1038300085838CE697E065ED77E049EC57E020E082
:1038400001E032E0E32E0E9461548091D50790910F
:10385000D607A091D707B091D80780936C079093B3
:103860006D07A0936E07B0936F078091D907909171
:10387000DA07A091DB07B091DC0780937007909383
:103880007107A0937207B09373078091DD07909141
:10389000DE07A091DF07B091E00780937407909353
:1038A0007507A0937607B09377078091E107909111
:1038B000E207A091E307B091E40780937807909323
:1038C0007907A0937A07B0937B078DB79EB70696CA
:1038D0000FB6F8949EBF0FBE8DBF0E94CD146093AB
:1038E000C1077093C2078093C3079093C4071F91C9
:1038F0000F91FF90EF90DF90CF90BF90AF909F908F
:103900008F907F906F900895CF92DF92EF92FF9209
:103910000F931F9385ED97E00E946F190E94CD14BD
:103920006093C1077093C2078093C3079093C40745
:1039300060916C0770916D0780916E0790916F0791
:103940002091D5073091D6074091D7075091D807DD
:103950000E94BDDB882309F07AC0609170077091E6
:10396000710780917207909173072091D907309168
:10397000DA074091DB075091DC070E94BDDB88230A
:1039800009F065C06091A5037091A6038091A7031B
:103990009091A80320E030E040E752E40E94C4DBAD
:1039A0007B018C0185ED97E069ED77E04DED57E007
:1039B00021EE37E0EBEACE2EE7E0DE2E0E94485DF6
:1039C0008091D5079091D607A091D707B091D807DD
:1039D00080936C0790936D07A0936E07B0936F0769
:1039E0008091D9079091DA07A091DB07B091DC07AD
:1039F0008093700790937107A0937207B093730739
:103A00008091DD079091DE07A091DF07B091E0077C
:103A10008093740790937507A0937607B093770708
:103A20008091E1079091E207A091E307B091E4074C
:103A30008093780790937907A0937A07B0937B07D8
:103A40001F910F91FF90EF90DF90CF9008956091BC
:103A5000830370918403882777FD8095982F0E94B7
:103A60005FDC2091A5033091A6034091A7035091FC
:103A7000A8030E949DDE20E030E040E752E40E946F
:103A8000C4DB20E030E048EC52E488CF87E09AE0E5
:103A90000E949241E7E0F3E0949108C08091C00059
:103AA00085FFFCCF9093C600319694919923B1F78E
:103AB0004091B9075091BA076091BB077091BC075C
:103AC0004F5F5F4F6F4F7F4F87E09AE02AE030E013
:103AD0000E9453428091C00085FFFCCF8AE0809312
:103AE000C6000E94271B08952F923F924F925F922B
:103AF0006F927F928F929F92AF92BF92CF92DF92FE
:103B0000EF92FF920F931F93DF93CF93CDB7DEB762
:103B100028970FB6F894DEBF0FBECDBF98878F836E
:103B20008330910508F056C1FC01E15BFA4FD49057
:103B30003C01660C771C660C771C93012459384FA6
:103B40003A83298380E090E0A0E0B0E0F90180832F
:103B50009183A283B3838CE697E060E777E044E744
:103B600057E028E737E00E943958F301EE5AFA4F40
:103B7000E590F590059114916D2D772767FD70956F
:103B8000882777FD8095982F0E945FDC1B012C0110
:103B900093012B52384F3C832B83C801B70120E09F
:103BA00030E040EC5FE30E949DDEA20191010E94A3
:103BB0009DDEAB81BC816D937D938D939C93139718
:103BC000F301ED58FC4FFE83ED83608171818281AA
:103BD00093816093A5037093A6038093A7039093AA
:103BE000A80320E030E040E752E40E94C4DB7B0100
:103BF0008C0185ED97E069ED77E04DED57E021EE22
:103C000037E0ABEACA2EA7E0DA2E0E94485D0E9498
:103C1000576B80E090E0A0E0B0E0E981FA8180831A
:103C20009183A283B3838CE697E060E777E044E773
:103C300057E028E737E00E943958F301EE57FA4F72
:103C400085909590A590B490C501B4019058A201BB
:103C500091010E949DDEAB81BC816D937D938D931C
:103C60009C9313976091A5037091A6038091A7037D
:103C70009091A80320E030E040E752E40E94C4DBCA
:103C80007B018C0185ED97E069ED77E04DED57E024
:103C900021EE37E00E94485D0E94576BC501B401D8
:103CA000A50194010E94E4DAA20191010E949DDE27
:103CB000EB81FC816083718382839383AD81BE81BC
:103CC0006D917D918D919C9120E030E040E05FE32B
:103CD0000E949DDE6093A5037093A6038093A703C3
:103CE0009093A80320E030E040E752E40E94C4DB58
:103CF0007B018C0185ED97E069ED77E04DED57E0B4
:103D000021EE37E00E94485D0E94576BF301E25AB2
:103D1000FA4F6591759185919491F301E458F84FAC
:103D2000A080B180C280D380A60195010E94E4DA10
:103D30007B018C01CB01D801E981FA8180839183D9
:103D4000A283B383F301E659FA4F6591759185918A
:103D50009491F8E88F2EF7E09F2E860C971CA60111
:103D600095010E94E4DAD4016D937D938D939C9329
:103D70001397F301EA58FA4F6591759185919491E3
:103D8000E3E9F3E06E0E7F1EA60195010E94E4DADE
:103D9000D3016D937D938D939C931397C701D801A5
:103DA000EB81FC8180839183A283B38380E090E0E8
:103DB000A0E0B0E08093A5039093A603A093A7038F
:103DC000B093A8030E94D369AF81B885AC56B84FB1
:103DD00081E08C9328960FB6F894DEBF0FBECDBF5E
:103DE000CF91DF911F910F91FF90EF90DF90CF90D7
:103DF000BF90AF909F908F907F906F905F904F900B
:103E00003F902F900895682F2091EA073091EB079B
:103E100080E690E0AC01249FC001259F900D349F67
:103E2000900D11248A50984F70E00E94B5119C01AA
:103E30009093F5078093F40780E0232B09F081E04D
:103E40000895FC01949108C08091C00085FFFCCFCB
:103E50009093C600319694919923B1F787E09AE048
:103E600022E030E00E9463430895FC01949108C071
:103E70008091C00085FFFCCF9093C600319694914D
:103E80009923B1F787E09AE02AE030E00E943442BB
:103E900008958091F4079091F507019660E070E035
:103EA0004AE050E00E941D1008958091F40790911F
:103EB000F507019660E070E00E94BD0E0895CF9373
:103EC000DF93EC018091AB078093B80784E50E94F3
:103ED000031F882309F482C00E94551F0E9431DC11
:103EE000262F6093B807623008F478C0EFE4F2E060
:103EF000949108C08091C00085FFFCCF9093C600CC
:103F0000319694919923B1F7CD36D105C1F0CE36D3
:103F1000D10544F4C836D105C1F0C936D10509F040
:103F20004DC010C0CA3DD10539F0CD3DD10509F0D5
:103F300045C0E0E0F2E03FC0E7E1F2E031C0EEE290
:103F4000F2E023C0E5E4F2E015C0ECE5F2E007C0E2
:103F50008091C00085FFFCCF31969093C600908180
:103F60009923B1F72BC08091C00085FFFCCF31961B
:103F70009093C60090819923B1F720C08091C00032
:103F800085FFFCCF31969093C60090819923B1F7BD
:103F900015C08091C00085FFFCCF31969093C6007C
:103FA00090819923B1F70AC08091C00085FFFCCFB2
:103FB00031969093C60090819923B1F787E09AE0FB
:103FC000622F40E050E00E9441428091C00085FF96
:103FD000FCCF8AE08093C60081E001C080E0DF91E1
:103FE000CF910895AF92BF92CF92DF92EF92FF925E
:103FF0000F931F93CF93DF931CE6E12E17E0F12E72
:10400000C5EDD7E000E010E0F801E251FC4F8081FF
:104010000E94031F882339F10E94551F5B016C0128
:10402000F801EA59F84F8081882311F061E002C05D
:104030006091E50770E0882777FD8095982F0E94B2
:104040005FDCF70120813181428153810E949DDE36
:104050009B01AC01C601B5010E94E4DA6883798353
:104060008A839B8309C0F70180819181A281B381FA
:1040700088839983AA83BB830F5F1F4F84E090E0FE
:10408000E80EF91E24960430110509F0BDCF86E430
:104090000E94031F8823E1F00E94551F7B018C01C1
:1040A0006093E6077093E7078093E8079093E9072A
:1040B00020E030E040E050E00E94CBDD181644F4F0
:1040C000E092A503F092A6030093A7031093A80320
:1040D000DF91CF911F910F91FF90EF90DF90CF90E4
:1040E000BF90AF9008950E94F21F89E40E94031FC1
:1040F000882359F00E94551F6093C9077093CA071F
:104100008093CB079093CC070CC080E090E0A0E0B8
:10411000B0E08093C9079093CA07A093CB07B093F0
:10412000CC078AE40E94031F882359F00E94551F80
:104130006093CD077093CE078093CF079093D007FD
:10414000089580E090E0A0E0B0E08093CD079093E8
:10415000CE07A093CF07B093D00708952F923F9238
:104160004F925F926F927F928F929F92AF92BF9287
:10417000CF92DF92EF92FF920F931F93DF93CF9333
:10418000CDB7DEB7EE970FB6F894DEBF0FBECDBF4A
:1041900087E40E94031F882309F44EC40E94551F20
:1041A0000E942CDC6430710509F441C06530710552
:1041B00054F46230710541F1633071056CF5772379
:1041C000CCF40C9477396A35710509F4E0C36B358A
:1041D000710534F46C31710511F00C9477396FC0AE
:1041E0006B35710509F4D7C36C35710511F00C946A
:1041F0007739D6C38091B607882331F40E94F21F25
:104200000E94841C0C949E398091B607882321F467
:104210000E94732081E007C08091B607882339F49B
:104220000E94732080E00E94C71B0C949E3986E494
:1042300095E00E9481CF80E50E94031F882321F42E
:10424000EE24FF24870106C00E94551F0E9431DC26
:104250007B018C0183E50E94031F882361F00E948B
:10426000551F20E030E04AE754E40E949DDE0E94A2
:1042700031DC7B018C010E94576B0E94CD145B01E5
:104280006C01AE0CBF1CC01ED11E0E94CD146093E9
:10429000C1077093C2078093C3079093C40706C0F9
:1042A0000E94EE780E945B1B0E94B3CF0E94CD1447
:1042B0006A157B058C059D0598F30C9477398091E0
:1042C000A5039091A603A091A703B091A8038093A2
:1042D000F0079093F107A093F207B093F307809152
:1042E00083039091840390936B0780936A0784E61D
:1042F00090E090938403809383030E94CD14609395
:10430000C1077093C2078093C3079093C40781E0ED
:104310000E94DA6980916C0790916D07A0916E07F9
:10432000B0916F078093D5079093D607A093D707D6
:10433000B093D8078091700790917107A091720790
:10434000B09173078093D9079093DA07A093DB07A6
:10435000B093DC078091740790917507A091760760
:10436000B09177078093DD079093DE07A093DF0776
:10437000B093E0078091780790917907A0917A0730
:10438000B0917B078093E1079093E207A093E30746
:10439000B093E40780E090E0A0E0B0E08093A50354
:1043A0009093A603A093A703B093A80388E50E9467
:1043B000031F882361F489E50E94031F882339F4D1
:1043C0008AE50E94031F882311F481E001C080E088
:1043D0008093A903882361F488E50E94031F882342
:1043E00009F41BC289E50E94031F882309F415C242
:1043F00080E090E0A0E0B0E080936C0790936D07C0
:10440000A0936E07B0936F07809370079093710726
:10441000A0937207B0937307BFE48B2EB5E09B2E79
:10442000F401E4908CE697E060E777E044E757E03A
:1044300028E737E00E943958A2E56A2EA5E07A2ED7
:10444000F301659175918591949120E030E040EC05
:104450005FE30E949DDE5B016C01FF24E7FCF094AA
:104460000027F7FC0095102FC801B7010E945FDC00
:104470009B01AC01C601B5010E949DDE6093D5078A
:104480007093D6078093D7079093D807F4E04F2E08
:10449000512C460C571CF2016591759185919491B0
:1044A0000894811C911CF401D49020E030E040EC91
:1044B0005FE30E949DDE7B018C016D2D772767FDF8
:1044C0007095872F972F0E945FDC9B01AC01C8017C
:1044D000B7010E949DDE6093D9077093DA0780933D
:1044E000DB079093DC0720917303309174034091B4
:1044F0007503509176032093A5033093A603409350
:10450000A7035093A803E0907703F09078030091FD
:10451000790310917A03C801B7010E94BDDB88239B
:1045200044F4E092A503F092A6030093A70310932E
:10453000A803F301A590B590C590D490F201E59041
:10454000F59005911491C601B501A80197010E944B
:10455000CBDD18162CF4C801B701A601950104C0E3
:10456000C601B501A80197010E94C4DB9B01AC0103
:104570000E949DDE9B01AC01CA0120E030E040E8D2
:104580005FE30E94E4DA0E940ADF9B01AC016091C4
:10459000A5037091A6038091A7039091A8030E94A0
:1045A0009DDE6093A5037093A6038093A703909369
:1045B000A8036091A5037091A6038091A703909131
:1045C000A80320E030E040E752E40E94C4DB7B0116
:1045D0008C0185ED97E069ED77E04DED57E021EE38
:1045E00037E0EBEACE2EE7E0DE2E0E94485D0E9427
:1045F000576BEEE5F5E06591759185919491209169
:104600007C0730917D0740917E0750917F070E9483
:10461000E4DA60936C0770936D0780936E07909354
:104620006F07EAE6F5E06591759185919491209187
:104630007C0730917D0740917E0750917F070E9453
:10464000E4DA609388077093890780938A079093D0
:104650008B07E6E7F5E0659175918591949120913E
:104660007C0730917D0740917E0750917F070E9423
:10467000E4DA60939303709394038093950390938B
:104680009603E2E6F5E0659175918591949120910C
:1046900080073091810740918207509183070E94E3
:1046A000E4DA6093700770937107809372079093B8
:1046B0007307EEE6F5E065917591859194912091EF
:1046C00080073091810740918207509183070E94B3
:1046D000E4DA60938C0770938D0780938E07909334
:1046E0008F07EAE7F5E065917591859194912091A6
:1046F00080073091810740918207509183070E9483
:10470000E4DA6093970370939803809399039093EE
:104710009A038CE697E060E777E044E757E028E704
:1047200037E00E94395880916C0790916D07A091F5
:104730006E07B0916F078093D5079093D607A0932B
:10474000D707B093D8078091700790917107A09117
:104750007207B09173078093D9079093DA07A093FB
:10476000DB07B093DC076091A5037091A6038091ED
:10477000A7039091A80320E030E040E752E40E94B4
:10478000C4DB7B018C0185ED97E069ED77E04DEDB1
:1047900057E021EE37E00E94485D80E090E0A0E025
:1047A000B0E08093A5039093A603A093A703B093D2
:1047B000A8030E94576B0E94D3698091D5079091FE
:1047C000D607A091D707B091D80780936C07909334
:1047D0006D07A0936E07B0936F078091D9079091F2
:1047E000DA07A091DB07B091DC0780937007909304
:1047F0007107A0937207B09373078091DD079091C2
:10480000DE07A091DF07B091E007809374079093D3
:104810007507A0937607B09377078091A903882343
:1048200029F488E50E94031F882321F080E090E0AE
:104830000E94741D8091A903882329F489E50E94B0
:10484000031F882321F081E090E00E94741D88E519
:104850000E94031F8823D9F00E94491F611571052A
:1048600081059105A1F00E94551F20917C07309190
:104870007D0740917E0750917F070E94E4DA6093A4
:104880006C0770936D0780936E0790936F0789E5AF
:104890000E94031F8823D9F00E94491F61157105EA
:1048A00081059105A1F00E94551F2091800730914C
:1048B000810740918207509183070E94E4DA609358
:1048C00070077093710780937207909373078091BC
:1048D000A903882329F48AE50E94031F882321F075
:1048E00082E090E00E94741D8AE50E94031F8823E5
:1048F000D9F00E94491F6115710581059105A1F04C
:104900000E94551F209184073091850740918607AA
:10491000509187070E94E4DA6093740770937507DB
:1049200080937607909377078CE697E060E777E0CF
:1049300044E757E028E737E00E94395880E00E94BA
:10494000DA698091F0079091F107A091F207B09198
:10495000F3078093A5039093A603A093A703B093B6
:10496000A80380916A0790916B07909384038093CA
:1049700083030E94CD146093C1077093C207809394
:10498000C3079093C4070E94D3690C94773910929F
:10499000E5070C94773981E08093E5070C9477392B
:1049A00085E40E94031F882311F40E94576B4CE694
:1049B000E42E47E0F42E3CE7C32E37E0D32E00E090
:1049C00010E0F801E251FC4F80810E94031F882310
:1049D00031F1033061F40E94551FF7016083718348
:1049E0008283938388E797E00E941B5818C00E9437
:1049F000551FF60120813181428153810E94E4DA02
:104A0000F70160837183828393838CE697E060E78C
:104A100077E044E757E028E737E00E9439580F5F16
:104A20001F4F24E030E0E20EF31EC20ED31E04300E
:104A3000110539F60C9477398DE40E94031F882301
:104A400011F40C941B380E94551F0E942CDC633714
:104A5000710511F40C94242F643771050CF096C085
:104A60006F31710509F487C3603271050CF041C0E4
:104A70006631710509F4F4C167317105E4F46131FF
:104A8000710509F4A5C16231710534F46230710514
:104A900010F00C9477393DC16431710509F4AAC155
:104AA000653171050CF0D6C16231710511F00C94BD
:104AB00077390C941E2E6A31710509F409C26B31E5
:104AC00071054CF46831710509F4ECC16931710567
:104AD0000CF0F8C1CBC16C31710509F41EC26C3108
:104AE00071050CF414C26E31710511F00C94773914
:104AF00051C26535710511F40C94872E6635710528
:104B0000F4F46135710511F40C94F22D62357105E0
:104B100054F46032710509F483C26A32710511F0F0
:104B20000C947739ADC36335710511F40C94192ECB
:104B30006435710514F00C941E2E0C94152E6A36F3
:104B4000710511F40C94BB2D6B3671057CF468363D
:104B5000710509F4DFC3693671050CF00CC46C35BE
:104B6000710511F00C9477390C949E2E6D367105F9
:104B700009F43EC56237710511F40C944B2F6B3666
:104B8000710511F00C9477390C94EC2D6D3D710585
:104B900011F40C94E9326E3D71050CF054C0683C80
:104BA000710511F40C94D230693C710514F5683725
:104BB000710511F40C944030693771055CF4653768
:104BC000710511F40C94342F6737710511F00C94B2
:104BD00077399BC06C38710509F4BCC36E3B710515
:104BE00009F4B6C66937710511F00C9477390C9445
:104BF00045306D3C710511F40C94B0316E3C71057B
:104C00008CF46B3C710511F40C946F316C3C7105A4
:104C100014F00C948E31693C710511F00C947739C5
:104C20000C944C316A3D710511F40C942C326C3D9E
:104C3000710511F40C94DA326E3C710511F00C948C
:104C400077390C940E3231E0653F730711F40C9400
:104C5000953441E0663F74074CF551E06E327507BC
:104C600011F40C94403481E06F32780764F4623EB2
:104C7000710511F40C9410336D52714011F00C94C5
:104C800077390C946833E1E060397E0711F40C94B5
:104C90008F34F1E0643F7F0711F40C9492346F522B
:104CA000714011F00C9477390C944F3433E0633534
:104CB000730711F40C949E3443E0643574079CF43C
:104CC00051E0673F750711F40C949B3481E0673F16
:104CD000780714F40C9498346855724011F00C94D1
:104CE00077390C94A335E3E0603A7E0709F408C2F3
:104CF000F3E0673E7F0711F40C9404386B5873405F
:104D000011F00C9477390C94D537E3E7F2E00C946A
:104D1000513085E395E00E9481CF80E50E94031F1A
:104D2000882321F4EE24FF24870106C00E94551F2A
:104D30000E9431DC7B018C0183E50E94031F8823E4
:104D400061F00E94551F20E030E04AE754E40E94E1
:104D50009DDE0E9431DC7B018C010E94576B0E941A
:104D6000CD146093C1077093C2078093C3079093DB
:104D7000C407E114F1040105110501F10E94CD14ED
:104D80005B016C01AE0CBF1CC01ED11E0E94CD1475
:104D90006A157B058C059D05A8F40E943C97882325
:104DA00089F40E94EE780E945B1B0E94B3CFEECF85
:104DB0000E94EE780E945B1B0E94B3CF0E943C973A
:104DC0008823B1F386E295E00E9481CF0C94773975
:104DD0008DE195E00E9481CF1598469843984098C0
:104DE0009FB7F89480910B018D7F80930B019FBF3B
:104DF0000C947739EDE0F5E0949108C08091C00003
:104E000085FFFCCF9093C600319694919923B1F71A
:104E10008091C00085FFFCCF8AE08093C60089EDB9
:104E200094E00E94768CEFEFF4E0949108C08091BA
:104E3000C00085FFFCCF9093C600319694919923D2
:104E4000B1F78091C00085FFFCCF8AE08093C60057
:104E50000C94773989ED94E00E94D5870C947739CA
:104E600089ED94E00E940D800C9477398091F407CD
:104E70009091F50704966AE270E00E94B511FC017A
:104E8000009711F0319710826091F4077091F50747
:104E90006C5F7F4F89ED94E041E021E00E94EB835D
:104EA0000C94773989ED94E00E9411800E94CD1412
:104EB0006093AE077093AF078093B0079093B107EC
:104EC0000C94773989ED94E00E9418800C9477391E
:104ED0008091DC04882311F40C94773983E50E94D7
:104EE000031F882311F40C9477390E94491FAB01EA
:104EF000BC0140935C0750935D0780935E077093FD
:104F00005F0787EA96E00E9466460C94773989ED40
:104F100094E00E94D6810C9477398091F4079091A7
:104F2000F50704966AE270E00E94B5118C010097C3
:104F300019F12091EA073091EB0780E690E0AC018F
:104F4000249FC001259F900D349F900D11248A50FD
:104F5000984F6EE470E00E94B51160E270E00E942C
:104F6000B5119C012F5F3F4F3093F5072093F40755
:104F700001501040F80110826091F4077091F5071C
:104F80006C5F7F4F89ED94E040E021E00E94EB836D
:104F90000C9477398091DC04882311F40C947739D0
:104FA00089ED94E060E00E9445818091F407909142
:104FB000F50704966AE270E00E94B5118C01009733
:104FC00019F12091EA073091EB0780E690E0AC01FF
:104FD000249FC001259F900D349F900D11248A506D
:104FE000984F6EE470E00E94B51160E270E00E949C
:104FF000B5119C012F5F3F4F3093F5072093F407C5
:1050000001501040F80110826091F4077091F5078B
:105010006C5F7F4F89ED94E00E9430820C94773969
:105020008091DB04882311F00E94576BE090F40715
:10503000F090F50724E030E0E20EF31EC7016AE2CB
:1050400070E00E94B5118C01C70161E270E00E941E
:10505000B511009721F07C010894E11CF11C0115A9
:10506000110521F001501040F801108280E50E94E6
:10507000031F182F8091F4079091F507E816F906A1
:1050800008F410E08091DC04882311F40C94773943
:1050900021E0212789ED94E0B70141E00E94EB83F4
:1050A00083E50E94031F8823B9F08091F407909153
:1050B000F5078E159F0580F40E94491FAB01BC01C6
:1050C00040935C0750935D0780935E0770935F0782
:1050D00087EA96E00E94664689ED94E00E9411807E
:1050E000112311F00C9477390E94CD146093AE0710
:1050F0007093AF078093B0079093B1070C94773902
:105100008091F4079091F50705966AE270E00E949D
:10511000B5118C01009719F12091EA073091EB0746
:1051200080E690E0AC01249FC001259F900D349F44
:10513000900D11248A50984F6EE470E00E94B511D2
:1051400060E270E00E94B5119C012F5F3F4F3093E9
:10515000F5072093F40701501040F8011082609188
:10516000F4077091F5076B5F7F4F89ED94E00E9423
:10517000CC870C9477390E94CD146093B20770935A
:10518000B3078093B4079093B5072091AE07309191
:10519000AF074091B0075091B107621B730B840BAE
:1051A000950B28EE33E040E050E00E94B5DFF22E90
:1051B000E32ED42EC52E2DB73EB7285030400FB663
:1051C000F8943EBF0FBE2DBF0DB71EB70F5F1F4F28
:1051D000CE018196EDB7FEB79283818380EF94E094
:1051E000F801938382836F2D7E2D842F952F2CE3DE
:1051F00030E040E050E00E94B5DFF80135832483C1
:105200006F2D7E2D8D2D9C2D2CE330E040E050E065
:105210000E94B5DFF801778366830E94E411EFE412
:10522000F2E094912DB73EB7285F3F4F0FB6F89448
:105230003EBF0FBE2DBF08C08091C00085FFFCCFD0
:105240009093C600319694919923B1F7FE01B196DF
:1052500007C08091C00085FFFCCF31969093C600B7
:1052600090819923B1F78091C00085FFFCCF8AE03F
:105270008093C600CE0181960E94A4CF0C9477390A
:1052800083E50E94031F882311F40C9477390E9450
:10529000551F0E942CDC7B018C016B0180E50E9474
:1052A000031F882369F0F7FC0BC03FEFE316F104FE
:1052B00009F034F40E94551F0E942CDC8B0102C0BF
:1052C00008E010E0E2EFF3E0808191818017910720
:1052D00011F40C947739329644E0E237F407A1F7E1
:1052E0000730110529F4D092AD07C092AC0704C075
:1052F00017FF02C00C947739802F61E00E9480165E
:10530000802F6C2D0E943317802FB6010E94A015AC
:105310000C94773988E690E00E945F1F882311F093
:105320000C94773983E50E94031F882379F00E944B
:10533000551F2091B807022F10E0000F111F0D54C8
:105340001E4E0E942CDCF801718360830E94087657
:105350000C94773983E50E94031F882311F40C9481
:1053600077390E94551F0E942CDC7093B81160930E
:10537000B7110C94773989E690E00E945F1F88236B
:1053800011F00C947739EAEEF4E0949108C0809122
:10539000C00085FFFCCF9093C6003196949199236D
:1053A000B1F7E091B807F0E0EE0FFF1FEE0FFF1F1F
:1053B000E354FE4E408151816281738187E09AE01F
:1053C00021E030E00E946343E7EEF4E0949108C0EE
:1053D0008091C00085FFFCCF9093C60031969491D8
:1053E0009923B1F7E091B807F0E0EE0FFF1FED54FD
:1053F000FE4E60817181882777FD8095982F0E94ED
:105400005FDCAB01BC0187E09AE021E030E00E9464
:105410006343E3EEF4E0949108C08091C00085FFFF
:10542000FCCF9093C600319694919923B1F74091A7
:10543000C7115091C8116091C9117091CA1187E0CC
:105440009AE021E030E00E946343E0EEF4E09491C2
:1054500008C08091C00085FFFCCF9093C6003196B4
:1054600094919923B1F76091B7117091B811882781
:1054700077FD8095982F0E945FDCAB01BC0187E02F
:105480009AE021E030E00E94634303EBC02E01E18B
:10549000D02E1DEBE12E11E1F12E00E010E0EDED3C
:1054A000F4E09490EBEDF4E0A490E8EDF4E0B49037
:1054B000992DEDEDF4E008C08091C00085FFFCCF90
:1054C0009093C600319694919923B1F787E09AE0C2
:1054D000B8014AE050E00E9488429A2DEBEDF4E0DA
:1054E00008C08091C00085FFFCCF9093C600319624
:1054F00094919923B1F7F7014081518162817381C1
:1055000087E09AE021E030E00E9463439B2DE8EDC4
:10551000F4E008C08091C00085FFFCCF9093C600E6
:10552000319694919923B1F7F601619171916F01D0
:10553000882777FD8095982F0E945FDCAB01BC0126
:1055400087E09AE021E030E00E9463430F5F1F4F45
:1055500024E030E0E20EF31E0230110509F0A8CF7E
:10556000E4EDF4E0949108C08091C00085FFFCCF89
:105570009093C600319694919923B1F78091B80722
:105580000E94D072BC0187E09AE04AE050E00E949D
:105590008842EFECF4E0949108C08091C00085FF50
:1055A000FCCF9093C600319694919923B1F78FEF79
:1055B0009FEF0E94D072BC0187E09AE04AE050E081
:1055C0000E948842ECE8F2E007C08091C00085FFAD
:1055D000FCCF31969093C60090819923B1F78091CA
:1055E000C00085FFFCCF8AE08093C6000C949E39F2
:1055F0008DE690E00E945F1F882311F00C947739AC
:1056000084EC94E00E9481CF83E50E94031F8823ED
:1056100099F00E94551F2091B807022F10E0000F4B
:10562000111F0D541E4E0E942CDCF8017183608303
:1056300081E08093A00316C082E50E94031F8823A7
:1056400089F00E94551F2091B807022F10E0000F2B
:10565000111F0D541E4E0E942CDCF80171836083D3
:105660001092A0030E9408760E94CD144B015C01A9
:105670002091B807022F10E01092B707000F111FFA
:10568000F801ED54FE4E60817181882777FD809589
:10569000982F0E945FDC000F111F03541E4EF8016B
:1056A00020813181428153810E94CBDD18161CF488
:1056B00081E08093B707CC24CA94DC2C7601E1EC1E
:1056C000F4E05490EDEBF4E06490E9EBF4E07490D6
:1056D0007AE0472E30C1952DE1ECF4E008C08091CE
:1056E000C00085FFFCCF9093C6003196949199231A
:1056F000B1F7E091B807F0E0EE0FFF1FEE0FFF1FCC
:10570000E354FE4E408151816281738187E09AE0CB
:1057100021E030E00E946343962DEDEBF4E008C0F9
:105720008091C00085FFFCCF9093C6003196949184
:105730009923B1F76091B80787E09AE070E04AE0FA
:1057400050E00E948842972DE9EBF4E008C0809178
:10575000C00085FFFCCF9093C600319694919923A9
:10576000B1F7F7FE03C0EDE8F2E028C00E94CD14C7
:10577000A70196012854344F4F4F5F4F261B370B1C
:10578000480B590BCA01B90128EE33E040E050E064
:105790000E94B5DF87E09AE0BA01A9012AE030E073
:1057A0000E9434428091C00085FFFCCF0EC08091E2
:1057B000C00085FFFCCF31969093C600908199235D
:1057C000B1F78091C00085FFFCCF4092C6000E94D7
:1057D000CD144B015C010E94EE780E945B1B0E947D
:1057E000B3CFFFEFCF16FFEFDF06FFEFEF06FFEFC0
:1057F000FF0609F052C08091B707E091B8078823EF
:1058000031F1F0E08F01000F111F000F111F035441
:105810001E4EEE0FFF1FED54FE4E608171818827F2
:1058200077FD8095982F0E945FDC20E030E040E813
:105830005FE30E94E3DA9B01AC01F80160817181B2
:10584000828193810E94CBDD87FF58C05EC0F0E06B
:105850008F01000F111F000F111F03541E4EEE0F7A
:10586000FF1FED54FE4E60817181882777FD809582
:10587000982F0E945FDC20E030E040E85FE30E9468
:10588000E4DA9B01AC01F80160817181828193812E
:105890000E94BDDB181694F538C0F7FC36C0E091C5
:1058A000B807F0E08F01000F111F000F111F035404
:1058B0001E4EEE0FFF1FED54FE4E60817181882752
:1058C00077FD8095982F0E945FDC9B01AC01F80169
:1058D00060817181828193810E94E3DA0E942CDCD5
:1058E00097FF07C090958095709561957F4F8F4F7A
:1058F0009F4F64307105810591053CF00E94CD14E5
:10590000AC01CB01DA016C017D01FFEFCF16FFEF97
:10591000DF06FFEFEF06FFEFFF0669F0F7FE02C0BC
:105920000C947A390E94CD146C197D09685B7B4018
:1059300010F00C947A390E94CD14681979098A09FB
:105940009B09695E73408040904008F0C4CE43CF0D
:105950008EE994E00E9481CF83E50E94031F882393
:1059600061F00E94551F0E942CDC7093B811609367
:10597000B71181E08093A0030FC082E50E94031F4E
:10598000882351F00E94551F0E942CDC7093B8119F
:105990006093B7111092A0030E94CD147B018C017B
:1059A0001092B7076091B7117091B811882777FDF1
:1059B0008095982F0E945FDC2091C7113091C8110B
:1059C0004091C9115091CA110E94CBDD18160CF0FC
:1059D00082C081E08093B7077EC00E94CD146E190B
:1059E0007F09800B910B695E73408040904008F402
:1059F0006BC0E091AB07F0E0EE0FFF1FEE0FFF1F53
:105A0000E354FE4E40815181628173819B2DEBE90D
:105A1000F4E008C08091C00085FFFCCF9093C600E1
:105A2000319694919923B1F787E09AE022E030E033
:105A30000E9463439C2DE7E9F4E008C08091C00018
:105A400085FFFCCF9093C600319694919923B1F7CE
:105A50006091AB0787E09AE070E04AE050E00E9476
:105A600088429D2DE3E9F4E008C08091C00085FFE5
:105A7000FCCF9093C600319694919923B1F7409151
:105A8000C7115091C8116091C9117091CA1187E076
:105A90009AE021E030E00E946343ECE8F2E007C0C6
:105AA0008091C00085FFFCCF31969093C600908115
:105AB0009923B1F78091C00085FFFCCFA092C6006A
:105AC0000E94CD147B018C010E94EE780E945B1B2A
:105AD0000E94B3CF0BC0EBE9F4E0B490E7E9F4E047
:105AE000C490E3E9F4E0D490BAE0AB2E8091B7071C
:105AF0002091B7113091B8118823A9F0B9018827F6
:105B000077FD8095982F0E945FDC2091C71130911E
:105B1000C8114091C9115091CA110E94CBDD1816CD
:105B20000CF45BCF18C0B901882777FD8095982FBA
:105B30000E945FDC2091C7113091C8114091C911BA
:105B40005091CA110E94BDDB88232CF48091A003E0
:105B5000882309F442CF89E894E00E9481CF0E9413
:105B6000CD146093C1077093C2078093C3079093CD
:105B7000C4070C94773983E50E94031F882321F121
:105B80000E94551F20E030E040E050E00E94BDDB65
:105B900088231CF460E070E011C00E94551F20E0D3
:105BA00030E04FE753E40E94CBDD18161CF46FEF92
:105BB00070E004C00E94551F0E942CDC7093AD075A
:105BC0006093AC070C9477398FEF90E09093AD071A
:105BD0008093AC070C9477391092AD071092AC0704
:105BE0000C9477390E948B730E94576B409A9FB731
:105BF000F89480910B01826080930B019FBF0E94FB
:105C0000656B1092AD071092AC0768EE73E080E010
:105C100090E00E94DB1410929F038AE794E00E94B8
:105C200081CF0E94B3CF0C947739109269070C94FE
:105C3000773981E0809369070C94773983E50E9476
:105C4000031F8823A1F00E94551F20E030E04AE79F
:105C500054E40E949DDE0E9431DC6093A1037093A6
:105C6000A2038093A3039093A4030C94773988E54F
:105C70000E94031F882311F00C94933989E50E9438
:105C8000031F882311F00C9493398AE50E94031FA7
:105C9000882311F00C94933985E40E94031F882314
:105CA00011F00C9493390E94576B409A9FB7F89467
:105CB00080910B01826080930B019FBF0E94656BF6
:105CC0000C947739159A1092940789E50E94031F66
:105CD000882319F0469A109295078AE50E94031FBF
:105CE000882319F0439A1092960785E40E94031FB7
:105CF000882311F40C947739409A9FB7F8948091D7
:105D00000B01826080930B019FBF0C94773983E570
:105D10000E94031F0E94551F20E030E04AE754E430
:105D20000E949DDE0E9431DC6093C5077093C60718
:105D30008093C7079093C8070C947739A9E26A2E1D
:105D4000ACE07A2EF9E12F2EFCE03F2EE5E64E2E58
:105D5000ECE05E2E88249924F401E251FC4F80810E
:105D60000E94031F882309F45DC053E0851609F0E3
:105D700052C00E94551F5B016C0120E030E040EAF8
:105D800051E40E94BDDB88230CF03FC0F301608129
:105D9000718182819381A60195010E94C4DB7B0100
:105DA0008C0160915D0C70915E0C80915F0C909104
:105DB000600CA80197010E949DDE60935D0C7093BA
:105DC0005E0C80935F0C9093600CF1016081718197
:105DD00082819381A80197010E949DDEF101608379
:105DE000718382839383F2016081718182819381C7
:105DF0000E945DDCA80197010E949DDE0E9431DCBB
:105E0000F2016083718382839383F301A082B18264
:105E1000C282D38207C00E94551FF3016083718341
:105E2000828393830894811C911C24E030E0620EED
:105E3000731E220E331E420E531E34E0831691044D
:105E400009F08ACF0C947739E0EBF3E0949108C025
:105E50008091C00085FFFCCF9093C600319694914D
:105E60009923B1F70C9477398091F4079091F50755
:105E700005966AE270E00E94B511FC01009711F0EE
:105E8000319710828091F4079091F50705960E9452
:105E9000A4CF0C947739EDEAF3E0949108C0809197
:105EA000C00085FFFCCF9093C60031969491992352
:105EB000B1F740916C0750916D0760916E0770913A
:105EC0006F0787E09AE022E030E00E946343E9EA4E
:105ED000F3E0949108C08091C00085FFFCCF9093BF
:105EE000C600319694919923B1F740917007509173
:105EF0007107609172077091730787E09AE022E062
:105F000030E00E946343E5EAF3E0949108C0809199
:105F1000C00085FFFCCF9093C600319694919923E1
:105F2000B1F74091740750917507609176077091B1
:105F3000770787E09AE022E030E00E946343E1EADD
:105F4000F3E0949108C08091C00085FFFCCF90934E
:105F5000C600319694919923B1F7409178075091FA
:105F6000790760917A0770917B0787E09AE022E0D9
:105F700030E00E946343E6E9F3E0949108C0809129
:105F8000C00085FFFCCF9093C60031969491992371
:105F9000B1F780E00E942E6A0E945FDC2091290CFC
:105FA00030912A0C40912B0C50912C0C0E94C4DB98
:105FB000AB01BC0187E09AE022E030E00E9463433D
:105FC000E2E9F3E0949108C08091C00085FFFCCF26
:105FD0009093C600319694919923B1F781E00E9485
:105FE0002E6A0E945FDC20912D0C30912E0C409186
:105FF0002F0C5091300C0E94C4DBAB01BC0187E038
:106000009AE022E030E00E946343EEE8F3E09491EE
:1060100008C08091C00085FFFCCF9093C6003196E8
:1060200094919923B1F782E00E942E6A0E945FDC6E
:106030002091310C3091320C4091330C5091340C42
:106040000E94C4DBAB01BC0187E09AE022E030E0B3
:106050000E946343ECE8F2E007C08091C00085FF36
:10606000FCCF31969093C60090819923B1F780912F
:10607000C00085FFFCCF8AE08093C6000C9477397E
:1060800080E00E94DA690C94773981E00E94DA6935
:106090000C9477398091C00085FFFCCF31969093A6
:1060A000C60090819923B1F78091C00085FFFCCF95
:1060B0008AE08093C600E6E8F3E0949108C08091FE
:1060C000C00085FFFCCF9093C60031969491992330
:1060D000B1F7009B03C0EFE8F2E00AC0E4E9F2E0A8
:1060E00007C08091C00085FFFCCF31969093C60019
:1060F00090819923B1F78091C00085FFFCCF8AE0A1
:106100008093C600EEE7F3E0949108C08091C00050
:1061100085FFFCCF9093C600319694919923B1F7F7
:10612000049B03C0EFE8F2E00AC0E4E9F2E007C034
:106130008091C00085FFFCCF31969093C60090817E
:106140009923B1F78091C00085FFFCCF8AE080934E
:10615000C600E6E7F3E0949108C08091C00085FF97
:10616000FCCF9093C600319694919923B1F7079B89
:1061700003C0EFE8F2E00AC0E4E9F2E007C0809172
:10618000C00085FFFCCF31969093C6009081992383
:10619000B1F78091C00085FFFCCF8AE08093C600F4
:1061A0000C94773984E40E94031F882311F40C9423
:1061B00077390E94551F20E030E040E05FE30E9405
:1061C0009DDE7B018C0120E030E040E050E00E9449
:1061D000BDDB882359F40F2EF0E0CF2EF0E0DF2E48
:1061E000F0E8EF2EFFE3FF2EF02D11C0C801B7013C
:1061F000A80197010E949DDE9B01AC01CA012BED15
:106200003FE049E450E40E949DDE6B017C018091F7
:10621000AB078093B80784E50E94031F882319F118
:106220000E94551F0E9431DC6093B8076230D8F09D
:10623000EFE4F2E0949108C08091C00085FFFCCFAC
:106240009093C600319694919923B1F7EEE9F2E06C
:1062500007C08091C00085FFFCCF31969093C600A7
:1062600090819923B1F78091B807082F10E0000FB3
:10627000111F000F111F05571C4F60E070E080E8F0
:106280009FE3A70196010E94C4DBF801608371833C
:10629000828393830C9477390EEE13E069E3E62E44
:1062A0006CE0F62EF80180810E94031F882349F0DC
:1062B0000E94551F0E9431DCF70160837183828345
:1062C00093830F5F1F4F24E030E0E20EF31E33E0B4
:1062D000023F130739F70E94F0570C9477390EEEFE
:1062E00013E059E1E52E5CE0F52EF80180810E9473
:1062F000031F882339F00E94551FF70160837183C3
:10630000828393830F5F1F4F24E030E0E20EF31E81
:1063100033E0023F130749F70C94773983E50E9475
:10632000031F882351F00E94551F60934D0C7093FA
:106330004E0C80934F0C9093500C84E50E94031FE9
:10634000882311F40C9477390E94551F6093510CE7
:106350007093520C8093530C9093540C0C94773997
:1063600083E50E94031F882351F00E94551F60930C
:10637000490C70934A0C80934B0C90934C0C84E521
:106380000E94031F882351F00E94551F6093610CE7
:106390007093620C8093630C9093640C82E40E946F
:1063A000031F882361F00E94551F0E9431DC609317
:1063B000150C7093160C8093170C9093180C88E5AD
:1063C0000E94031F882351F00E94551F6093550CB3
:1063D0007093560C8093570C9093580C8AE50E944A
:1063E000031F882351F00E94551F6093590C70932E
:1063F0005A0C80935B0C90935C0C85E40E94031F05
:10640000882309F474C70E94551F60935D0C709334
:106410005E0C80935F0C9093600C69C70EEE13E0E6
:106420004CE7E42E47E0F42EF80180810E94031F20
:10643000882339F00E94551FF7016083718382839E
:1064400093830F5F1F4F24E030E0E20EF31E33E032
:10645000013F130749F74BC78AED90E00E945F1F89
:10646000882309F044C788E50E94031F882389F028
:106470008091B807082F10E00E94551F000F111FD0
:10648000000F111F0556184FF80160837183828336
:10649000938389E50E94031F882389F08091B807C0
:1064A000082F10E00E94551F000F111F000F111F31
:1064B0000D55184FF8016083718382839383EFE455
:1064C000F2E0949108C08091C00085FFFCCF9093CA
:1064D000C600319694919923B1F7E6E6F3E09491E2
:1064E00008C08091C00085FFFCCF9093C600319614
:1064F00094919923B1F71092B80740C08091C000E1
:1065000085FFFCCF11969093C6009C919923B1F71B
:10651000F0E0EE0FFF1FEE0FFF1FE556F84F408132
:1065200051816281738187E09AE022E030E00E942D
:106530006343E5EBF2E007C08091C00085FFFCCF2C
:1065400031969093C60090819923B1F7E091B807F6
:10655000F0E0EE0FFF1FEE0FFF1FED55F84F4081EB
:1065600051816281738187E09AE022E030E00E94ED
:1065700063438091B8078F5F8093B807E091B807B5
:10658000E23018F0ECE8F2E00AC0A7EBB2E0BDCFD1
:106590008091C00085FFFCCF31969093C60090811A
:1065A0009923B1F78091C00085FFFCCF8AE08093EA
:1065B000C6009DC683E50E94031F882309F497C681
:1065C0000E94551F0E942CDC709384036093830308
:1065D0008EC683E50E94031F882309F488C60E94A3
:1065E000551F0E942CDC7B018C0184E50E94031F57
:1065F000882389F08DED90E00E945F1F882309F0C9
:1066000076C6E091B807F0E0EE0FFF1FE957FC4FA8
:10661000F182E0826CC6F0928603E092850367C641
:1066200080E50E94031F882309F461C60E94551F5C
:106630000E942CDC7B0183E50E94031F882319F450
:106640000FEF1FEF05C00E94551F0E942CDC8B012D
:10665000C8010196039708F04AC6E2EFF3E0808193
:1066600091818E159F0509F442C6329624E0E237E7
:10667000F207A9F7F7FC3BC60E94576BDE2C8E2D64
:1066800060E00E9480160115110541F001301105EE
:1066900079F03FEF0F3F1307A1F403C000E010E0D3
:1066A00010C08E2D0E94661700E010E0892B49F47F
:1066B00001E010E006C00E94EE780E945B1B0E9481
:1066C000B3CF8D2D0E94661780179107A1F70FC6D3
:1066D00080E50E94031F882351F00E94551F60939C
:1066E000B9037093BA038093BB039093BC0389E40E
:1066F0000E94031F882361F00E94551F0E94A1730E
:106700006093BD037093BE038093BF039093C00357
:1067100084E40E94031F882361F00E94551F0E9499
:10672000AF736093C1037093C2038093C3039093CC
:10673000C40383E40E94031F882351F00E94551F65
:106740006093C5037093C6038093C7039093C803F7
:106750000E94AD72E9EBF2E007C08091C00085FFB6
:10676000FCCF31969093C60090819923B1F7ECEB62
:10677000F2E007C08091C00085FFFCCF3196909376
:10678000C60090819923B1F74091B9035091BA03A3
:106790006091BB037091BC0387E09AE022E030E097
:1067A0000E946343E0ECF2E007C08091C00085FFE7
:1067B000FCCF31969093C60090819923B1F76091F8
:1067C000BD037091BE038091BF039091C0030E94EE
:1067D000A873AB01BC0187E09AE022E030E00E94A0
:1067E0006343E4ECF2E007C08091C00085FFFCCF7A
:1067F00031969093C60090819923B1F76091C103BF
:106800007091C2038091C3039091C4030E94B67338
:10681000AB01BC0187E09AE022E030E00E946343D4
:10682000E8ECF2E007C08091C00085FFFCCF319614
:106830009093C60090819923B1F74091C503509180
:10684000C6036091C7037091C80387E09AE022E015
:1068500030E00E946343ECE8F2E007C08091C000A2
:1068600085FFFCCF31969093C60090819923B1F7B4
:106870008091C00085FFFCCF8AE08093C60037C5B9
:1068800083E50E94031F882329F460E070E080E024
:1068900090E002C00E94551F0E94E75728C585E47A
:1068A0000E94031F882319F4CC24DD2412C00E9407
:1068B000551F0E942CDC6B0177FF0BC00F2EF0E000
:1068C000EF2EF0E0FF2EFCE80F2FF2E41F2FF02D4B
:1068D0000AC00F2EF0E0EF2EF0E0FF2EF6E10F2FB2
:1068E000F3E41F2FF02D83E50E94031F882321F07E
:1068F0000E94551F7B018C0183E40E94031F8823A3
:1069000019F425E030E005C00E94551F0E942CDCE0
:106910009B01C801B701A6010E94987BE8C40E94B0
:10692000576BE5C40E945F8DE2C40E94A494DFC44B
:106930000E94C18FDCC40E946E91D9C48AE50E9476
:10694000031F882309F4B8C00E94551F7B018C01E6
:1069500020E030E040E751EC0E94CBDD88230CF4CE
:106960004EC0C801B70120E030E040EA50EC0E9480
:10697000BDDB18160CF443C0D801C701B058809392
:10698000970790939807A0939907B0939A07EFE41D
:10699000F2E0949108C08091C00085FFFCCF9093F5
:1069A000C600319694919923B1F7EAE5F3E094910A
:1069B00008C08091C00085FFFCCF9093C60031963F
:1069C00094919923B1F78091C00085FFFCCF8AE0B4
:1069D0008093C600ECE8F2E007C08091C00085FF1C
:1069E000FCCF31969093C60090819923B1F78091A6
:1069F000C00085FFFCCF8AE08093C60078C4EFE436
:106A0000F2E0949108C08091C00085FFFCCF909384
:106A1000C600319694919923B1F7E1E5F3E09491A2
:106A200008C08091C00085FFFCCF9093C6003196CE
:106A300094919923B1F7E9E4F3E0949108C080912F
:106A4000C00085FFFCCF9093C600319694919923A6
:106A5000B1F787E09AE061EF7FEF4AE050E00E94F3
:106A60008842E1E4F3E0949108C08091C00085FF82
:106A7000FCCF9093C600319694919923B1F787E0AB
:106A80009AE06BEF7FEF4AE050E00E948842ECE82A
:106A9000F2E007C08091C00085FFFCCF3196909353
:106AA000C60090819923B1F78091C00085FFFCCF8B
:106AB0008AE08093C6001BC4EFE4F2E0949108C022
:106AC0008091C00085FFFCCF9093C60031969491D1
:106AD0009923B1F7E5E3F3E0949108C08091C000F9
:106AE00085FFFCCF9093C600319694919923B1F71E
:106AF0008091C00085FFFCCF8AE08093C600409162
:106B00009707509198076091990770919A0770586C
:106B100087E09AE022E030E00E946343ECE8F2E094
:106B200007C08091C00085FFFCCF31969093C600CE
:106B300090819923B1F78091C00085FFFCCF8AE056
:106B40008093C600D4C3A0906C07B0906D07C0902E
:106B50006E07D0906F07A982BA82CB82DC82E09068
:106B60007007F09071070091720710917307ED8222
:106B7000FE820F831887209174073091750740912A
:106B800076075091770729873A874B875C878091F2
:106B9000780790917907A0917A07B0917B078D874C
:106BA0009E87AF87B88BA98ABA8ACB8ADC8AED8A9E
:106BB000FE8A0F8B188F298F3A8F4B8F5C8F8D8FAA
:106BC0009E8FAF8FB8A385E40E94031F882369F0CE
:106BD000ED84FE840F8518890E94551F9B01AC012E
:106BE000C801B7010E94E4DA0AC06D857E858F85F1
:106BF000988920E030E040E050E40E94E3DA6D87BD
:106C00007E878F87988B6091A5037091A6038091F2
:106C1000A7039091A80320E030E040E752E40E94EF
:106C2000C4DB7B018C01CE010196BE016B5F7F4FFF
:106C3000AE01475F5F4F9E01235F3F4FBBEACB2E04
:106C4000B7E0DB2E0E94485D8AE50E94031F88237F
:106C500059F0E984FA840B851C850E94551F9B011D
:106C6000AC01C801B70108C069857A858B859C8510
:106C700020E030E040E251E40E94E4DA69877A875C
:106C80008B879C876091A5037091A6038091A703D1
:106C90009091A80320E030E040E752E40E94C4DB7A
:106CA0007B018C01CE010196BE016B5F7F4FAE016F
:106CB000475F5F4F9E01235F3F4FABEACA2EA7E0BD
:106CC000DA2E0E94485D88E50E94031F882389F020
:106CD000E980FA800B811C810E94551F9B01AC0149
:106CE000C801B7010E94E4DA69837A838B839C83AD
:106CF00008C080E090E0A0E4B0E489839A83AB838D
:106D0000BC8389E50E94031F882339F00E94551F28
:106D10006D837E838F83988708C080E090E0A0E435
:106D2000B0E48D839E83AF83B8876091A503709193
:106D3000A6038091A7039091A80320E030E040E7EC
:106D400052E40E94C4DB7B018C01CE010196BE019E
:106D50006B5F7F4FAE01475F5F4F9E01235F3F4FE9
:106D6000FBEACF2EF7E0DF2E0E94485D8CE40E9404
:106D7000031F882369F0ED84FE840F8518890E9423
:106D8000551F9B01AC01C801B7010E94E4DA0AC09B
:106D90006D857E858F85988920E030E048EC52E44F
:106DA0000E94E3DA6D877E878F87988B6091A503B9
:106DB0007091A6038091A7039091A80320E030E092
:106DC00040E752E40E94C4DB7B018C01CE010196B6
:106DD000BE016B5F7F4FAE01475F5F4F9E01235F38
:106DE0003F4FEBEACE2EE7E0DE2E0E94485D0E9488
:106DF000576B409A9FB7F89480910B018260809303
:106E00000B019FBF64E670E080E090E00E94DB141D
:106E100085E293E00E9490CF10E018C01F5F0E94AF
:106E2000EE780E945B1B0E94B3CF112379F4539A32
:106E30005B9A63E070E080E090E00E94DB145B9876
:106E400063E070E080E090E00E94DB140E943C97D9
:106E5000882321F38CE40E94031F882369F0ED84CA
:106E6000FE840F8518890E94551F9B01AC01C80143
:106E7000B7010E94E3DA0AC06D857E858F85988907
:106E800020E030E048EC52E40E94E4DA6D877E872F
:106E90008F87988B8D859E85AF85B889809378077D
:106EA00090937907A0937A07B0937B0788E797E0E0
:106EB0000E941B58B9E04B2E512C4C0E5D1EADE0CC
:106EC0006A2E712C6C0E7D1E6091A5037091A60335
:106ED0008091A7039091A80320E030E040E752E4BE
:106EE0000E94C4DB7B018C01CE010196BE016B5F69
:106EF0007F4FA2019301FBEACF2EF7E0DF2E0E9425
:106F0000485DE1E1AE2EB12CAC0EBD1E75E1872EC1
:106F1000912C8C0E9D1E6091A5037091A60380910B
:106F2000A7039091A80320E030E040E752E40E94DC
:106F3000C4DB7B018C01C501B401A20193010E9455
:106F4000485D69E1462E512C4C0E5D1E6091A503F3
:106F50007091A6038091A7039091A80320E030E0F0
:106F600040E752E40E94C4DB7B018C01C501B401FF
:106F7000A20193010E94485D6091A5037091A60350
:106F80008091A7039091A80320E030E040E752E40D
:106F90000E94C4DB7B018C01C501B401A2019E01EA
:106FA000235E3F4F0E94485DA2C188E50E94031FF7
:106FB000882351F00E94551F0E942CDC9B01AC01DC
:106FC00080E0B9010E94636A8AE50E94031F88235A
:106FD00051F00E94551F0E942CDC9B01AC0181E006
:106FE000B9010E94636A85E40E94031F882309F4A3
:106FF0007EC10E94551F0E942CDC9B01AC0182E0E7
:10700000B9010E94636A73C11092B6070E94399752
:107010008091BD079091BE07A091BF07B091C007B6
:107020008093B9079093BA07A093BB07B093BC07AE
:107030000E94461D5CC184E50E94031F882309F459
:107040000BC10E94551F0E9431DC262F6093B807A8
:107050006230B8F1EFE4F2E0949108C08091C00092
:1070600085FFFCCF9093C600319694919923B1F798
:10707000ECECF2E007C08091C00085FFFCCF3196B8
:107080009093C60090819923B1F787E09AE0622F30
:1070900040E050E00E944142EEECF2E007C08091F7
:1070A000C00085FFFCCF31969093C6009081992354
:1070B000B1F78091C00085FFFCCF8AE08093C600C5
:1070C00016C186E40E94031F882311F4EE241EC01B
:1070D0000E94551F7B018C016093E6077093E707C0
:1070E0008093E8079093E90720E030E040E050E02B
:1070F0000E94CBDD181644F4E092A503F092A6039B
:107100000093A7031093A803EE24E3949091B8078B
:107110008091AB07981709F473C0A5EDB7E0ECE6D2
:10712000F7E080E101900D928150E1F72091AB07EB
:10713000C22EDD24CC0CDD1CCC0CDD1CF601E5568A
:10714000F84F60916C0770916D0780916E07909178
:107150006F0720813181428153810E94E3DAF090F0
:10716000B8070F2D10E0000F111F000F111FF801BD
:10717000E556F84F20813181428153810E94E4DA43
:1071800060936C0770936D0780936E0790936F0701
:1071900043EA57E0C40ED51E6091700770917107E5
:1071A0008091720790917307F601208131814281AD
:1071B00053810E94E3DA0D55184FF8012081318187
:1071C000428153810E94E4DA6093700770937107E3
:1071D0008093720790937307F092AB078CE697E069
:1071E00060E777E044E757E028E737E00E94395846
:1071F000EE2031F08091B607882311F40E94841CA0
:10720000EFE4F2E0949108C08091C00085FFFCCFCC
:107210009093C600319694919923B1F7EFEDF2E087
:1072200007C08091C00085FFFCCF31969093C600C7
:1072300090819923B1F76091AB0787E09AE070E005
:107240004AE050E00E9488428091C00085FFFCCF58
:107250008AE08093C6004BC0EFE4F2E0949108C04E
:107260008091C00085FFFCCF9093C6003196949129
:107270009923B1F7E2E1F3E0949108C08091C00056
:1072800085FFFCCF9093C600319694919923B1F776
:107290002091EA073091EB0780E690E0289FF0010B
:1072A000299FF00D389FF00D1124EA50F84F07C0C8
:1072B0008091C00085FFFCCF31969093C6009081ED
:1072C0009923B1F7E0E1F3E0949108C08091C00008
:1072D00085FFFCCF9093C600319694919923B1F726
:1072E0008091C00085FFFCCF8AE08093C6000E9499
:1072F000271B24C08BEA94E00E9481CF0E94CD140A
:107300006093AE077093AF078093B0079093B10777
:107310000E94CD146093C1077093C2078093C30786
:107320009093C407E4CF0E94576B88E50E94031F27
:10733000882311F00C94622E0C94652EEE960FB6F5
:10734000F894DEBF0FBECDBFCF91DF911F910F919B
:10735000FF90EF90DF90CF90BF90AF909F908F9075
:107360007F906F905F904F903F902F9008952F9255
:107370003F924F925F926F927F928F929F92AF92C5
:10738000BF92CF92DF92EF92FF920F931F93DF9302
:10739000CF93CDB7DEB76E970FB6F894DEBF0FBEB2
:1073A000CDBF20E6A22EB12CEFEBF5E084909AE061
:1073B000792EE5E3F6E094906624639413C22D30B1
:1073C00071F02A3321F480917709882341F080916C
:1073D0007809909179098F3591050CF4DFC1E0911E
:1073E0007809F0917909309709F404C3A0917A09DA
:1073F000B0917B09AA9D7001AB9DF00CBA9DF00C79
:107400001124EE0DFF1DEA50F84F1082809177098C
:10741000882309F0BEC110927709A451B84F1C927D
:1074200087010A50184FC8016EE470E00E94B51140
:107430009C01009709F4F7C09093F5078093F40737
:107440002F5F3F4F201B310B2E0D3F1DC9018A506E
:10745000984F60E070E04AE050E00E941D10609399
:107460007C0970937D0980937E0990937F09C09079
:10747000B907D090BA07E090BB07F090BC07A7010E
:1074800096012F5F3F4F4F4F5F4F6217730784077F
:10749000950709F457C380917A0990917B099C0163
:1074A0002A9DC0012B9D900D3A9D900D11248A506C
:1074B000984F6EED76E00E947A11892B09F042C355
:1074C000E5E5F2E0949108C08091C00085FFFCCF13
:1074D0009093C600319694919923B1F7EBEAF6E0C8
:1074E000949108C08091C00085FFFCCF9093C600A6
:1074F000319694919923B1F787E09AE0B701A601FC
:107500002AE030E00E9453428091C00085FFFCCF0A
:1075100073C0FE264F5FFC01E40FF11DEA50F84FE7
:10752000E081EA32B1F73093F5072093F407C901FF
:10753000019660E070E00E94BD0E0E942CDC2F2DB1
:1075400030E02617370709F45DC0E5E5F2E09491D5
:1075500008C08091C00085FFFCCF9093C600319693
:1075600094919923B1F7ECE8F6E0949108C08091EA
:10757000C00085FFFCCF9093C6003196949199236B
:10758000B1F74091B9075091BA076091BB0770916C
:10759000BC0787E09AE02AE030E00E9453428091E5
:1075A000C00085FFFCCF28C0E5E5F2E0949108C05B
:1075B0008091C00085FFFCCF9093C60031969491D6
:1075C0009923B1F7E2E6F6E0949108C08091C000FB
:1075D00085FFFCCF9093C600319694919923B1F723
:1075E00087E09AE0B701A6012AE030E00E9453420A
:1075F0008091C00085FFFCCF8AE08093C6000E9486
:10760000461D4AC080917C0990917D09A0917E0918
:10761000B0917F098093B9079093BA07A093BB07F5
:10762000B093BC073EC0C8016AE270E00E94B51189
:10763000009709F436C0E5E5F2E0949108C0809126
:10764000C00085FFFCCF9093C6003196949199239A
:10765000B1F7E8E3F6E0949108C08091C00085FF9F
:10766000FCCF9093C600319694919923B1F7409145
:10767000B9075091BA076091BB077091BC0787E0CA
:107680009AE02AE030E00E9453428091C00085FFDA
:10769000FCCF8AE08093C600109279091092780995
:1076A00070C280917A0990917B098A9D70018B9DAF
:1076B000F00C9A9DF00C112487010A50184FC80154
:1076C00067E470E00E94B5119C01009709F44BC07B
:1076D0009093F5078093F4072F5F3F4F201B310BEA
:1076E0002E0D3F1DC9018A50984F60E070E00E9446
:1076F000BD0E0E942CDC64307105A8F58091B607A0
:107700008823C9F48091D904882369F5992DE5E38C
:10771000F6E008C08091C00085FFFCCF9093C600C2
:10772000319694919923B1F78091C00085FFFCCFE9
:107730007092C60018C0982DEFEBF5E008C080915C
:10774000C00085FFFCCF9093C60031969491992399
:10775000B1F78091C00085FFFCCF7092C60085EB29
:1077600095E00E9481CF80917A0990917B090196E2
:1077700064E070E00E94A2DF90937B0980937A0915
:10778000809180099091810901969093810980935D
:107790008009109279091092780924C02B3311F4D2
:1077A00060927709809177098823E1F42091780924
:1077B0003091790980917A0990917B098A9DF00135
:1077C0008B9DF00D9A9DF00D1124E20FF31FEA50EE
:1077D000F84F8091760980832F5F3F4F309379096E
:1077E000209378098091030A9091040A2091050A58
:1077F0003091060A821B930B8F779070892B09F4C6
:10780000BBC1809180099091810904970CF0B4C1AB
:1078100087E09AE00E947441282F809376098A308D
:1078200009F0CDCDDCCD8091780990917909892B33
:1078300009F0A7C18091800990918109892B09F0F5
:107840002FC1109282092CC14D3099F0433211F0B2
:107850004A3321F480917709882359F0809178097F
:10786000909179098F35910524F42F5F3F4F09F0EE
:10787000F2C020915C0730915D0740915E07509106
:107880005F078091540790915507A0915607B091DA
:107890005707281739074A075B0708F49EC0932D3E
:1078A000E2EAF5E008C08091C00085FFFCCF90932C
:1078B000C600319694919923B1F78091C00085FF5D
:1078C000FCCF2092C6000E94CD146093B207709343
:1078D000B3078093B4079093B5072091AE0730911A
:1078E000AF074091B0075091B107621B730B840B37
:1078F000950B28EE33E040E050E00E94B5DFF22E19
:10790000E32ED42EC52EEDB7FEB738970FB6F894F8
:10791000FEBF0FBEEDBF0DB71EB70F5F1F4FB28288
:10792000A182F80153824282622F732F842F952FF8
:1079300020E13EE040E050E00E94B5DFF8013583F1
:1079400024836F2D7E2D8D2D9C2D2CE330E040E087
:1079500050E00E94B5DFCA01B9012CE330E040E0FD
:1079600050E00E94B5DFF801778366830E94E4113E
:10797000982DEFE4F2E02DB73EB7285F3F4F0FB6EA
:10798000F8943EBF0FBE2DBF08C08091C00085FF98
:10799000FCCF9093C600319694919923B1F7F501ED
:1079A00007C08091C00085FFFCCF31969093C60040
:1079B00090819923B1F78091C00085FFFCCF209280
:1079C000C600C5010E94A4CF89ED94E00E94718792
:1079D00089ED94E061E00E94B58880917609833258
:1079E00011F490928209209178093091790921153A
:1079F000310519F410927709C4C080917A099091E9
:107A00007B09869DF001879DF00D969DF00D112458
:107A1000E20FF31FEA50F84F1082FC01E451F84FD7
:107A2000908220918009309181092F5F3F4F3093E0
:107A3000810920938009019664E070E00E94A2DF32
:107A400090937B0980937A091092770910927909B3
:107A5000109278093AC04B3311F4909277098091D3
:107A60007709882391F520917809309179098091DF
:107A70007A0990917B09869DF001879DF00D969D76
:107A8000F00D1124E20FF31FEA50F84F80917609B0
:107A900080832F5F3F4F309379092093780915C079
:107AA00080E6682E712C99249394E2EAF5E03490F4
:107AB0000AE0202E5E010894A11CB11C1EE8412E94
:107AC00015E0512EEFE4F2E0849020915C073091B4
:107AD0005D0740915E0750915F0780915407909138
:107AE0005507A0915607B0915707281739074A073D
:107AF0005B0708F046C08091800990918109049746
:107B00000CF03FC0809182098823D9F58091AF069F
:107B10009091B006A091B106B091B20680935C0737
:107B200090935D07A0935E07B0935F0787EA96E0A6
:107B30000E942D4A9C01482F809376098A3009F0D3
:107B400083CE97CE80917A0990917B098A9D80019E
:107B50008B9D100D9A9D100D1124C8018A50984FCD
:107B60006AE270E00E94B5119C01009709F41CCDF7
:107B7000FF2440E0C801CFCC8091DB04882309F0CA
:107B800052CE6E960FB6F894DEBF0FBECDBFCF912A
:107B9000DF911F910F91FF90EF90DF90CF90BF90FA
:107BA000AF909F908F907F906F905F904F903F909D
:107BB0002F900895CF93DF93809180099091810950
:107BC000039714F40E94B73989ED94E060E00E94B5
:107BD000B5888091800990918109892B09F46AC048
:107BE0008091D904882309F44DC02091EA0730918F
:107BF000EB0780E690E0289FE001299FD00D389F99
:107C0000D00D1124CA50D84FCE0168EF76E00E9403
:107C10007A11892BE1F489ED94E0BE010E945E8126
:107C20008091DA04882371F5E5EFF6E0949108C0BD
:107C30008091C00085FFFCCF9093C600319694914F
:107C40009923B1F78091C00085FFFCCF17C089ED63
:107C500094E060E00E944581E3EEF6E0949108C074
:107C60008091C00085FFFCCF9093C600319694911F
:107C70009923B1F78091C00085FFFCCF8AE0809303
:107C8000C60002C00E94AE208091800990918109B7
:107C9000019790938109809380098091EA079091E0
:107CA000EB07019664E070E00E94A2DF9093EB077F
:107CB0008093EA070E94EE780E945B1B0E94037289
:107CC0000E94B3CFDF91CF910895DF93CF930F92AE
:107CD0000F92CDB7DEB787E09AE040E052EC61E06A
:107CE00070E00E943C41EEECF7E0949108C0809176
:107CF000C00085FFFCCF9093C600319694919923E4
:107D0000B1F78091C00085FFFCCF8AE08093C60068
:107D10004FE452E0FA01949108C08091C00085FFC1
:107D2000FCCF9093C600319694919923B1F784B714
:107D3000282F80FF15C0E6ECF7E0949108C08091F1
:107D4000C00085FFFCCF9093C60031969491992393
:107D5000B1F78091C00085FFFCCF8AE08093C60018
:107D600021FF15C0E6EBF7E0949108C08091C000B8
:107D700085FFFCCF9093C600319694919923B1F77B
:107D80008091C00085FFFCCF8AE08093C60022FF6F
:107D900015C0E5EAF7E0949108C08091C00085FF26
:107DA000FCCF9093C600319694919923B1F78091BE
:107DB000C00085FFFCCF8AE08093C60023FF15C07A
:107DC000E5E9F7E0949108C08091C00085FFFCCF01
:107DD0009093C600319694919923B1F78091C00099
:107DE00085FFFCCF8AE08093C60025FF15C0E5E83B
:107DF000F7E0949108C08091C00085FFFCCF90937C
:107E0000C600319694919923B1F78091C00085FF07
:107E1000FCCF8AE08093C60014BEEEE7F7E09491B1
:107E200008C08091C00085FFFCCF9093C6003196BA
:107E300094919923B1F7E8E7F7E0949108C0809115
:107E4000C00085FFFCCF9093C60031969491992392
:107E5000B1F78091C00085FFFCCF8AE08093C60017
:107E6000FA019491EFE4F2E008C08091C00085FF30
:107E7000FCCF9093C600319694919923B1F7E8E630
:107E8000F7E0949108C08091C00085FFFCCF9093EB
:107E9000C600319694919923B1F7E3E5F7E0949108
:107EA00008C08091C00085FFFCCF9093C60031963A
:107EB00094919923B1F7E7E4F7E0949108C0809199
:107EC000C00085FFFCCF9093C60031969491992312
:107ED000B1F7E9E3F7E0949108C08091C00085FF15
:107EE000FCCF9093C600319694919923B1F780917D
:107EF000C00085FFFCCF8AE08093C600EEE2F7E089
:107F0000949108C08091C00085FFFCCF9093C6007B
:107F1000319694919923B1F7E2E2F7E0949108C089
:107F20008091C00085FFFCCF9093C600319694915C
:107F30009923B1F78091C00085FFFCCF8AE0809340
:107F4000C600FA019491EFE4F2E008C08091C0000D
:107F500085FFFCCF9093C600319694919923B1F799
:107F6000E3E1F7E0949108C08091C00085FFFCCF69
:107F70009093C600319694919923B1F72091A21263
:107F80003091A312CE0101962115310519F4885ABA
:107F9000924102C0821B930B9A83898369817A8103
:107FA00087E09AE04AE050E00E948842ECEFF6E079
:107FB000949108C08091C00085FFFCCF9093C600CB
:107FC000319694919923B1F787E09AE060ED74E0DF
:107FD0004AE050E00E9488428091C00085FFFCCFBB
:107FE0008AE08093C6001092EC071092ED07109281
:107FF000EE071092EF070E94A4940E94A2770E94BD
:10800000855A0E9481960E94D16A0E948ED080E19A
:1080100097E220E931E0F9013197F1F70197D9F7BB
:108020000F900F90CF91DF910895BC01809180094E
:108030009091810904970CF070C020917A093091D9
:108040007B0980E690E0AC01249FC001259F900D44
:10805000349F900D11248A50984F0E944C11EFE4E8
:10806000F2E0949108C08091C00085FFFCCF90930E
:10807000C600319694919923B1F7E6EDF7E094911B
:1080800008C08091C00085FFFCCF9093C600319658
:1080900094919923B1F720917A0930917B0980E678
:1080A00090E0289FF001299FF00D389FF00D1124DA
:1080B000EA50F84F07C08091C00085FFFCCF319691
:1080C0009093C60090819923B1F7E4EDF7E0949185
:1080D00008C08091C00085FFFCCF9093C600319608
:1080E00094919923B1F78091C00085FFFCCF8AE07D
:1080F0008093C600C901019664E070E00E94A2DF8F
:1081000090937B0980937A098091800990918109ED
:10811000019690938109809380090895BC01809114
:1081200080099091810904970CF070C020917A0920
:1081300030917B0980E690E0AC01249FC001259F2F
:10814000900D349F900D11248A50984F0E94C011B9
:10815000EFE4F2E0949108C08091C00085FFFCCF6D
:108160009093C600319694919923B1F7E3EEF7E02E
:10817000949108C08091C00085FFFCCF9093C60009
:10818000319694919923B1F720917A0930917B0926
:1081900080E690E0289FF001299FF00D389FF00DB8
:1081A0001124EA50F84F07C08091C00085FFFCCF32
:1081B00031969093C60090819923B1F7E1EEF7E0F4
:1081C000949108C08091C00085FFFCCF9093C600B9
:1081D000319694919923B1F78091C00085FFFCCF2F
:1081E0008AE08093C600C901019664E070E00E94B5
:1081F000A2DF90937B0980937A0980918009909106
:1082000081090196909381098093800908951F92B6
:108210000F920FB60F920BB60F9211242F933F932C
:108220004F938F939F93EF93FF934091C600E091FC
:10823000030AF091040A31969F012F77307031972D
:108240008091050A9091060A2817390739F0ED57F1
:10825000F64F40833093040A2093030AFF91EF9175
:108260009F918F914F913F912F910F900BBE0F9047
:108270000FBE0F901F9018959A01AB01203081EE30
:10828000380780E0480780E0580749F182E0809392
:10829000C00060E079E08DE390E00E94D7DF2150DC
:1082A000304040405040CA01B90122E030E040E097
:1082B00050E00E94D7DF3093C5002093C400809126
:1082C000C10080618093C1008091C100886080936B
:1082D000C1008091C10080688093C1000895109210
:1082E000C00020E130E0E7CF2091050A3091060A76
:1082F0008091030A9091040A8217930719F42FEFD3
:108300003FEF0EC0F901ED57F64F80812F5F3F4FD1
:108310002F7730703093060A2093050A282F30E01B
:10832000C90108958091050A9091060A9093040A64
:108330008093030A089508952F923F924F925F927F
:108340006F927F928F929F92AF92BF92CF92DF9265
:10835000EF92FF920F931F93DF93CF93CDB7DEB7CA
:10836000A0970FB6F894DEBF0FBECDBF1C016A0107
:108370007B01411551056105710549F440E350E069
:1083800060E070E020E030E00E94534254C0882456
:1083900099245401422E55246624772401E010E0EC
:1083A0000C0F1D1F080D191DC701B601A301920175
:1083B0000E94B5DFF80160830894811C911CA11C08
:1083C000B11CC701B601A30192010E94B5DFC9012A
:1083D000DA016C017D01C114D104E104F104F1F66C
:1083E00081E0E82EF12CEC0EFD1EE80CF91C3E019C
:1083F0000894611C711CD501C4010197A109B10940
:108400006C01C818D90814C0F601EE0DFF1D40819B
:108410004A3010F4405D01C0495C50E060E070E01B
:10842000C10120E030E00E9453420894E108F108C5
:108430006E147F0449F7A0960FB6F894DEBF0FBE06
:10844000CDBFCF91DF911F910F91FF90EF90DF9003
:10845000CF90BF90AF909F908F907F906F905F90E4
:108460004F903F902F9008952115310539F4809158
:10847000C00085FFFCCF4093C60008950E949C4138
:108480000895EF92FF920F931F939A01E62EFF2417
:1084900000E010E0B801A7010E9434421F910F9143
:1084A000FF90EF900895EF92FF920F931F93CF9359
:1084B000DF93EC017A018B012115310539F48091AC
:1084C000C00085FFFCCFE092C6001BC02A303105FA
:1084D000B1F477FF10C04DE250E060E070E020E0C2
:1084E00030E00E94534210950095F094E094E11C16
:1084F000F11C011D111DCE01B801A7012AE00E9447
:108500009C41DF91CF911F910F91FF90EF900895C3
:10851000EF92FF920F931F937B019A010027F7FCC4
:108520000095102FB801A7010E9453421F910F918F
:10853000FF90EF9008950F931F938C014DE050E052
:1085400060E070E020E030E00E945342C8014AE061
:1085500050E060E070E020E030E00E9453421F9164
:108560000F910895CF92DF92EF92FF920F931F9396
:108570008C019A016B01EE24FF24B701A6010E9431
:108580003442C8010E949B421F910F91FF90EF90CF
:10859000DF90CF9008959F92AF92BF92CF92DF92DB
:1085A000EF92FF920F931F93CF93DF93EC017A0129
:1085B0008B01922ECB01BA0120E030E040E050E088
:1085C0000E94BDDB88236CF4CE014DE250E060E0F8
:1085D00070E020E030E00E94534217FB109517F93D
:1085E000109520E030E040E05FE3AA240BC0CA0110
:1085F000B90120E030E040E251E40E94C4DB9B017D
:10860000AC01A394A91498F3C801B7010E94E4DA5D
:108610007B018C010E9431DC5B016C010E945DDCFE
:108620009B01AC01C801B7010E94E3DA7B018C0118
:10863000CE01B601A5012AE030E00E943442992023
:10864000A1F1E1EFF2E007C08091C00085FFFCCF0F
:1086500031969093C60090819923B1F726C0C80146
:10866000B70120E030E040E251E40E949DDE7B0152
:108670008C010E942CDC5B016C01CC24B7FCC09403
:10868000DC2CCE01B601A5012AE030E00E94534265
:10869000C601B5010E945FDC9B01AC01C801B701B6
:1086A0000E94E3DA7B018C019A949920C1F6DF9154
:1086B000CF911F910F91FF90EF90DF90CF90BF90DF
:1086C000AF909F9008950E94CB420895FF920F9320
:1086D0001F93CF93DF938B010E94CD14EB01FF24F6
:1086E000FA9409C00E94CD146C1B7D0B60177107B2
:1086F00010F080E008C0FEBC0DB407FEFDCF8EB5C3
:108700008F3F81F781E0DF91CF911F910F91FF9013
:108710000895FC014281242F30E0C9019595879589
:1087200080658CBD40FF02C080E004C080E0463020
:1087300009F081E08DBD808160E00E9433170895CB
:10874000DF92EF92FF920F931F93CF93DF93EC0191
:10875000D62E79018A010E948943CE016CE271E034
:108760000E9466438D2D80648EBD0DB407FEFDCF43
:1087700028E130E0D801C701022E04C0B695A795C4
:10878000979587950A94D2F78EBD0DB407FEFDCF5D
:10879000285030408FEF283F380761F7DD2011F473
:1087A00085E906C088E0D81611F487E801C08FEF8C
:1087B0008EBD0DB407FEFDCF8CE0D81631F48FEFDF
:1087C0008EBD0DB407FEFDCF8EB59FEF2FEF2EBDF2
:1087D0000DB407FEFDCF8EB587FF04C0992311F0BD
:1087E0009150F5CF8B83DF91CF911F910F91FF9027
:1087F000EF90DF900895FC01808161E00E943317C3
:108800000895DC016EBDFA0120E030E00DB407FEF2
:10881000FDCF80818EBD0DB407FEFDCF81818EBD61
:108820002E5F3F4F329682E02030380779F70DB443
:1088300007FEFDCF8FEF8EBD0DB407FEFDCF8FEF8E
:108840008EBD0DB407FEFDCF8FEF8EBD0DB407FEBC
:10885000FDCF8EB513968C9313978F71853011F4DD
:1088600081E0089583E111968C931197CD010E94C8
:10887000FB4380E00895CF92DF92EF92FF920F9337
:108880001F93CF93DF93EC017A018B0169018C81F7
:10889000833039F059E0EE0CFF1C001F111F5A9570
:1088A000D1F7CE0168E1A80197010E94A043882377
:1088B00011F086E023C0CE016EEFA6010E940144B4
:1088C0008823E9F0CE0168E572E00E9466438823C0
:1088D00011F487E113C0CE016DE020E030E040E00C
:1088E00050E00E94A043882341F48FEF8EBD0DB469
:1088F00007FEFDCF8EB5882379F086E18983CE010E
:108900000E94FB4380E0DF91CF911F910F91FF9078
:10891000EF90DF90CF900895CE010E94FB4381E05D
:10892000F2CFBF92CF92DF92EF92FF920F931F93FD
:10893000CF93DF93EC016B017A010E94CD148B0180
:10894000BB24BA9409C00E94CD14601B710B6D52F8
:10895000714010F081E10BC0BEBC0DB407FEFDCF2D
:108960008EB58B838F3F79F38E3F39F08FE089830B
:10897000CE010E94FB4380E02FC0D7011197EF2862
:10898000D9F08FEF8EBD20E030E09FEF0BC00DB42B
:1089900007FEFDCF8EB5F601E20FF31F80839EBD6B
:1089A0002F5F3F4F2A173B0790F30DB407FEFDCF13
:1089B0008EB5AC0DBD1D8C938FEF8EBD0DB407FE33
:1089C000FDCF8EB58FEF8EBD0DB407FEFDCF8EB5FA
:1089D000CE010E94FB4381E0DF91CF911F910F9167
:1089E000FF90EF90DF90CF90BF900895CF92DF92ED
:1089F000EF92FF920F931F93CF93DF93EC017A01D5
:108A00008B0169018C81833039F0A9E0EE0CFF1CE9
:108A1000001F111FAA95D1F7CE0161E1A8019701AE
:108A20000E94A043882339F084E08983CE010E940C
:108A3000FB4380E006C0CE01B60140E052E00E9458
:108A40009144DF91CF911F910F91FF90EF90DF90B4
:108A5000CF900895BF92CF92DF92EF92FF920F9343
:108A60001F93CF93DF93EC01B62E1C8219824883AB
:108A70000E94CD146B01888161E00E948016CE01B6
:108A80000E94FB4382E360E00E94801683E361E082
:108A90000E94801684E361E00E94801685E361E015
:108AA0000E94801685E361E00E94331785E08A8387
:108AB00082E58CBD1DBC80E09FEF9EBD0DB407FE1E
:108AC000FDCF8F5F8A30C9F709C00E94CD146C19A1
:108AD0007D09615D774010F081E05EC0CE0160E00D
:108AE00020E030E040E050E00E94A043182F8B834C
:108AF000813059F7CE0168E02AEA31E040E050E0E9
:108B00000E94A04382FF02C01C8311C080E02FEFAF
:108B10002EBD0DB407FEFDCF9EB58F5F8430C1F72B
:108B20009B839A3A11F082E037C082E08C838C817B
:108B3000823021F0EE24FF2487010FC0E12CF12CBC
:108B4000012D00E4102F09C00E94CD146C197D097D
:108B5000615D774010F08AE01FC0CE0167E320E03E
:108B600030E040E050E00E94A043CE0169E2A8015D
:108B700097010E94A0438B83882331F78C81823038
:108B800029F5CE016AE320E030E040E050E00E94A9
:108B9000A043882331F088E08983CE010E94FB4303
:108BA00021C08FEF8EBD0DB407FEFDCF8EB5807C4A
:108BB000803C11F483E08C8380E09FEF9EBD0DB478
:108BC00007FEFDCF2EB58F5F8330C1F7CE010E9427
:108BD000FB4386E08B1518F488E1898303C0BA82D1
:108BE00081E001C080E0DF91CF911F910F91FF9054
:108BF000EF90DF90CF90BF900895CF93DF93EB017C
:108C0000DC0190E020E03EE28C91803269F0283077
:108C100029F4FE01E90FF11D30839F5FFE01E90F8A
:108C2000F11D8C9180839F5F2F5F11962B3061F730
:108C3000C90FD11D1882DF91CF910895CF93DF9393
:108C4000DC01EB01BA0180E090E020E2FE01E80FD8
:108C5000F91F208301968B309105C1F757E040E062
:108C600022C02E3219F08EEE97E007C05A3049F13B
:108C70005AE048E017C0321721F1FC010196349107
:108C80003323C9F75417E8F02132D8F02F37C8F44E
:108C9000822F81568A3108F42052FE01E40FF11D23
:108CA00020834F5F11962C91222311F02F32C9F6A9
:108CB000FB01B183A08390E08881803219F091E0BC
:108CC00001C090E0892FDF91CF9108956F927F923C
:108CD0008F929F92AF92BF92CF92DF92EF92FF92CC
:108CE0000F931F93CF93DF93EC017A018B012B81BC
:108CF000222309F480C089899A89AB89BC898417A9
:108D00009507A607B70708F476C085C0E114F104FB
:108D10000105110551F41C821D821E821F821886D6
:108D200019861A861B8681E067C0288539854A85A1
:108D30005B85E98DFA8D858590E00996215030405C
:108D40004040504039014A01082E04C0969487944F
:108D5000779467940A94D2F72F5F3F4F4F4F5F4F3E
:108D60000894E108F108010911095701680104C0DC
:108D7000D694C794B794A7948A95D2F70894E11C27
:108D8000F11C011D111DA614B704C804D90428F054
:108D9000211531054105510549F48D899E89AF8919
:108DA000B88D8C839D83AE83BF8316C0A618B70889
:108DB000C808D90811C04C815D816E817F81898D81
:108DC0009A8D94010E9412520894A108B108C1081A
:108DD000D108882331F40FC084E0882E912C8C0EAA
:108DE0009D1EA114B104C104D10429F7E886F986B7
:108DF0000A871B8798CF80E0DF91CF911F910F9159
:108E0000FF90EF90DF90CF90BF90AF909F908F90AA
:108E10007F906F900895223009F078CFE7CFCF93FD
:108E2000DF93EC018C859D85AE85BF8540E06111A7
:108E300041E0BC01CD010E94E84F882319F420E0F5
:108E400030E00AC08889282F30E095E0220F331FD8
:108E50009A95E1F7225F354FC901DF91CF910895CF
:108E60000F931F93CF93DF938C01FC0183818823A1
:108E7000F1F1818187FF38C0C80161E00E940F478E
:108E8000EC010097A1F18881853E89F1F801838189
:108E9000823040F481899289A389B4898C8F9D8F17
:108EA000AE8FBF8FF801858996899B8F8A8F8589C0
:108EB0009689A789B08DCD01AA27BB279D8B8C8B66
:108EC000E091080AF091090A309751F0BE016A5EFC
:108ED0007F4FCE0148961995888D998D9B8B8A8BF3
:108EE000F80181818F7781830E94AD4F04C081E0BA
:108EF000F801808380E0DF91CF911F910F91089559
:108F00000F931F938C010E943047F80113821F9129
:108F10000F910895FC018381882319F0CF010E94ED
:108F200080470895CF93DF93FC01EB018381882371
:108F300091F08250823020F48FE28883198209C038
:108F4000CF0160E00E940F47009729F0BE010E9408
:108F5000FD4581E001C080E0DF91CF9108956F92DF
:108F60007F928F929F92AF92BF92CF92DF92EF92B9
:108F7000FF920F931F93DF93CF9300D00F92CDB743
:108F8000DEB77C015A016B01DC0113968C911397BB
:108F9000813009F091C011968C9181FF8DC0A0C0E5
:108FA0000097A105B10511F481E087C0F701608445
:108FB000718482849384C701B601A5010E9466462C
:108FC000882309F479C0D70159968D919C915A97BD
:108FD000A114B104C104D10489F455964D915D9159
:108FE0006D917C9158970E948852882309F464C03F
:108FF000F701158A168A178A108E44C0D701149675
:109000004D915D916D917C9117979E012F5F3F4F20
:109010000E941252882309F44FC0D7015996ED914E
:10902000FC915A9749815A816B817C818789803173
:1090300049F4483FBFEF5B07B0E06B07B0E07B0748
:1090400048F020C0483F8FEF58078FEF68078FE048
:109050007807C0F4CF010E948852882369F1D701B4
:1090600014964D915D916D917C91179759968D91C4
:109070009C915A970FEF1FEF2FEF3FE00E948B510B
:109080008823D1F0F701A18AB28AC38AD48A818168
:1090900080688183C7010E943047882369F0B60148
:1090A000A5016A147B048C049D0410F4B401A3018F
:1090B000C7010E94664601C080E00F900F900F909C
:1090C0000F90CF91DF911F910F91FF90EF90DF9064
:1090D000CF90BF90AF909F908F907F906F900895AA
:1090E000F70181899289A389B48984179507A60716
:1090F000B70708F055CFE0CFCF93DF93EC0140E006
:1091000050E060E070E00E94AF47882369F0CE0134
:1091100061E00E940F47FC01009731F085EE8083EB
:109120001B820E94AD4F01C080E0DF91CF91089576
:109130002F923F924F925F926F927F928F929F9267
:10914000AF92BF92CF92DF92EF92FF920F931F9355
:10915000CF93DF93EC012A018B81882309F4B6C0F9
:10916000898180FFB3C0C8C025014E185F083B014C
:1091700074E0272E312C2C0E3D1E4201A1C0288503
:1091800039854A855B856FEFA62E61E0B62EA22257
:10919000B3228B8179018A0199E016950795F7949E
:1091A000E7949A95D1F7E98DFA8D823049F4428D92
:1091B000538D648D758D4E0D5F1D601F711F3FC0F7
:1091C000D480DA94DE20A114B104D9F4DD20C9F4EE
:1091D000211531054105510549F48D899E89AF89D5
:1091E000B88D8C839D83AE83BF830BC04C815D8122
:1091F0006E817F81CF0191010E941252882309F470
:1092000065C0E98DFA8D4C815D816E817F81425010
:10921000504060407040058404C0440F551F661FD5
:10922000771F0A94D2F786859785A089B189480F60
:10923000591F6A1F7B1F4D0D511D611D711D80E05F
:1092400092E08A199B0984018815990508F48C011C
:1092500082E00030180709F067C080910A0A9091F7
:109260000B0AA0910C0AB0910D0A481759076A071A
:109270007B0709F459C080910E0C90910F0C93015B
:109280000E94F644882349F421C09501225F354F9E
:10929000C301B901A8010E94A111600E711E9801BD
:1092A00040E050E088859985AA85BB85820F931F91
:1092B000A41FB51F88879987AA87BB87801A910A40
:1092C0008114910409F05BCFA20102C04FEF5FEF60
:1092D000CA01DF91CF911F910F91FF90EF90DF9026
:1092E000CF90BF90AF909F908F907F906F905F9046
:1092F0004F903F902F900895A988BA88CB88DC883A
:10930000E884F9840A851B859A0140E050E0D60183
:10931000C5018E199F09A00BB10B281739074A0701
:109320005B0708F021CF23CFCB01BA0140E00E94B8
:10933000E84F882309F0A9CFC9CFCF92DF92EF92EF
:10934000FF920F931F93CF93DF937C01EB018A0170
:10935000FC018381823008F46FC080859185A285ED
:10936000B3858F719070A070B0700097A105B105A2
:1093700009F062C06DC0F8011082EDE0CE2ED12C54
:10938000C701BE0140E250E00E9498489C01803233
:10939000910521F0009709F04FC050C04881442347
:1093A00009F44CC0453E61F34E3251F38B858F7307
:1093B0008F30E9F501151105D1F18A8D9B8D892B2F
:1093C000B1F5842F90E08F719070009781F1833018
:1093D00091056CF58C9D90018D9D300D9C9D300DFF
:1093E00011242D503040F801E20FF31F8981808352
:1093F0008B8181838D8182838F818383898584831F
:109400008E858583888986838A8987838C898087EE
:109410008E898187888D82878C8D83878E8D8487C6
:10942000888186FF04C0F801E20FF31F15868B8543
:1094300083FDA6CF822F03C08FEF01C080E0DF91B4
:10944000CF911F910F91FF90EF90DF90CF900895F3
:109450004115510509F08FCF90CFDF93CF930F9235
:10946000CDB7DEB7BE016F5F7F4F41E050E00E9495
:109470009848019719F02FEF3FEF03C08981282FFB
:1094800030E0C9010F90CF91DF910895EF92FF92E4
:109490000F931F93CF93DF93EC018B81823038F1D0
:1094A000E884F9840A851B85CE010E942D4A97FD28
:1094B0001EC088859985AA85BB854F96A11DB11DC3
:1094C00088879987AA87BB87A5E016950795F794A3
:1094D000E794AA95D1F72E2D30E02F703070F5E08B
:1094E000220F331FFA95E1F7225F354F02C020E0CB
:1094F00030E0C901DF91CF911F910F91FF90EF9064
:1095000008950F931F93CF93DF93EC018B018B8111
:10951000882309F040C0FB018789803109F041C0F0
:1095200082E08B831D8A1E8A1F8A188E808D918D02
:10953000A0E0B0E045E0880F991FAA1FBB1F4A9525
:10954000D1F7898B9A8BAB8BBC8B13C083E08B8359
:10955000F801428D538D648D758D4D8B5E8B6F8BB5
:10956000788F9E012F5E3F4FC8010E94E6528823EC
:1095700091F01A8F098F81E089831C821D821E82DF
:109580001F82188619861A861B861C861D861E86D3
:109590001F86188A01C080E0DF91CF911F910F9143
:1095A00008958032C1F7D2CF1F93CF93DF93EC01A0
:1095B000142F262F30E0F90175E0EE0FFF1F7A958A
:1095C000E1F7E25FF54F8385817121F0842F82718D
:1095D00009F069C080910A0A90910B0AA0910C0AC7
:1095E000B0910D0A8C879D87AE87BF87688BF90184
:1095F00065E0EE0FFF1F6A95E1F7E25FF54F8489A2
:109600009589A0E0B0E0DC01992788278D8B9E8B9F
:10961000AF8BB88F228D338DA90160E070E0482BAD
:10962000592B6A2B7B2B4D8B5E8B6F8B788F8385B1
:1096300090E088719070009751F4848D958DA68D7F
:10964000B78D898B9A8BAB8BBC8B81E00CC040971C
:1096500051F59E012F5E3F4F898D9A8D0E94E652F3
:10966000882309F184E08B83812F8F7089831C828A
:109670001D821E821F82188619861A861B8614FF79
:1096800018C0CE0140E050E060E070E00E94AF47BB
:10969000882379F40AC049895A896B897C89CE016B
:1096A0000E94664602C01B8280E0DF91CF911F912D
:1096B000089515FDF0CF81E0F8CFCF93DF93EC0153
:1096C0009C012C5F3F4F898D9A8D41E050E060E016
:1096D00070E00E9452538823A1F08D899E89AF8942
:1096E000B88D0097A105B10559F48C819D81AE819B
:1096F000BF818D8B9E8BAF8BB88F8981806889836A
:1097000081E0DF91CF9108952F923F924F925F9227
:109710007F928F929F92AF92BF92CF92DF92EF9201
:10972000FF920F931F93DF93CF9300D000D0CDB75C
:10973000DEB76C01162F072F5E834D83DC01139675
:109740008C911397813009F06FC111968C9181FF34
:109750006BC188C1F601418952896389748980850A
:109760009185A285B38584179507A607B70731F0C1
:10977000C6010E946646882309F456C1812F902FA6
:109780009C0119014D805E8013C1D6015996ED915F
:10979000FC915A97DA01C90149E0B695A7959795CA
:1097A00087954A95D1F774807A9478228FEF882E26
:1097B00081E0982E82229322772009F053C08114F1
:1097C000910409F04FC0D60114964D915D916D91B1
:1097D0007C911797411551056105710581F45596E6
:1097E0008D919D910D90BC91A02D0097A105B10583
:1097F00061F1F60184839583A683B78333C0CF01DB
:109800009E012F5F3F4F0E941252882309F40CC122
:1098100029813A814B815C81D6015996ED91FC9169
:109820005A978789803149F4283FBFEF3B07B0E062
:109830004B07B0E05B0778F008C0283FEFEF3E072A
:10984000EFEF4E07EFE05E0730F0C6010E945D4B80
:10985000882341F4E9C0D60114962D933D934D938E
:109860005C93179780E092E088199909520184155A
:10987000950508F45C01D6015996ED91FC915A9733
:109880001496ED90FD900D911C9117978EEF9FEF20
:10989000AFEFBFEFE80EF91E0A1F1B1F058404C0BF
:1098A000EE0CFF1C001F111F0A94D2F786859785C6
:1098B000A089B189E80EF91E0A1F1B1FE70CF11CD5
:1098C000011D111D90E0A91692E0B90639F58091AD
:1098D0000A0A90910B0AA0910C0AB0910D0A8E15FC
:1098E0009F05A007B10771F41092100C8FEF9FEF46
:1098F000AFEFBFEF80930A0A90930B0AA0930C0A74
:10990000B0930D0A80910E0C90910F0CB801A70135
:1099100091010E943B448823B9F586C081149104CB
:1099200019F5D60118962D913D914D915C911B979B
:1099300051968D919D910D90BC91A02D28173907BE
:109940004A075B0788F00E94AD4F882309F46CC07A
:1099500081E08093100CE0920A0AF0920B0A0093C7
:109960000C0A10930D0A08C0C801B70141E00E941B
:10997000E84F882309F458C09401225F354FC9018C
:10998000B101A5010E94A111950140E050E0F6014E
:1099900080859185A285B385820F931FA41FB51F73
:1099A00080879187A287B3872A0C3B1C4A185B08E3
:1099B000D60118962D913D914D915C911B974114C4
:1099C000510409F0E2CE51968D919D910D90BC917C
:1099D000A02D82179307A407B50748F4F601218B41
:1099E000328B438B548B81818068818311C080913D
:1099F000080A9091090A892B59F08D819E81892B43
:109A000039F0D60111968C911197806811968C933C
:109A1000F601818183FF05C0C6010E94304788237B
:109A200019F04D815E8105C081E0D6018C934FEF26
:109A30005FEFCA0126960FB6F894DEBF0FBECDBF0A
:109A4000CF91DF911F910F91FF90EF90DF90CF901A
:109A5000BF90AF909F908F907F905F904F903F907E
:109A60002F90089582FD76CE89CEDF92EF92FF92FD
:109A70000F931F93CF93DF93EC0189899A89AB8968
:109A8000BC89805E9F4FAF41B04008F071C0CE01ED
:109A90000E945D4B882309F46BC00E94AD4F882360
:109AA00009F466C0E98DFA8DEC80FD800E811F817E
:109AB0008EEF9FEFAFEFBFEFE80EF91E0A1F1B1FDF
:109AC000058404C0EE0CFF1C001F111F0A94D2F77E
:109AD00086859785A089B189E80EF91E0A1F1B1F8C
:109AE00081E08093100CE0920A0AF0920B0A009336
:109AF0000C0A10930D0A80E092E0EEE0FAE0DF013C
:109B00009C011D9221503040E1F7DD24D39411C017
:109B1000B801A7014D0D511D611D711D80910E0CE5
:109B200090910F0C2EE03AE00E943B44882301F113
:109B3000D394E98DFA8D8481D81650F320E032E079
:109B400040E050E0058404C0220F331F441F551F1E
:109B50000A94D2F789899A89AB89BC89820F931FAD
:109B6000A41FB51F898B9A8BAB8BBC8B81E001C086
:109B700080E0DF91CF911F910F91FF90EF90DF90E8
:109B800008958F929F92AF92BF92CF92DF92EF9201
:109B9000FF920F931F93CF93DF936C01EB01942EF1
:109BA000852EA22E898D9A8DD6015A969C938E93DE
:109BB0005997CB0140E050E060E070E00E946646BB
:109BC000BB2438C0CE010E94464AFC01009709F42C
:109BD00093C055E016950795F794E7945A95D1F7F9
:109BE0001E2D1F708081882311F0853EC9F4BB2093
:109BF00099F420910A0A30910B0A40910C0A509175
:109C00000D0AD6011C962D933D934D935C931F979F
:109C100050961C93BB24B3948081882359F418C0B8
:109C2000892D982DBF014BE050E00E9494110097C0
:109C300009F470C0E884F9840A851B8589899A89AA
:109C4000AB89BC89E816F9060A071B0708F4BACFE6
:109C5000A6FE52C0A1FE50C0BB2051F0F6011089F3
:109C6000C60161E00E940F47EC01009769F444C00F
:109C70008B81823009F440C0CE010E94354D88238B
:109C8000D9F110E0CEE0DAE080E2DE011D928A95A3
:109C9000E9F7DE01292D382DC901FC018BE0019087
:109CA0000D928150E1F7E091080AF091090A30978E
:109CB00039F0BE01625F7F4FCE014096199508C012
:109CC00081E298E2998B888B80E098E09F878E876D
:109CD000888999899B8B8A8B998F888F8E859F85A0
:109CE0009F8B8E8B0E94AD4F882331F0C601612F70
:109CF0004A2D0E94D44A01C080E0DF91CF911F918C
:109D00000F91FF90EF90DF90CF90BF90AF909F901A
:109D10008F900895A7FEEACFEFCF2F923F924F92F8
:109D20005F926F927F928F929F92AF92BF92CF92EB
:109D3000DF92EF92FF920F931F93DF93CF93CDB7F4
:109D4000DEB7C654D0400FB6F894DEBF0FBECDBF0D
:109D50003C016B01DE01AE5BBF4F11965C934E93ED
:109D600025962FAF25971C861F861FA21AA6611560
:109D7000710509F480C0FC018381882309F07BC050
:109D8000FA0180818F32F1F08601ECE0EE2EF12CA9
:109D9000EC0EFD1E72E4A72EB12CAC0EBD1E4E01C2
:109DA0000894811C911C2796FFAEEEAE279767E2C0
:109DB000262E312C2C0E3D1E270124C01196B18376
:109DC000A08301C0FD01A081B1818C918F32B1F3DC
:109DD000D60113968C91139782508230A8F28E018F
:109DE000095D1F4F59966D917C915A97C8010E9449
:109DF000814A882351F63FC0342D252D8701832FBA
:109E0000922F7C01F50180819181B401A5010E940E
:109E10001E46882329F42FC03196D501ED93FC937B
:109E2000D501ED91FC9180818F32B1F38823C9F087
:109E3000C701B801A40121E00E94C14D8823D9F0D7
:109E40000C151D0519F0C8010E9480472796EEAD3C
:109E5000FFAD2797EE16FF0679F6C101322D292FA7
:109E6000CDCFC301B801A40125962FAD25970E943F
:109E7000C14D182F01C010E0CE0187960E948A477D
:109E8000CE010C960E948A47812FCA5BDF4F0FB626
:109E9000F894DEBF0FBECDBFCF91DF911F910F9120
:109EA000FF90EF90DF90CF90BF90AF909F908F90FA
:109EB0007F906F905F904F903F902F9008950F93F9
:109EC0001F93DF93CF93CDB7DEB76B970FB6F894A0
:109ED000DEBF0FBECDBF9C01AB0119821C828E017B
:109EE0000F5F1F4FC801B90122E00E948D4E8823E9
:109EF00011F410E004C0C8010E947C48182FCE0164
:109F000001960E948A47812F6B960FB6F894DEBFA8
:109F10000FBECDBFCF91DF911F910F910895DB014F
:109F20000D900020E9F71197A61BB70B0496AD0121
:109F30000E94844B0895DF93CF930F92CDB7DEB785
:109F400069830496BE016F5F7F4F41E050E00E943D
:109F5000844B0F90CF91DF9108958091100C88234E
:109F600099F140910A0A50910B0A60910C0A709184
:109F70000D0A80910E0C90910F0C2EE03AE00E9499
:109F80003B44882319F14091110C5091120C6091BF
:109F9000130C7091140C411551056105710591F078
:109FA00080910E0C90910F0C2EE03AE00E943B4401
:109FB000882361F01092110C1092120C1092130C65
:109FC0001092140C1092100C81E0089580E0089516
:109FD000DF92EF92FF920F931F937B018C01D42E9F
:109FE00080910A0A90910B0AA0910C0AB0910D0A77
:109FF0008E159F05A007B107C1F00E94AD4F8823C1
:10A00000E1F080910E0C90910F0CB801A7012EE0A9
:10A010003AE00E94F644882381F0E0920A0AF09226
:10A020000B0A00930C0A10930D0ADD2011F481E055
:10A0300005C081E08093100C01C080E01F910F915A
:10A04000FF90EF90DF9008958F929F92AF92BF9212
:10A05000CF92DF92EF92FF920F931F93CF93DF93F4
:10A060006C01142F70930F0C60930E0CFC01178A77
:10A0700082E090E0A0E0B0E080839183A283B3838C
:10A080001092100C1092110C1092120C1092130CD2
:10A090001092140C8FEF9FEFAFEFBFEF80930A0A7F
:10A0A00090930B0AA0930C0AB0930D0A442321F459
:10A0B00088249924540140C0453008F01EC160E056
:10A0C00070E080E090E040E00E94E84F882309F4CF
:10A0D00014C1C12FD0E02197FE0174E0EE0FFF1FE5
:10A0E0007A95E1F7E25FF54FE254FE4F8081EE5B37
:10A0F000F14090E08F779070892B09F0FEC0E65315
:10A10000FE4F80819181A281B38184369105A105A2
:10A11000B10508F4F2C064E0CC0FDD1F6A95E1F7E9
:10A12000CC52D44F88809980AA80BB80811491043E
:10A13000A104B10409F4E1C0C501B40140E00E94EA
:10A14000E84F882309F4D9C08091190A90911A0A1E
:10A150008050924009F0D1C020911E0A222309F4B8
:10A16000CCC080911C0A90911D0A892B09F4C5C0AE
:10A1700080911B0A882309F4C0C0F601228B8091CC
:10A180001B0A8483158661E070E007C04F5FF6010B
:10A1900045874150483008F0B0C0F60145858481BC
:10A1A00090E09B01042E02C0220F331F0A94E2F7B5
:10A1B0008217930759F72091240A3091250A211517
:10A1C000310519F040E050E008C02091320A30918A
:10A1D000330A4091340A5091350AF60125833683BB
:10A1E00047835087E0901C0AF0901D0A00E010E0C1
:10A1F000E80CF91C0A1D1B1DE38AF48A058B168BDB
:10A2000080911F0A9091200A918F808F60911E0A81
:10A2100070E080E090E00E946FDF6E0D7F1D801F78
:10A22000911FF601628F738F848F958F20911F0A83
:10A230003091200A55E0220F331F5A95E1F7215043
:10A240003E4F232F3327269540E050E0260F371F3F
:10A25000481F591F26873787408B518B8091210AD1
:10A260009091220A009719F0A0E0B0E008C0809118
:10A270002E0A90912F0AA091300AB091310A8501DF
:10A280007401E21AF30A040B150BA8019701280FB9
:10A29000391F4A1F5B1FF601058404C05695479578
:10A2A000379527950A94D2F72187328743875487B9
:10A2B000253FFFE03F07F0E04F07F0E05F0720F4A5
:10A2C0008CE0F601878B19C0255F3F4F404050401E
:10A2D00018F480E1F6010EC080913A0A90913B0A91
:10A2E000A0913C0AB0913D0AF601828F938FA48F12
:10A2F000B58F80E2878B81E001C080E0DF91CF9154
:10A300001F910F91FF90EF90DF90CF90BF90AF9093
:10A310009F908F9008956F927F928F929F92AF92AD
:10A32000BF92CF92DF92EF92FF920F931F93CF9342
:10A33000DF93EC015A016B013801490142305105AC
:10A340006105710508F45EC089859A85AB85BC8579
:10A350000196A11DB11D84179507A607B70708F43C
:10A3600051C08F89803129F4E52EF62E072F112751
:10A370000CC0803209F046C07A018B0187E0169547
:10A380000795F794E7948A95D1F78B899C89AD89D5
:10A39000BE89E80EF91E0A1F1B1FC801B70141E064
:10A3A0000E94E84F882371F18F89803149F4F501CB
:10A3B000F070EE0FFF1FE25FF54F718260820DC0FB
:10A3C000F501EF77F070EE0FFF1FEE0FFF1FE25F5A
:10A3D000F54F60827182828293828A89823080F016
:10A3E0008D819E81AF81B885E80EF91E0A1F1B1F63
:10A3F000E092110CF092120C0093130C1093140CB9
:10A4000081E001C080E0DF91CF911F910F91FF901B
:10A41000EF90DF90CF90BF90AF909F908F907F9004
:10A420006F900895CF92DF92EF92FF920F931F9358
:10A43000CF93DF93EC017A018B01690189859A85BD
:10A44000AB85BC850196A11DB11D84179507A60794
:10A45000B70708F453C08F89803129F45527412F5D
:10A46000302F2F2D0CC0803209F048C09A01AB016B
:10A4700067E056954795379527956A95D1F78B896B
:10A480009C89AD89BE89280F391F4A1F5B1F8091A7
:10A490000A0A90910B0AA0910C0AB0910D0A281794
:10A4A00039074A075B0739F0CA01B90140E00E9449
:10A4B000E84F882319F18F89803159F4F701F07042
:10A4C000EE0FFF1FE25FF54F80819181A0E0B0E0C9
:10A4D0000EC0F701EF77F070EE0FFF1FEE0FFF1FBA
:10A4E000E25FF54F80819181A281B381BF70F60157
:10A4F00080839183A283B38381E001C080E0DF91F8
:10A50000CF911F910F91FF90EF90DF90CF90089522
:10A51000AF92BF92CF92DF92EF92FF920F931F9371
:10A52000DF93CF9300D00F92CDB7DEB76C017A01E5
:10A530008B0182E090E0A0E0B0E0F601808391839F
:10A54000A283B3835E010894A11CB11CC601B801AB
:10A55000A70195010E941252882341F1C601B8015A
:10A56000A70100E010E020E030E00E948B5188233A
:10A57000E9F0E980FA800B811C81F601878980313E
:10A5800051F4F8EFEF16FFEFFF06F0E00F07F0E0F1
:10A590001F07E0F209C088EFE8168FEFF8068FEF8B
:10A5A00008078FE0180790F281E001C080E00F906B
:10A5B0000F900F900F90CF91DF911F910F91FF900F
:10A5C000EF90DF90CF90BF90AF9008954F925F9241
:10A5D0006F927F928F929F92AF92BF92CF92DF92B3
:10A5E000EF92FF920F931F93DF93CF9300D00F92C0
:10A5F000CDB7DEB76C0149835A836B837C83390105
:10A60000EE24FF2487012E010894411C511C812C4B
:10A61000E2E09E2EA12CB12C49815A816B817C8174
:10A62000C60192010E941252882339F1D501C4015A
:10A63000F601058404C0880F991FAA1FBB1F0A9446
:10A64000D2F7E80EF91E0A1F1B1F29813A814B81A0
:10A650005C818789803131F4285F3F4F4040504012
:10A66000D8F205C0285F3F4F4F4F5F40A8F2F3017B
:10A67000E082F1820283138381E00F900F900F90AC
:10A680000F90CF91DF911F910F91FF90EF90DF908E
:10A69000CF90BF90AF909F908F907F906F905F9082
:10A6A0004F9008952F923F924F925F926F927F92B8
:10A6B0008F929F92AF92BF92CF92DF92EF92FF92D2
:10A6C0000F931F93DF93CF93CDB7DEB72F970FB6BE
:10A6D000F894DEBF0FBECDBF1C014A875B876C8735
:10A6E0007D873F872E87DC0119968D919D910D9076
:10A6F000BC91A02D0196A11DB11D8E839F83A887BB
:10A70000B987F90100811181228133810115110579
:10A710002105310549F0480159010894811C911C1B
:10A72000A11CB11C1D8210C0D1018D909D90AD90D7
:10A73000BC901D828A859B85AC85BD850197A1054E
:10A74000B10511F491E09D83750164014424552401
:10A7500032018E010F5F1F4FF10181859285A38524
:10A76000B485481659066A067B0608F090C08E81AB
:10A770009F81A885B9858C159D05AE05BF0550F450
:10A78000A2E08A2E912CA12CB12CF2E0CF2ED12C5C
:10A79000E12CF12CC101B701A60198010E941252CF
:10A7A000882309F474C089819A81AB81BC81A70197
:10A7B00096012F5F3F4F4F4F5F4F0097A105B105A7
:10A7C00019F049015A010DC0281939094A095B09D4
:10A7D0008A859B85AC85BD85281739074A075B07A5
:10A7E00059F00894411C511C611C711C0894C11C37
:10A7F000D11CE11CF11CB0CFC101A601B7010FEFC4
:10A800001FEF2FEF3FE00E948B51882399F43FC048
:10A810002601370108944108510861087108C101F7
:10A82000B301A201970186010E948B51882379F11F
:10A83000730162018C149D04AE04BF0448F3AE851D
:10A84000BF854D915D916D917C91411551056105DB
:10A85000710539F0C101950184010E948B51882353
:10A86000B1F0EE85FF8580829182A282B382FD8164
:10A87000FF2359F00894811C911CA11CB11CD1012B
:10A880008D929D92AD92BC92139781E001C080E0C1
:10A890002F960FB6F894DEBF0FBECDBFCF91DF91DC
:10A8A0001F910F91FF90EF90DF90CF90BF90AF90EE
:10A8B0009F908F907F906F905F904F903F902F90E0
:10A8C00008952F923F924F925F926F927F928F9254
:10A8D0009F92AF92BF92CF92DF92EF92FF920F932F
:10A8E0001F93DF93CF93CDB7DEB7CD55D0400FB6D2
:10A8F000F894DEBF0FBECDBF2F969FAF8EAF2F97C0
:10A9000061967FAF6EAF61972A0162962FAF629713
:10A9100063960FAF63976496EFAE64976896ACAE9C
:10A92000BDAECEAEDFAE6897E22EFF24EE0CFF1C6C
:10A93000EE0CFF1C9A012E0D3F1D2D963FAF2EAF42
:10A940002D97D9016D907D908D909C90FC01EE0D1E
:10A95000FF1DC401B30120813181428153810E94D6
:10A96000E4DA69AF7AAF8BAF9CAF10E0000F111F34
:10A97000000F111FF201E00FF11F2B96FFAFEEAF9A
:10A980002B97A080B180C280D3802F96EEADFFAD13
:10A990002F97E00FF11FC601B5012081318142815F
:10A9A00053810E94E4DA6DAB7EAB8FAB98AF6496B7
:10A9B0002FAD6497E22FF0E0EE0FFF1FEE0FFF1FA9
:10A9C0002F96AEADBFAD2F97AE0FBF1F4D915D91CE
:10A9D0006D917C9129964CAF5DAF6EAF7FAF29979B
:10A9E00061966EAD7FAD6197E60FF71F6081718153
:10A9F0008281938129962CAD3DAD4EAD5FAD2997F7
:10AA00000E94E3DA69AB7AAB8BAB9CAB6196AEADDF
:10AA1000BFAD61971C968D919D910D90BC91A02D1D
:10AA200025968CAF9DAFAEAFBFAF25972F96AEAD3D
:10AA3000BFAD2F971C962D913D914D915C911F9725
:10AA400021962CAF3DAF4EAF5FAF2197A40193018C
:10AA500050582DA73EA74FA758ABB601A501705877
:10AA600049A75AA76BA77CA761966EAD7FAD61978A
:10AA7000E60EF71ED7016D917D918D919C9129ADC8
:10AA80003AAD4BAD5CAD0E94E3DA3B014C016196FF
:10AA9000EEADFFAD61970E0F1F1FD8016D917D9137
:10AAA0008D919C912DA93EA94FA958AD0E94E3DA42
:10AAB0005B016C016DA57EA58FA598A9A6019501E6
:10AAC0000E949DDE7B018C0169A57AA58BA59CA5C2
:10AAD000A40193010E949DDE9B01AC01C801B70156
:10AAE0000E94E3DA1B012C016DA57EA58FA598A914
:10AAF000A40193010E949DDE7B018C0169A57AA5CA
:10AB00008BA59CA5A60195010E949DDE9B01AC0131
:10AB1000C801B7010E94E4DA9B01AC01C201B10196
:10AB20000E9457DB5B016C0120E030E040E050E028
:10AB30000E94BDDB882354F4C601B5012BED3FE034
:10AB400049EC50E40E94E4DA5B016C01E8968FADB9
:10AB5000E897882351F0C601B5012BED3FE049ECA1
:10AB600050E40E94E3DA5B016C01C601B501E7968F
:10AB70002CAD3DAD4EAD5FADE7970E949DDE29A99E
:10AB80003AA94BA95CA95F770E94D8DD7B018C01B3
:10AB90002FE632E143E85AE30E94BDDB87FDF6C1B0
:10ABA000C801B7010E949ADC0E9431DC78A76FA32C
:10ABB000672B21F4E1E0F0E0F8A7EFA32FA138A57F
:10ABC000B90180E090E00E945DDC7B018C01C60150
:10ABD000B501A80197010E94C4DB6BA37CA38DA3E0
:10ABE0009EA369A97AA98BA99CA9A80197010E9493
:10ABF000C4DB6F8F78A389A39AA325966CAD7DAD36
:10AC00008EAD9FAD259721962CAD3DAD4EAD5FAD80
:10AC100021970E94E3DAA80197010E94C4DB6B8FA1
:10AC20007C8F8D8F9E8F6BA17CA18DA19EA120E03A
:10AC300030E040E05FEB0E949DDE2BA13CA14DA1E6
:10AC40005EA10E949DDE20E030E040E85FE30E94CC
:10AC5000E4DA6F8B788F898F9A8F64963FAD649713
:10AC6000E32FF0E0EE0FFF1FEE0FFF1F9E012F5F9F
:10AC70003F4FE20FF31F29964CAD5DAD6EAD7FAD3A
:10AC8000299740835183628373832F96AEADBFAD06
:10AC90002F971C964D915D916D917C911F974D87DB
:10ACA0005E876F87788B41E050E05A8B498B662432
:10ACB00062967FAD6297672F70E0660F771F660F11
:10ACC000771FC901860F971F6A969FAF8EAF6A974D
:10ACD0006396BFAD6397AB2FB0E0AA0FBB1FAA0F5F
:10ACE000BB1F21E030E02C0F3D1F2A0F3B1F6C964D
:10ACF0003FAF2EAF6C976E96FFAFEEAF6E971AC157
:10AD000038E136150CF446C06DA57EA58FA598A92F
:10AD10002BA13CA14DA15EA10E949DDE7B018C0177
:10AD200069A57AA58BA59CA52F89388D498D5A8D4B
:10AD30000E949DDE9B01AC01C801B7010E94E4DACC
:10AD40007B018C016DA57EA58FA598A92F89388DD3
:10AD5000498D5A8D0E949DDE5B016C0169A57AA523
:10AD60008BA59CA52BA13CA14DA15EA10E949DDEBF
:10AD70009B01AC01C601B5010E94E3DA6DA77EA775
:10AD80008FA798AB6394C701D80189A79AA7ABA7EF
:10AD9000BCA765C049895A89BA0180E090E00E9449
:10ADA0005DDC2BA13CA14DA15EA10E949DDE7B013B
:10ADB0008C01C8010E94C1DB6B8B7C8B8D8B9E8BC1
:10ADC000B701C8010E9400DF3B014C012D96AEADDA
:10ADD000BFAD2D97ED90FD900D911C9117FB109537
:10ADE00017F910952B96EEADFFAD2B972080318093
:10ADF00042805380C801B7012B893C894D895E8907
:10AE00000E949DDE5B016C01C201B101A4019301AE
:10AE10000E949DDE9B01AC01C601B5010E94E4DAEF
:10AE20006DA77EA78FA798ABC801B701A4019301B6
:10AE30000E949DDE7B018C01C201B1012B893C89FE
:10AE40004D895E890E949DDE9B01AC01C801B7015E
:10AE50000E94E3DA69A77AA78BA79CA7662469AD4D
:10AE60007AAD8BAD9CAD2DA53EA54FA558A90E94EE
:10AE7000E4DA6A96AEADBFAD6A976D937D938D931C
:10AE80009C9313976DA97EA98FA998AD29A53AA582
:10AE90004BA55CA50E94E4DA6C96EEADFFAD6C9715
:10AEA00060837183828393836E96AEADBFAD6E97E0
:10AEB0006D917D918D919C912F8D38A149A15AA1C1
:10AEC0000E94E4DA6E96EEADFFAD6E9760837183FB
:10AED000828393836D857E858F8598892B8D3C8DAC
:10AEE0004D8D5E8D0E94E4DA6D877E878F87988B0B
:10AEF000CE0101960E946F19CE010196BE016B5FD3
:10AF00007F4FAE01475F5F4F9E01235F3F4F6896C3
:10AF1000ECACFDAC0EAD1FAD6897F8E7CF2ED12C91
:10AF2000CC0EDD1E0E94485D29893A892F5F3F4F74
:10AF30003A8B298B49895A896FA178A546175707FB
:10AF400008F4DECE61964EAD5FAD6197485F5F4F0E
:10AF500061962EAD3FAD6197245F3F4F61968EADF8
:10AF60009FAD6197DC0114966196BFAFAEAF61975C
:10AF7000BD016896ECACFDAC0EAD1FAD6897E8E77F
:10AF8000CE2ED12CCC0EDD1E0E94485DC35ADF4F61
:10AF90000FB6F894DEBF0FBECDBFCF91DF911F91EA
:10AFA0000F91FF90EF90DF90CF90BF90AF909F9068
:10AFB0008F907F906F905F904F903F902F9008956B
:10AFC0008091551190915611891B8F70089560934F
:10AFD000AA037093AB038093AC039093AD030895E1
:10AFE0000F931F93CF93DF93C0E0D0E08E010B59F6
:10AFF000134FFE01E75CF34F608171818281938181
:10B000000E945DDCFE01E75DF34F208131814281CA
:10B0100053810E949DDE0E9431DCF80160837183C0
:10B02000828393832496C031D10501F7DF91CF91BC
:10B030001F910F910895FC0160817181828193813C
:10B040002091350C3091360C4091370C5091380CD2
:10B050000E949DDE0E946DDE6093810C7093820CD5
:10B060008093830C9093840C81E89CE00E941D6A7D
:10B0700008958F929F92AF92BF92CF92DF92EF92FC
:10B08000FF920F931F93FC018B015A0149016081CC
:10B090007181828193812091290C30912A0C4091F9
:10B0A0002B0C50912C0C0E949DDE0E946DDE35E72A
:10B0B000C32E3CE0D32E6093750C7093760C809376
:10B0C000770C9093780CF801608171818281938173
:10B0D00020912D0C30912E0C40912F0C5091300C62
:10B0E0000E949DDE0E946DDE24E0E22EF12CEC0C2D
:10B0F000FD1C6093790CF701718382839383F501C2
:10B1000060817181828193812091310C3091320C68
:10B110004091330C5091340C0E949DDE0E946DDEF4
:10B120008601085F1F4F60937D0CF8017183828355
:10B130009383F40160817181828193812091350C28
:10B140003091360C4091370C5091380C0E949DDEA6
:10B150000E946DDEF6013C966093810C71838283C0
:10B160009383C601B701A8019F010E94E36980E0B3
:10B1700090E0A0E0B0E08093571190935811A09315
:10B180005911B0935A1180935B1190935C11A09365
:10B190005D11B0935E1180935F1190936011A09345
:10B1A0006111B09362118093631190936411A09325
:10B1B0006511B09366118093671190936811A09305
:10B1C0006911B0936A111F910F91FF90EF90DF907A
:10B1D000CF90BF90AF909F908F9008958F929F9245
:10B1E000AF92BF92CF92DF92EF92FF920F931F9395
:10B1F000CF93DF93EC016B01009709F45CC08FA93A
:10B20000882309F058C0EEA0FFA008A519A5FB01EE
:10B21000B6A0A7A090A481A4C801B7012B2D3A2DF8
:10B22000492D582D0E94BDDB88230CF044C0C80175
:10B23000B701A80197010E949DDE7B018C016AA9DC
:10B240007BA98CA99DA9905820E030E040E050EC0B
:10B250000E949DDE2EA53FA548A959A90E949DDE0A
:10B260009B01AC01C801B7010E94E4DA0E940ADF29
:10B270007B018C016B2D7A2D892D982D9701A801CA
:10B280000E94BDDB882324F4EB2CFA2C092D182D09
:10B290006B2D7A2D892D982D9701A8010E94BDDB79
:10B2A000882349F0C701D801F60186A397A3A0A778
:10B2B000B1A781E086ABDF91CF911F910F91FF90F5
:10B2C000EF90DF90CF90BF90AF909F908F900895B8
:10B2D000EF92FF920F931F93CF93DF93F09056114D
:10B2E00000E010E020E030E04DE4E42E12C0FE9CCF
:10B2F000E0011124CB57D34FC901B801AE010E9420
:10B30000EE588F2D8F5F803109F480E0F82E980180
:10B310008E0180915511F81651F7C901B80140E02E
:10B3200050E00E94EE58DF91CF911F910F91FF9056
:10B33000EF900895AF92BF92CF92DF92EF92FF927B
:10B340000F931F93CF93DF93EB018A016115710572
:10B3500009F466C04115510509F462C0DAA4CBA412
:10B36000BCA4ADA46EA17FA188A599A52D2D3C2DCF
:10B370004B2D5A2D0E94BDDB882309F451C08FA9A3
:10B38000882309F043C0F801E6A0F7A000A511A5A5
:10B390006D2D7C2D8B2D9A2DA80197010E94CBDD60
:10B3A0001816A4F5C801B701A80197010E949DDEF7
:10B3B0007B018C016AA97BA98CA99DA9905820E0EA
:10B3C00030E040E050EC0E949DDE2EA53FA548A94C
:10B3D00059A90E949DDE9B01AC01C801B7010E94E2
:10B3E000E4DA0E940ADF7B018C016D2D7C2D8B2D10
:10B3F0009A2D9701A8010E94BDDB882324F4ED2C2F
:10B40000FC2C0B2D1A2DC701D80104C08D2D9C2DAD
:10B41000AB2DBA2D8EA39FA3A8A7B9A781E08EABB1
:10B42000DF91CF911F910F91FF90EF90DF90CF9020
:10B43000BF90AF900895CF92DF92EF92FF920F935B
:10B44000DF93CF930F920F92CDB7DEB78091551156
:10B450008FB7F894F09056118FBF8091551190E0FE
:10B4600040968F1991098F709070049704F10091A4
:10B47000551103500F70CC24DD2440E050E06DE402
:10B48000E62E13C0802F002309F480E1082F01501D
:10B490000E9DC00111248B57934F9A838983B60167
:10B4A0000E949A59A601C980DA800F1559F70F90AA
:10B4B0000F90CF91DF910F91FF90EF90DF90CF90A1
:10B4C00008956091AC07909156118091551198178D
:10B4D000B9F040915611242F30E08DE490E0289F80
:10B4E000F001299FF00D389FF00D1124E353F34F25
:10B4F000608102C04F5F4F70809155114817D1F79E
:10B5000087E070E00E94A0150895109255111092E6
:10B51000561180E1E5E7FCE0DF011D928A95E9F72D
:10B5200080E090E0A0E0B0E080935B1190935C112C
:10B53000A0935D11B0935E1180935F1190936011A1
:10B54000A0936111B0936211809363119093641181
:10B55000A0936511B0936611809367119093681161
:10B56000A0936911B0936A11809357119093581169
:10B57000A0935911B0935A1108952F923F924F9270
:10B580005F926F927F928F929F92AF92BF92CF9273
:10B59000DF92EF92FF920F931F93DF93CF93CDB77C
:10B5A000DEB766970FB6F894DEBF0FBECDBF9E8B99
:10B5B0008D8B6A017B0148015901DC01D8966D91A0
:10B5C0007D918D919C91DB970E945DDC698B7A8BDC
:10B5D0008B8B9C8BA70196010E949DDE0E94AADBAB
:10B5E0000E9431DC6D837E838F83988769897A8995
:10B5F0008B899C89A50194010E949DDE0E94AADB93
:10B600000E9431DC69837A838B839C832D813E8108
:10B610004F815885283731054105510540F448E7E9
:10B6200050E060E070E04D835E836F8378876981CE
:10B630007A818B819C81683771058105910540F481
:10B6400088E790E0A0E0B0E089839A83AB83BC8375
:10B65000AD89BE89AC5BBF4FAD90BD90CD90DC9005
:10B660001397A454B040BE8BAD8B6D817E818F81CA
:10B6700098850E945DDC6D877E878F87988BC601D9
:10B68000B5010E945FDC1B012C0120E030E040E0AE
:10B6900050E00E94BDDB882321F4E0E070E060E030
:10B6A00028C069897A898B899C899B01AC010E9499
:10B6B0009DDE7B018C016D857E858F8598899B0140
:10B6C000AC010E949DDE9B01AC01C801B7010E9444
:10B6D000E3DA7B018C01C201B101A20191010E9458
:10B6E000E4DA9B01AC01C801B7010E94C4DBE62F7C
:10B6F000692F2E2F372F482F562FB901CA010E94CC
:10B70000AADB0E942CDC3B014C0169817A818B8190
:10B710009C810E945DDC69877A878B879C8766277E
:10B720007727CB016A197B098C099D090E945FDC90
:10B730005B016C0120E030E040E050E00E94BDDBA6
:10B74000882321F4E0E070E060E028C069857A8514
:10B750008B859C859B01AC010E949DDE7B018C0149
:10B7600069897A898B899C899B01AC010E949DDE45
:10B770009B01AC01C801B7010E94E3DA7B018C0197
:10B78000C601B501A60195010E94E4DA9B01AC0156
:10B79000C801B7010E94C4DBE62F692F2E2F372F77
:10B7A000482F562FB901CA010E949ADCED89FE8903
:10B7B000A088B188C288D38886017501E618F70889
:10B7C000080919090E942CDCA8019701261B370BD8
:10B7D000480B590B57FF71C0C201B10120E030E0A6
:10B7E00040E050E00E94BDDB882321F4E0E070E0FF
:10B7F00060E044C0C201B101A20191010E94E4DAFB
:10B800007B018C01C601B5010E945DDC9B01AC018E
:10B81000C801B7010E949DDE7B018C016D857E858C
:10B820008F8598899B01AC010E949DDE9B01AC0134
:10B83000C801B7010E94E3DA7B018C0169857A8532
:10B840008B859C859B01AC010E949DDE9B01AC0118
:10B85000C801B7010E94E4DA7B018C01C201B10189
:10B8600020E030E040E850E40E949DDE9B01AC0106
:10B87000C801B7010E94C4DBE62F692F2E2F372F96
:10B88000482F562FB901CA010E94AADB0E942CDC66
:10B89000AC01CB01DA013C014D0197FE03C06624E7
:10B8A000772443016A147B048C049D0410F0350155
:10B8B000460120E030E040E050E09FB7F8946D8909
:10B8C0007E89645B7F4FDB018C91AC54B040BE8BB2
:10B8D000AD8B882321F5FD01648A758A868A978A53
:10B8E000260D371D481D591D58962D933D934D9398
:10B8F0005C935B972D813E814F815885DC962D931B
:10B900003D934D935C93DF97A05CBF4F29813A81B3
:10B910004B815C812D933D934D935C9313979FBF17
:10B9200066960FB6F894DEBF0FBECDBFCF91DF9104
:10B930001F910F91FF90EF90DF90CF90BF90AF904D
:10B940009F908F907F906F905F904F903F902F903F
:10B9500008954F925F927F928F929F92AF92BF9283
:10B96000CF92DF92EF92FF920F931F93CF93DF93CB
:10B9700070905611C0E0D0E07DE4472E512C46C0B7
:10B980002097B1F18EA9882361F4849CF001859CF5
:10B99000F00D949CF00D1124EB57F34F86A98823EA
:10B9A00039F1EAA0FBA00CA11DA16EA17FA188A581
:10B9B00099A5A80197010E94C4DB5B016C01849CDE
:10B9C000F001859CF00D949CF00D1124EB57F34F82
:10B9D00066A177A180A591A5A80197010E94C4DB6B
:10B9E0008B019C01CE01B601A5010E94BD5A1EAA81
:10B9F000739480E1781609F47724849CE001859C97
:10BA0000D00D949CD00D1124CB57D34F872C992463
:10BA100087FC90948091551190E08816990609F062
:10BA2000AFCF2097F1F0EAA0FBA00CA11DA16EA161
:10BA30007FA188A599A5A80197010E94C4DB5B019D
:10BA40006C016DEC7CEC8CE49DE3A80197010E94F5
:10BA5000C4DB8B019C01CE01B601A5010E94BD5A39
:10BA60001EAADF91CF911F910F91FF90EF90DF9071
:10BA7000CF90BF90AF909F908F907F905F904F90AE
:10BA800008950E941B5A0E9468590E94A95C08955B
:10BA90002F923F924F925F926F927F928F929F92DE
:10BAA000AF92BF92CF92DF92EF92FF920F931F93CC
:10BAB000DF93CF93CDB7DEB7CC59D0400FB6F89413
:10BAC000DEBF0FBECDBF5C014B013A012901C75655
:10BAD000DF4FE882C959D040C656DF4FF882CA59B5
:10BAE000D040C556DF4F0883CB59D040C456DF4FF6
:10BAF0001883CC59D040E796DFAECEAEE797809161
:10BB000055118F5F803109F480E0282F332727FDFE
:10BB100030953CA72BA706C00E94EE780E945B1BC5
:10BB20000E94B3CF8091561190E04BA55CA584177D
:10BB3000950791F36091290C70912A0C80912B0C40
:10BB400090912C0CE5966CAF7DAF8EAF9FAFE597D3
:10BB5000D5012D913D914D915C910E949DDE0E94F9
:10BB60006DDECD57DF4F6883C358D040CC57DF4FD1
:10BB70007883C458D040CB57DF4F8883C558D04016
:10BB8000CA57DF4F9883C658D04020912D0C309172
:10BB90002E0C40912F0C5091300CE1962CAF3DAF04
:10BBA0004EAF5FAFE197CA01B901D4012D913D912C
:10BBB0004D915C910E949DDE0E946DDEC957DF4F62
:10BBC0006883C758D040C857DF4F7883C858D040E3
:10BBD000C757DF4F8883C958D040C657DF4F988377
:10BBE000CA58D0402091310C3091320C4091330C26
:10BBF0005091340CAD962CAF3DAF4EAF5FAFAD97CB
:10BC0000CA01B901D3012D913D914D915C910E94E2
:10BC10009DDE0E946DDEC557DF4F6883CB58D04054
:10BC2000C457DF4F7883CC58D040C357DF4F888349
:10BC3000CD58D040C257DF4F9883CE58D040209186
:10BC4000350C3091360C4091370C5091380CA99638
:10BC50002CAF3DAF4EAF5FAFA997CA01B901D2017A
:10BC60002D913D914D915C910E949DDE0E946DDE73
:10BC7000C157DF4F6883CF58D040C057DF4F78831C
:10BC8000C059D040CF56DF4F8883C159D040CE56DF
:10BC9000DF4F9883C259D0408091810C9091820CE3
:10BCA000A091830CB091840CC157DF4F288139815A
:10BCB0004A815B81CF58D040281739074A075B0774
:10BCC00009F4B8C0E091AB07F0E0EE0FFF1FEE0FF4
:10BCD000FF1FE354FE4E6081718182819381209128
:10BCE000AA033091AB034091AC035091AD030E9485
:10BCF000BDDB88230CF033C0C157DF4F4881598129
:10BD00006A817B81CF58D0404093810C5093820C44
:10BD10006093830C7093840CEEEFF7E0949108C06D
:10BD20008091C00085FFFCCF9093C600319694911E
:10BD30009923B1F7E2E2F8E0949108C08091C00045
:10BD400085FFFCCF9093C600319694919923B1F76B
:10BD50008091C00085FFFCCF8AE08093C60080916F
:10BD6000810C9091820CA091830CB091840CC157EE
:10BD7000DF4F288139814A815B81CF58D040281B11
:10BD8000390B4A0B5B0BCA01B90157FF07C09095ED
:10BD90008095709561957F4F8F4F9F4F0E945FDC1C
:10BDA0007B018C01A9966CAD7DAD8EAD9FADA99741
:10BDB00020E030E042ED53E40E949DDE9B01AC01A7
:10BDC000C801B7010E94CBDD18160CF033C0C15773
:10BDD000DF4F488159816A817B81CF58D0404093A1
:10BDE000810C5093820C6093830C7093840CEEEF63
:10BDF000F7E0949108C08091C00085FFFCCF90933C
:10BE0000C600319694919923B1F7E4E0F8E094915B
:10BE100008C08091C00085FFFCCF9093C60031968A
:10BE200094919923B1F78091C00085FFFCCF8AE0FF
:10BE30008093C60080915511682F70E0A5967FAF62
:10BE40006EAFA5978DE490E0689FF001699FF00DBB
:10BE5000789FF00D1124EB57F34FE45BFF4F1082F6
:10BE6000EC54F0408091750C9091760CA091770C79
:10BE7000B091780CA3968CAF9DAFAEAFBFAFA39738
:10BE8000CD57DF4F288139814A815B81C358D0402B
:10BE9000281B390B4A0B5B0B6F962CAF3DAF4EAF97
:10BEA0005FAF6F97208331834283538357FF0DC069
:10BEB000DA01C901B095A095909581959F4FAF4F3C
:10BEC000BF4F80839183A283B3834091790C5091BB
:10BED0007A0C60917B0C70917C0C6B964CAF5DAFD3
:10BEE0006EAF7FAF6B97C957DF4F88819981AA8169
:10BEF000BB81C758D040841B950BA60BB70B679628
:10BF00008CAF9DAFAEAFBFAF67978DE490E0A596C5
:10BF1000AEADBFADA597A89FF001A99FF00DB89F4A
:10BF2000F00D1124EB57F34F67962CAD3DAD4EADA0
:10BF30005FAD6797248335834683578357FF0DC0D2
:10BF4000DA01C901B095A095909581959F4FAF4FAB
:10BF5000BF4F84839583A683B78340917D0C509116
:10BF60007E0C60917F0C7091800C63964CAF5DAF3E
:10BF70006EAF7FAF6397C557DF4F88819981AA81E4
:10BF8000BB81CB58D040841B950BA60BB70B2F96CB
:10BF90008CAF9DAFAEAFBFAF2F978DE490E0A5966D
:10BFA000AEADBFADA597A89FF001A99FF00DB89FBA
:10BFB000F00D1124EB57F34F2F962CAD3DAD4EAD48
:10BFC0005FAD2F97208731874287538757FF0DC07A
:10BFD000DA01C901B095A095909581959F4FAF4F1B
:10BFE000BF4F80879187A287B3872090810C3090C4
:10BFF000820C4090830C5090840CC157DF4F4881D5
:10C0000059816A817B81CF58D04042195309640914
:10C0100075094DA35EA36FA378A7E091AB07F0E08D
:10C02000EE0FFF1FEE0FFF1FE557FC4F6081718180
:10C03000828193812B966CAF7DAF8EAF9FAF2B9794
:10C04000809185039091860327969FAF8EAF2797A7
:10C050006DA17EA18FA198A597FF07C090958095AF
:10C06000709561957F4F8F4F9F4F0E945FDC2B969D
:10C070002CAD3DAD4EAD5FAD2B970E949DDE0E9475
:10C080002CDC2796AEADBFAD27979D01442737FD29
:10C090004095542F0E946FDF24E630E040E050E0EE
:10C0A0000E94D7DF8DE490E0A5966EAD7FADA59799
:10C0B000689FF001699FF00D789FF00D1124EB57F8
:10C0C000F34FDF011C96248711963C93119712962B
:10C0D0004C93129713965C9360807180828093805A
:10C0E000A480B580C680D780E084F1840285138562
:10C0F000C901DA018E159F05A007B10714F4D80114
:10C10000C7018A159B05AC05BD0514F4D601C50110
:10C110009C01AD0186159705A805B90514F4A40185
:10C1200093018DE490E0A596AEADBFADA597A89F15
:10C13000B001A99F700DB89F700D11246B57734FFC
:10C14000FB01208B318B428B538B2630310541050F
:10C15000510510F40C94B969E85BFF4F8091AC076E
:10C160009091AD07AA2797FDA095BA2F8083918360
:10C17000A283B383DB0190961C92CD57DF4F2881B9
:10C1800039814A815B81C358D040A3968CAD9DAD67
:10C19000AEADBFADA397281739074A075B0724F454
:10C1A00081E0DB0190968C93C957DF4F288139815C
:10C1B0004A815B81C758D0406B966CAD7DAD8EAD2A
:10C1C0009FAD6B97261737074807590794F48DE4FE
:10C1D00090E0A596AEADBFADA597A89FF001A99F31
:10C1E000F00DB89FF00D1124EB57F34F80A1826042
:10C1F00080A3C557DF4F288139814A815B81CB58A5
:10C20000D04063966CAD7DAD8EAD9FAD6397261724
:10C2100037074807590794F48DE490E0A596AEAD32
:10C22000BFADA597A89FF001A99FF00DB89FF00D95
:10C230001124EB57F34F80A1846080A3C157DF4FD7
:10C24000288139814A815B81CF58D040221533053E
:10C250004405550594F48DE490E0A5964EAD5FAD90
:10C26000A597489FF001499FF00D589FF00D1124AC
:10C27000EB57F34F80A1886080A38DE490E0A596F2
:10C280006EAD7FADA597689FF001699FF00D789F17
:10C29000F00D1124EB57F34FE796AEADBFADE79726
:10C2A0008C9181A3208131814281538125962CAFCD
:10C2B0003DAF4EAF5FAF25972115310541055105C3
:10C2C00009F015988DE490E0A5964EAD5FADA59769
:10C2D000489FF001499FF00D589FF00D1124EB5736
:10C2E000F34F6480758086809780611471048104A7
:10C2F000910409F046988DE490E0A5966EAD7FAD6F
:10C30000A597689FF001699FF00D789FF00D1124AB
:10C31000EB57F34FA084B184C284D384A114B10439
:10C32000C104D10409F043988DE490E0A596AEAD28
:10C33000BFADA597A89FF001A99FF00DB89FF00D84
:10C340001124EB57F34F84859585A685B785009713
:10C35000A105B10591F040989FB7F89480910B0129
:10C360008D7F80930B019FBF2090490C30904A0C29
:10C3700040904B0C50904C0C08C02090610C3090B9
:10C38000620C4090630C5090640CC756DF4F68817C
:10C39000C959D040C656DF4F7881CA59D040C556DA
:10C3A000DF4F8881CB59D040C456DF4F9881CC599C
:10C3B000D040A20191010E94BDDB87FD16C0C75687
:10C3C000DF4F8881C959D040C656DF4F9881CA597E
:10C3D000D040C556DF4FA881CB59D040C456DF4F5F
:10C3E000B881CC59D0401C012D016F966CAD7DAD4C
:10C3F0008EAD9FAD6F970E945FDCE5962CAD3DAD95
:10C400004EAD5FADE5970E94C4DBC158DF4F688336
:10C41000CF57D040C058DF4F7883C058D040CF5757
:10C42000DF4F8883C158D040CE57DF4F9883C25822
:10C43000D040AC01CB01DA0189839A83AB83BC8302
:10C4400067966CAD7DAD8EAD9FAD67970E945FDC4A
:10C45000E1962CAD3DAD4EAD5FADE1970E94C4DBE2
:10C46000EC966FAFEC97ED967FAFED97EE968FAFB2
:10C47000EE97EF969FAFEF97AC01CB01DA018D837A
:10C480009E83AF83B8872F966CAD7DAD8EAD9FAD8B
:10C490002F970E945FDCAD962CAD3DAD4EAD5FADEC
:10C4A000AD970E94C4DBE8966FAFE897E9967FAF3F
:10C4B000E997EA968FAFEA97EB969FAFEB97AC01BF
:10C4C000CB01DA0189879A87AB87BC876DA17EA1F2
:10C4D0008FA198A50E945FDCA9962CAD3DAD4EAD15
:10C4E0005FADA9970E94C4DB2B962CAD3DAD4EAD40
:10C4F0005FAD2B970E949DDE7B018C012796EEADF0
:10C50000FFAD2797BF01882777FD8095982F0E9460
:10C510005FDC9B01AC01C801B7010E949DDE20E0F9
:10C5200030E048EC52E40E94C4DB9B01AC016D8713
:10C530007E878F87988B25966CAD7DAD8EAD9FAD38
:10C54000259766307105810591051CF576E0671623
:10C55000710481049104ECF486E0A816B104C104CE
:10C56000D104BCF48DE490E0A596AEADBFADA59727
:10C57000A89FF001A99FF00DB89FF00D1124EB5773
:10C58000F34FDA01C901BF7786A797A7A0ABB1AB7C
:10C590005DC0C158DF4F2881CF57D040C058DF4F12
:10C5A0003881C058D040CF57DF4F4881C158D04064
:10C5B000CE57DF4F5881C258D040B901CA010E94FE
:10C5C00054DF3B014C01EC962FADEC97ED963FAD5F
:10C5D000ED97EE964FADEE97EF965FADEF97B90101
:10C5E000CA010E9454DF5B016C01E8962FADE89709
:10C5F000E9963FADE997EA964FADEA97EB965FADC6
:10C60000EB97B901CA010E9454DF7B018C01C40180
:10C61000B301A60195010E94E4DAA80197010E94E6
:10C62000E4DA0E940ADF2DE430E0A5964EAD5FAD5E
:10C63000A597429FF001439FF00D529FF00D1124EA
:10C64000EB57F34F66A777A780AB91AB8DE490E0F3
:10C65000A5966EAD7FADA597689FF001699FF00D1F
:10C66000789FF00D1124EB57F34F86A597A5A0A94D
:10C67000B1A921968CAF9DAFAEAFBFAF219760E05F
:10C6800070E080E89FE321962CAD3DAD4EAD5FADEF
:10C6900021970E94C4DB9B01AC01C201B1010E9441
:10C6A0009DDE2B013C018091551190915611A82FD0
:10C6B000B0E05096A91BB109AF70B070BAA7A9A796
:10C6C000A230B1050CF451C05D01CC24B7FCC0947C
:10C6D000DC2CC601B5010E945FDC20E030E040E0C8
:10C6E00051E40E94BDDB88230CF03FC060E074E29F
:10C6F00084E799E4A30192010E94C4DB0E946DDEED
:10C700007B018C016091150C7091160C8091170CB7
:10C710009091180CE616F7060807190730F56E1900
:10C720007F09800B910B660F771F881F991FA60149
:10C7300095010E94B5DFCA01B9010E945DDC0E942B
:10C740006DDE9B01AC012E0D3F1D401F511FCA0124
:10C75000B9010E945DDC9B01AC0160E074E284E7FA
:10C7600099E40E94C4DB2B013C018DE490E0A59686
:10C77000EEADFFADA597E89F8001E99F100DF89FF2
:10C78000100D11240B57134F21966CAD7DAD8EAD5E
:10C790009FAD2197A30192010E949DDED801929640
:10C7A0006D937D938D939C93959750966D917D910C
:10C7B0008D919C9153970E945DDCA30192010E9490
:10C7C0009DDE0E94AADB0E9431DCF80160AF71AFF0
:10C7D00082AF93AFCD56DF4F1882C359D040CC56AD
:10C7E000DF4F1882C459D04020E8222E9FE3392E13
:10C7F00088249924E1E0F0E0EC0FFD1FE80DF91D1D
:10C80000C301B20120813181428153810E949DDEAA
:10C81000E1E1F0E0EC0FFD1FE80DF91D608371838D
:10C82000828393835B016C01E894D7F8F401E75E9F
:10C83000F34FE080F18002811381C601B501A801A8
:10C8400097010E94CBDD1816CCF4C801B701A601F0
:10C8500095010E94C4DB6B017C01CD56DF4F6881DE
:10C86000C359D040CC56DF4F7881C459D040C10164
:10C87000A70196010E94BDDB88236CF4CD56DF4FE3
:10C880008881C359D040CC56DF4F9881C459D040DD
:10C89000D1016C017D0124E030E0820E931E30E175
:10C8A0008316910471F0D701C601CD56DF4FC882BF
:10C8B000C359D040CC56DF4F9883C459D0401D0196
:10C8C00099CFC701B60120E030E040E85FE30E9465
:10C8D000BDDB88230CF04CC08E010F5E1F4F81E240
:10C8E000A82EB12CAC0EBD1ED8016D917D918D91FD
:10C8F0009C91A70196010E949DDEF80161937193BE
:10C90000819391938F01EA15FB0571F78DE490E017
:10C91000A5962EAD3FADA597289F8001299F100DAC
:10C92000389F100D11240B57134FD80192966D911B
:10C930007D918D919C919597A70196010E949DDE16
:10C94000F80162A373A384A395A360AD71AD82AD1A
:10C9500093AD0E945DDCA70196010E949DDE0E94BE
:10C9600031DCD801D8966D937D938D939C93DB97A2
:10C970008DE490E0A596EEADFFADA597E89F800110
:10C98000E99F100DF89F100D11240B57134FD8017C
:10C9900050966D917D918D919C9153970E945DDC95
:10C9A000F80126A537A540A951A90E94C4DB1B01A7
:10C9B0002C01F80180819181A281B3810097A105AA
:10C9C000B10549F584819581A681B7810097A105BC
:10C9D000B10509F580859185A285B3850097A105EC
:10C9E000B105C9F4C201B1012091510C3091520C32
:10C9F0004091530C5091540C0E949DDE0E94AADB82
:10CA00000C5B1F4F0E9431DCD8016D937D938D9399
:10CA10009C93139771C1C201B10120914D0C3091CB
:10CA20004E0C40914F0C5091500C0E949DDE0E9484
:10CA3000AADB0E9431DC2DE430E0A596EEADFFAD1F
:10CA4000A597E29F6001E39FD00CF29FD00C1124C8
:10CA500025E83CE0C20ED31EB4E46B2E712C6C0CA6
:10CA60007D1CD3016D937D938D939C931397809040
:10CA7000650C9090660CA090670CB090680C0E94BA
:10CA80005DDC7B018C01F601608171818281938183
:10CA90000E945FDC9B01AC01C801B7010E949DDED2
:10CAA0007B018C01D60150966D917D918D919C9169
:10CAB00053970E945DDC9B01AC01C801B7010E9445
:10CAC000C4DB7B018C01C501B4010E945DDC9B01CC
:10CAD000AC01C801B7010E94CBDD18162CF4F3019C
:10CAE00080829182A282B3828090690C90906A0CBD
:10CAF000A0906B0CB0906C0C8DE490E0A5962EADE0
:10CB00003FADA597289F6001299FD00C389FD00C7E
:10CB1000112445E85CE0C40ED51EA4E46A2E712CF5
:10CB20006C0C7D1CD3016D917D918D919C910E9427
:10CB30005DDC7B018C01F6016481758186819781C2
:10CB40000E945FDC9B01AC01C801B7010E949DDE21
:10CB50007B018C01D60150966D917D918D919C91B8
:10CB600053970E945DDC9B01AC01C801B7010E9494
:10CB7000C4DB7B018C01C501B4010E945DDC9B011B
:10CB8000AC01C801B7010E94CBDD18162CF4F301EB
:10CB900080829182A282B3828090710C9090720CFC
:10CBA000A090730CB090740C8DE490E0A5962EAD1F
:10CBB0003FADA597289F6001299FD00C389FD00CCE
:10CBC000112445E85CE0C40ED51EF4E46F2E712CF0
:10CBD0006C0C7D1CD3016D917D918D919C910E9477
:10CBE0005DDC7B018C01F601648575858685978502
:10CBF0000E945FDC9B01AC01C801B7010E949DDE71
:10CC00007B018C01D60150966D917D918D919C9107
:10CC100053970E945DDC9B01AC01C801B7010E94E3
:10CC2000C4DB7B018C01C501B4010E945DDC9B016A
:10CC3000AC01C801B7010E94CBDD18162CF4F3013A
:10CC400080829182A282B38280906D0C90906E0C53
:10CC5000A0906F0CB090700C8DE490E0A5962EAD76
:10CC60003FADA597289F6001299FD00C389FD00C1D
:10CC7000112445E85CE0C40ED51EE4E46E2E712C50
:10CC80006C0C7D1CD3016D917D918D919C910E94C6
:10CC90005DDC7B018C01F601608571858285938561
:10CCA0000E945FDC9B01AC01C801B7010E949DDEC0
:10CCB0007B018C01D60150966D917D918D919C9157
:10CCC00053970E945DDC9B01AC01C801B7010E9433
:10CCD000C4DB7B018C01C501B4010E945DDC9B01BA
:10CCE000AC01C801B7010E94CBDD18162CF4F3018A
:10CCF00080829182A282B3828DE490E0A5962EADCF
:10CD00003FADA597289F6001299FD00C389FD00C7C
:10CD1000112445E85CE0C40ED51EF601EC5BFF4F24
:10CD200060817181828193810E945DDC7B018C0135
:10CD3000A20191010E94C4DBD601D2966D937D932E
:10CD40008D939C93D597C801B7012DEB37E346E04F
:10CD500051E40E949DDE0E942CDCF601648F758FE9
:10CD6000868F978F6090550C7090560C8090570C62
:10CD70009090580CC401B30120E030E040E05FE344
:10CD80000E949DDE5B016C01298D3A8D4B8D5C8D7F
:10CD900029AF3AAF4BAF5CAF4091590C50915A0C50
:10CDA00060915B0C70915C0C4DAB5EAB6FAB78AF80
:10CDB000CB01BA0120E030E040E05FE30E949DDE5D
:10CDC0007B018C0169AD7AAD8BAD9CAD9F77A801DD
:10CDD00097010E94CBDD181644F4C601B501A801E5
:10CDE00097010E94BDDB882314F4860175016D8DC7
:10CDF0007E8D8F8D98A169AB7AAB8BAB9CAB80910C
:10CE00005D0C90915E0CA0915F0CB091600C8DA7B1
:10CE10009EA7AFA7B8ABBC01CD0120E030E040E059
:10CE20005FE30E949DDE1B012C0169A97AA98BA9F1
:10CE30009CA99F77A20191010E94CBDD181644F4B2
:10CE4000C801B701A20191010E94BDDB882314F43F
:10CE5000170128018DE490E0A596AEADBFADA59772
:10CE6000A89FF001A99FF00DB89FF00D1124EB577A
:10CE7000F34F22A133A144A155A129A33AA34BA367
:10CE80005CA3C201B1010E94BDDB87FD04C029A0E3
:10CE90003AA04BA05CA049A55AA5423051050CF41C
:10CEA00005C150915711CB56DF4F5883C559D0401B
:10CEB00060915811CA56DF4F6883C659D0407091AF
:10CEC0005911C956DF4F7883C759D04080915A1104
:10CED000C856DF4F8883C859D040652FCA56DF4FE8
:10CEE0007881C659D040C956DF4F8881C759D04094
:10CEF000C856DF4F9881C859D04027E137EB41ED44
:10CF000058E30E94CBDD18160CF0D0C069897A89ED
:10CF10008B899C8920915B1130915C1140915D114E
:10CF200050915E110E94E3DA9B01AC010E949DDEEC
:10CF30007B018C016D897E898F89988D20915F118D
:10CF40003091601140916111509162110E94E3DAB9
:10CF50009B01AC010E949DDE9B01AC01C801B701A1
:10CF60000E94E4DA0E940ADF7B018C01A401930194
:10CF70000E94CBDD18165CF00F2EF0E06F2EF0E073
:10CF80007F2EF0E88F2EFFE39F2EF02D08C0C40106
:10CF9000B301A80197010E94C4DB3B014C0169ADBC
:10CFA0007AAD8BAD9CAD20916311309164114091AD
:10CFB0006511509166110E94E3DA7B018C01E894BF
:10CFC00017F9C801B7012DA93EA94FA958AD0E9474
:10CFD000CBDD181694F46DA97EA98FA998ADA80190
:10CFE00097010E94C4DB5B016C01C401B301A6017F
:10CFF00095010E94BDDB882314F46401530169A9E3
:10D000007AA98BA99CA92091671130916811409150
:10D01000691150916A110E94E3DA7B018C01E89456
:10D0200017F9C801B7012DA53EA54FA558A90E9423
:10D03000CBDD181694F46DA57EA58FA598A9A8013F
:10D0400097010E94C4DB7B018C01C601B501A801D8
:10D0500097010E94BDDB882314F48601750169A144
:10D060007AA18BA19CA1A80197010E949DDE7B0162
:10D070008C01CB56DF4F6881C559D040CA56DF4F6F
:10D080007881C659D040C956DF4F8881C759D040F2
:10D09000C856DF4F9881C859D040A80197010E9417
:10D0A000BDDB87FD19C0D801C70102C0D201C10193
:10D0B000CB56DF4F8883C559D040CA56DF4F98837F
:10D0C000C659D040C956DF4FA883C759D040C8566B
:10D0D000DF4FB883C859D0408DE490E0A596AEAD3F
:10D0E000BFADA597A89F8001A99F100DB89F100DF7
:10D0F00011240B57134FCB56DF4F8881C559D040B1
:10D10000CA56DF4F9881C659D040C956DF4FA88113
:10D11000C759D040C856DF4FB881C859D040F80130
:10D1200082A793A7A4A7B5A762A973A984A995A963
:10D13000905820E030E040E050EC0E949DDED801A5
:10D140009E962D913D914D915C91D1970E949DDECF
:10D150002BE037ED43E25BE30E94E4DA0E940ADF52
:10D16000F62EE72ED82EC92ECB56DF4F6881C55933
:10D17000D040CA56DF4F7881C659D040C956DF4FDC
:10D180008881C759D040C856DF4F9881C859D040D0
:10D190002F2D3E2D4D2D5C2D0E94BDDB87FD14C033
:10D1A000CB56DF4FF882C559D040CA56DF4FE882D0
:10D1B000C659D040C956DF4FD882C759D040C8564B
:10D1C000DF4FC882C859D0408DE490E0A596EEADFF
:10D1D000FFADA597E89F8001E99F100DF89F100D06
:10D1E00011240B57134FCB56DF4F8881C559D040C0
:10D1F000CA56DF4F9881C659D040C956DF4FA88123
:10D20000C759D040C856DF4FB881C859D040F8013F
:10D2100086A397A3A0A7B1A762A173A184A195A19A
:10D220002F2D3E2D4D2D5C2D0E94BDDB18162CF0B0
:10D2300081E0D801D7968C9302C0F80117AA8DE43B
:10D2400090E0A5962EAD3FADA597289FF001299FB0
:10D25000F00D389FF00D1124EB57F34F81E086ABB2
:10D26000ABE5B1E1FE01719680E101900D92815034
:10D27000E1F78DE490E0A5964EAD5FADA597489F90
:10D280006001499FD00C589FD00C112465E87CE0C8
:10D29000C60ED71ED6019296ED90FD900D911C9171
:10D2A0009597E0925711F0925811009359111093ED
:10D2B0005A1196966D917D918D919C919997A801A7
:10D2C00097010E94C4DB4B015C01C201B101A801BE
:10D2D00097010E94C4DB8B019C01C601B501A4012A
:10D2E0000E94BD5ABBA5B0935511C157DF4F28818D
:10D2F00039814A815B81CF58D0402093810C309393
:10D30000820C4093830C5093840CC557DF4F4881A7
:10D3100059816A817B81CB58D04040937D0C5093DA
:10D320007E0C60937F0C7093800CC957DF4F68812F
:10D3300079818A819B81C758D0406093790C709322
:10D340007A0C80937B0C90937C0CCD57DF4F8881B7
:10D350009981AA81BB81C358D0408093750C90936A
:10D36000760CA093770CB093780C0E94415D0E94DC
:10D37000DD69C456DF4F0FB6F894DEBF0FBECDBFD8
:10D38000CF91DF911F910F91FF90EF90DF90CF90A1
:10D39000BF90AF909F908F907F906F905F904F90D5
:10D3A0003F902F90089510929F111092A11110920A
:10D3B000A31108958093B8030895EFE6F0E080810B
:10D3C0008260808308951F93FC011FB7F8948081C9
:10D3D0009181A281B3818093791190937A11A09366
:10D3E0007B11B0937C11FB0180819181A281B3817B
:10D3F00080937D1190937E11A0937F11B093801143
:10D40000FA0180819181A281B381809381119093EF
:10D410008211A0938311B0938411F90180819181CD
:10D42000A281B3818093851190938611A093871177
:10D43000B09388111FBF1F910895FC012FB7F89476
:10D4400080819181A281B38180938511909386110F
:10D45000A0938711B09388112FBF0895E82F8FB73D
:10D46000F894F0E0EE0FFF1FEE0FFF1FE758FE4E9F
:10D4700020813181428153818FBFB901CA01089552
:10D4800080916F008D7F80936F0006C08091561150
:10D490008F5F8F7080935611909155118091561126
:10D4A000981751F410926C1110926B1180916F00CB
:10D4B000826080936F00089590915511809156116C
:10D4C000981751F3E3CF9B01882399F4B90188277A
:10D4D00077FD8095982F2FEF30E040E050E00E94DC
:10D4E0006FDF20ED37E040E050E00E94D7DF8CE2B4
:10D4F00014C08130B1F4B901882777FD8095982F49
:10D500002FEF30E040E050E00E946FDF20ED37E089
:10D5100040E050E00E94D7DF8DE2B9010E94A015E3
:10D5200008958230A9F4B901882777FD8095982F56
:10D530002FEF30E040E050E00E946FDF20ED37E059
:10D5400040E050E00E94D7DF8EE2B9010E94A015B2
:10D5500008958CE261E00E9480168DE261E00E94F5
:10D5600080168EE261E00E9480166091AE03709199
:10D57000AF0380E00E94636A6091B0037091B103D1
:10D5800081E00E94636A6091B2037091B30382E00C
:10D590000E94636AE1E2F1E08081887F816080839C
:10D5A00008950E94A96A099A3C9A399AEAE0F1E042
:10D5B0008081806480838081846080830D9A159A45
:10D5C0003E9A469A3B9A439A389A409A8081826062
:10D5D00080839FB7F894EBE0F1E0808182608083E4
:10D5E0009FBF0898109A0C98149A0F98179A0B9A44
:10D5F0001398159A109294073D9A4598469A10925E
:10D6000095073A9A4298439A10929607EAE0F1E019
:10D610008081806880839FB7F894EBE0F1E080819F
:10D620008F7780839FBF409AEAE0F1E0808181603C
:10D6300080839FB7F894EBE0F1E080818E7F808358
:10D640009FBF9FB7F894EBE0F1E080818260808318
:10D650009FBFA1E8B0E08C918F7E8C938C91886005
:10D660008C93E0E8F0E080818D7F808380818E7FE5
:10D67000808380818F73808380818F7C80838C9175
:10D68000887F82608C9380E090E4909389008093FF
:10D6900088001092850010928400EFE6F0E080810F
:10D6A0008260808381E08093B8037894089590919C
:10D6B000551180915611981739F00E94EE780E940A
:10D6C0005B1B0E94B3CFF3CF08950E94576B159A4E
:10D6D00010929407469A10929507439A10929607D3
:10D6E000409A9FB7F894EBE0F1E0808182608083FC
:10D6F0009FBF08951F920F920FB60F920BB60F9215
:10D700001124AF92BF92CF92DF92EF92FF920F93CC
:10D710001F932F933F934F935F936F937F938F93B9
:10D720009F93AF93BF93CF93DF93EF93FF9380913A
:10D730006B1190916C11892B09F094C19091551146
:10D7400080915611981719F4E0E0F0E014C0809130
:10D75000561190E02DE430E0829FF001839FF00DA0
:10D76000929FF00D1124EB57F34FE45BFF4F81E0E4
:10D770008083EC54F040F0936C11E0936B11309780
:10D7800009F46AC1E45BFF4F81E08083EC54F04010
:10D790001092AB111092AC111092AD111092AE110B
:10D7A00060AD71AD2CE96134720718F060E47CE97A
:10D7B00004C03EE46132730730F076956795769544
:10D7C000679584E007C047E26131740730F07695D1
:10D7D000679582E08093A41107C08093A411603202
:10D7E000710510F460E270E06052704058E0603003
:10D7F0007507E8F0472F50E0440F551F440F551FA1
:10D80000455A574F9A012E5F3F4FF90185919491E8
:10D810009C01AA27639FC001629F810D9A1F0694F5
:10D820008A1F9A1F1124FA01459154911EC0CB0101
:10D83000969587958C7F855A934FFC01459154911D
:10D84000FC01329625913491862F90E0877090707C
:10D85000FC012E9FC0012F9F900D3E9F900D112423
:10D86000B3E096958795BA95E1F7481B590B443676
:10D870005105A8F4E3EFF2E007C08091C00085FFF6
:10D88000FCCF31969093C60090819923B1F787E041
:10D890009AE04AE050E00E94B24244E650E05093E1
:10D8A000B0114093AF118091A4118093B1111092E7
:10D8B000B211E0916B11F0916C1164AD75AD709384
:10D8C000AA116093A911FCE961347F0718F060E4A4
:10D8D0007CE904C02EE46132720730F076956795DA
:10D8E0007695679584E007C037E26131730730F0C1
:10D8F0007695679582E08093A41108C081E08093BB
:10D90000A4116032710510F460E270E06052704062
:10D9100048E060307407E8F0472F50E0440F551F8F
:10D92000440F551F455A574F9A012E5F3F4FF9013B
:10D93000859194919C01AA27639FC001629F810DEC
:10D940009A1F06948A1F9A1F1124FA014591549137
:10D950001EC0CB01969587958C7F855A934FFC010D
:10D9600045915491FC01329625913491862F90E097
:10D9700087709070FC012E9FC0012F9F900D3E9FDD
:10D98000900D112433E0969587953A95E1F7481B61
:10D99000590B44365105A8F4E3EFF2E007C080913B
:10D9A000C00085FFFCCF31969093C60090819923EB
:10D9B000B1F787E09AE04AE050E00E94B24244E6C4
:10D9C00050E0CA01A0E0B0E08093A5119093A611A9
:10D9D000A093A711B093A811509389004093880099
:10D9E000E0916B11F0916C1180899189A289B389C2
:10D9F000B695A79597958795B095A09590958195A3
:10DA00009F4FAF4FBF4F8093891190938A11A0937E
:10DA10008B11B0938C1180938D1190938E11A093E4
:10DA20008F11B09390118093911190939211A093C4
:10DA30009311B09394118093951190939611A093A4
:10DA40009711B09398111092991110929A11109207
:10DA50009B1110929C1106C080ED97E09093890075
:10DA600080938800C0916B11D0916C11209709F4BC
:10DA7000ADC488A180939D1180FF03C0119A8FEFE0
:10DA800002C0119881E08093B40380919D1181FFC1
:10DA900003C044988FEF02C0449A81E08093B5039D
:10DAA00080919D1180FF36C08091B803882391F149
:10DAB00020B1217031E0232759F180919E118823F4
:10DAC00039F188819981AA81BB81181619061A0635
:10DAD0001B06F4F48091791190917A11A0917B1139
:10DAE000B0917C1180936D1190936E11A0936F1182
:10DAF000B093701130939F1188899989AA89BB8945
:10DB00008093991190939A11A0939B11B0939C11BB
:10DB100020939E1180919D1181FF3AC08091B8039E
:10DB20008823B1F180B182958F708095282F217064
:10DB300080FF2CC08091A011882341F18C819D81B0
:10DB4000AE81BF81181619061A061B06FCF48091D7
:10DB50007D1190917E11A0917F11B09180118093E1
:10DB6000711190937211A0937311B093741181E0AD
:10DB70008093A11188899989AA89BB898093991179
:10DB800090939A11A0939B11B0939C112093A01194
:10DB900080919D1182FF3AC0419A8FEF8093B60326
:10DBA0008091B8038823B1F120E007992CC021E0CF
:10DBB0008091A211882339F188859985AA85BB8532
:10DBC000181619061A061B06F4F48091811190911B
:10DBD0008211A0918311B09184118093751190935B
:10DBE0007611A0937711B09378112093A3118889AF
:10DBF0009989AA89BB898093991190939A11A093CE
:10DC00009B11B0939C112093A21104C0419881E014
:10DC10008093B60380919D1199A183FF12C091302A
:10DC200031F49FB7F89480910B018B7F05C09FB7AB
:10DC3000F89480910B018F7B80930B019FBF8FEF36
:10DC400011C0913031F49FB7F89480910B0184603A
:10DC500005C09FB7F89480910B01806480930B01FD
:10DC60009FBF81E08093B70360E070E08CC180913A
:10DC7000C00087FF19C04091C600E091030AF091EF
:10DC8000040A31969F012F77307031978091050AF1
:10DC90009091060A2817390739F0ED57F64F40835F
:10DCA0003093040A2093030A288139814A815B81D9
:10DCB0008091891190918A11A0918B11B0918C1152
:10DCC000280F391F4A1F5B1F2093891130938A1137
:10DCD00040938B1150938C111216130614061506DF
:10DCE0006CF5139A88899989AA89BB89281B390BF5
:10DCF0004A0B5B0B2093891130938A1140938B114F
:10DD000050938C112091791130917A1140917B11AF
:10DD100050917C118091B403992787FD9095A92F8C
:10DD2000B92F820F931FA41FB51F80937911909371
:10DD30007A11A0937B11B0937C1113982C813D81B3
:10DD40004E815F8180918D1190918E11A0918F11E4
:10DD5000B0919011280F391F4A1F5B1F20938D111E
:10DD600030938E1140938F11509390111216130619
:10DD7000140615066CF5459A88899989AA89BB8984
:10DD8000281B390B4A0B5B0B20938D1130938E119E
:10DD900040938F115093901120917D1130917E11FD
:10DDA00040917F11509180118091B503992787FD93
:10DDB0009095A92FB92F820F931FA41FB51F809391
:10DDC0007D1190937E11A0937F11B093801145989F
:10DDD000288539854A855B858091911190919211B2
:10DDE000A0919311B0919411280F391F4A1F5B1F06
:10DDF0002093911130939211409393115093941169
:10DE000012161306140615066CF5429A888999892C
:10DE1000AA89BB89281B390B4A0B5B0B20939111F4
:10DE2000309392114093931150939411209181114A
:10DE30003091821140918311509184118091B603E9
:10DE4000992787FD9095A92FB92F820F931FA41FA3
:10DE5000B51F8093811190938211A0938311B09389
:10DE6000841142982C853D854E855F858091951162
:10DE700090919611A0919711B0919811280F391F88
:10DE80004A1F5B1F20939511309396114093971171
:10DE90005093981112161306140615060CF04DC077
:10DEA00089A1813031F49FB7F89480910B01816092
:10DEB00005C09FB7F89480910B01806880930B0197
:10DEC0009FBF88899989AA89BB89281B390B4A0B6E
:10DED0005B0B2093951130939611409397115093BB
:10DEE00098112091851130918611409187115091A0
:10DEF00088118091B703992787FD9095A92FB92F95
:10DF0000820F931FA41FB51F8093851190938611D4
:10DF1000A0938711B093881189A1813031F49FB704
:10DF2000F89480910B018E7F05C09FB7F894809183
:10DF30000B018F7780930B019FBF80919911909176
:10DF40009A11A0919B11B0919C110196A11DB11D38
:10DF50008093991190939A11A0939B11B0939C1167
:10DF60002091991130919A1140919B1150919C11DF
:10DF70006F5F7F4F88899989AA89BB8928173907DC
:10DF80004A075B0738F48091A41190E0681779077D
:10DF90000CF46DCE2091991130919A1140919B1102
:10DFA00050919C118C899D89AE89BF8982179307F6
:10DFB000A407B50708F4E3C0E090A511F090A611FE
:10DFC0000091A7111091A811AC8CBD8CCE8CDF8C68
:10DFD000A8019701C601B501AA27279FB12D389F37
:10DFE000F001489FF00D479FE00DF11D289FB00DF7
:10DFF000E11DFA1F379FB00DE11DFA1F469FB00DBE
:10E00000E11DFA1F369FB10DEA1FFA1FB695EA1FF0
:10E01000FA1F11248CAD9DAD8E0F9F1F9093AA11F6
:10E020008093A91128AD39AD4AAD5BADA0E0B0E059
:10E03000281739074A075B0720F43093AA11209369
:10E04000A9116091A9117091AA118CE96134780726
:10E0500018F060E47CE904C09EE46132790730F096
:10E06000769567957695679584E007C0E7E261311C
:10E070007E0730F07695679582E08093A41108C002
:10E0800081E08093A4116032710510F460E270E0C9
:10E0900060527040F8E060307F07E8F0472F50E0B2
:10E0A000440F551F440F551F455A574F9A012E5F75
:10E0B0003F4FF901859194919C01AA27639FC0016C
:10E0C000629F810D9A1F06948A1F9A1F1124FA01DC
:10E0D000459154911EC0CB01969587958C7F855AAA
:10E0E000934FFC0145915491FC0132962591349156
:10E0F000862F90E087709070FC012E9FC0012F9FAB
:10E10000900D3E9F900D1124B3E096958795BA959A
:10E11000E1F7481B590B44365105A8F4E3EFF2E050
:10E1200007C08091C00085FFFCCF31969093C60058
:10E1300090819923B1F787E09AE04AE050E00E948D
:10E14000B24244E650E050938900409388009A011F
:10E1500040E050E08091A5119091A611A091A711E7
:10E16000B091A811820F931FA41FB51F8093A51112
:10E170009093A611A093A711B093A81102C120916A
:10E18000991130919A1140919B1150919C11888D59
:10E19000998DAA8DBB8D82179307A407B50708F048
:10E1A000E4C06091AB117091AC118091AD11909170
:10E1B000AE112C8D3D8D4E8D5F8DAA27639FB12DA5
:10E1C000749FF001849FF00D839FE00DF11D649F0B
:10E1D000B00DE11DFA1F739FB00DE11DFA1F829F64
:10E1E000B00DE11DFA1F729FB10DEA1FFA1FB6951F
:10E1F000EA1FFA1F11248091A9119091AA118E177C
:10E200009F0738F4C05CDF4F68817981C054D040EB
:10E2100003C0BC016E1B7F0BC05CDF4F28813981BE
:10E220004A815B81CB01A0E0B0E082179307A4078D
:10E23000B50708F4B901FCE961347F0718F060E420
:10E240007CE904C02EE46132720730F07695679560
:10E250007695679584E007C037E26131730730F047
:10E260007695679582E08093A41108C081E0809341
:10E27000A4116032710510F460E270E060527040E9
:10E2800048E060307407E8F0472F50E0440F551F16
:10E29000440F551F455A574F9A012E5F3F4FF901C2
:10E2A000859194919C01AA27639FC001629F810D73
:10E2B0009A1F06948A1F9A1F1124FA0145915491BE
:10E2C0001EC0CB01969587958C7F855A934FFC0194
:10E2D00045915491FC01329625913491862F90E01E
:10E2E00087709070FC012E9FC0012F9F900D3E9F64
:10E2F000900D112423E0969587952A95E1F7481B08
:10E30000590B44365105A8F4E3EFF2E007C08091C1
:10E31000C00085FFFCCF31969093C6009081992371
:10E32000B1F787E09AE04AE050E00E94B24244E64A
:10E3300050E050938900409388009A0140E050E0FB
:10E340008091AB119091AC11A091AD11B091AE1133
:10E35000820F931FA41FB51F8093AB119093AC1134
:10E36000A093AD11B093AE110CC08091AF119091FC
:10E37000B01190938900809388008091B1118093AF
:10E38000A4112091991130919A1140919B115091B3
:10E390009C11E0916B11F0916C1180899189A28997
:10E3A000B389281739074A075B0780F010926C1170
:10E3B00010926B119091551180915611981731F070
:10E3C000809156118F5F8F7080935611FF91EF915E
:10E3D000DF91CF91BF91AF919F918F917F916F917D
:10E3E0005F914F913F912F911F910F91FF90EF906F
:10E3F000DF90CF90BF90AF900F900BBE0F900FBEED
:10E400000F901F90189580919F11882349F4809157
:10E41000A111882329F48091A311882309F49CC0B9
:10E42000EBE5F0E1949108C08091C00085FFFCCF3E
:10E430009093C600319694919923B1F7EDE9F0E1FC
:10E44000949108C08091C00085FFFCCF9093C600D6
:10E45000319694919923B1F780919F118823F1F01F
:10E4600060916D1170916E1180916F11909170118A
:10E470000E945FDC2091290C30912A0C40912B0CDA
:10E4800050912C0C0E94C4DBAB01BC0189E990E1E6
:10E490000E94211F89E890E10E9481CF8091A11103
:10E4A0008823F1F060917111709172118091731154
:10E4B000909174110E945FDC20912D0C30912E0CF4
:10E4C00040912F0C5091300C0E94C4DBAB01BC0179
:10E4D00085E890E10E94211F85E790E10E9481CFAD
:10E4E0008091A3118823F1F06091751170917611DC
:10E4F00080917711909178110E945FDC2091310C0E
:10E500003091320C4091330C5091340C0E94C4DB9A
:10E51000AB01BC0181E790E10E94211F81E690E1FF
:10E520000E9481CFE7E0F3E007C08091C00085FF43
:10E53000FCCF31969093C60090819923B1F78091DA
:10E54000C00085FFFCCF8AE08093C60010929F1127
:10E550001092A1111092A311089560E070E08FE76E
:10E5600093E42091BD033091BE034091BF035091CD
:10E57000C0030E94C4DBDC019B01AC012093FB11B2
:10E580003093FC114093FD115093FE11CB01809309
:10E59000FF1190930012A0930112B09302120895FC
:10E5A000FC0197FF03C08091CB1103C0E852FE4EDF
:10E5B000808190E008952F923F924F925F926F92E8
:10E5C0007F928F929F92AF92BF92CF92DF92EF9203
:10E5D000FF920F931F93CF93DF93EC0121E030E084
:10E5E000A901440F551F440F551FFA01E157FE4E74
:10E5F00085919491C817D9070CF059C0B9016150A1
:10E600007040660F771F660F771FCB018F569E4EA7
:10E61000FC010591149161577E4EFB01C590D49089
:10E62000FA01EF56FE4EE590F490FA01E157FE4EE6
:10E63000A590B490B801882777FD8095982F0E9407
:10E640005FDC1B012C01CC19DD09BE01882777FD99
:10E650008095982F0E945FDC3B014C01E01AF10A83
:10E660000027F7FC0095102FC801B7010E945FDC5E
:10E670009B01AC01C401B3010E949DDE7B018C01B2
:10E68000AC18BD08CC24B7FCC094DC2CC601B50185
:10E690000E945FDC9B01AC01C801B7010E94C4DB92
:10E6A0009B01AC01C201B1010E94E4DA19C0822FC2
:10E6B0008F5F2F5F3F4F2133310509F091CF8133B9
:10E6C00029F0E0E070E080E060E00CC0E1E5F2E11C
:10E6D00065917491882777FD8095982F0E945FDC63
:10E6E000E62F692F2E2F372F482F562FB901CA0139
:10E6F000DF91CF911F910F91FF90EF90DF90CF901E
:10E70000BF90AF909F908F907F906F905F904F9051
:10E710003F902F9008951092B4111092B31110925F
:10E72000D81174981092B6111092B5111092D91197
:10E7300075981092B8111092B7111092CB11A5983C
:10E7400008952DEB37E346E05EE30E949DDE0895D9
:10E750002DEB37E346E05EE30E94C4DB08952DEB2A
:10E7600037E346E05EE30E94C4DB08952DEB37E318
:10E7700046E05EE30E949DDE0895A5980E94011A7E
:10E78000882339F5ECEAF0E1949108C08091C0004B
:10E7900085FFFCCF9093C600319694919923B1F7F1
:10E7A000E4ECF0E1949108C08091C00085FFFCCFBB
:10E7B0009093C600319694919923B1F78091C0004F
:10E7C00085FFFCCF8AE08093C60083EB90E10E9436
:10E7D00090CF0E94A81A08951F93182F0E948B7340
:10E7E0000E94011A882309F036C0ECEAF0E1949106
:10E7F00008C08091C00085FFFCCF9093C600319681
:10E8000094919923B1F787E09AE0612F70E04AE094
:10E8100050E00E9488428091C00085FFFCCF8AE0D2
:10E820008093C600EBE0F1E1949108C08091C000B4
:10E8300085FFFCCF9093C600319694919923B1F750
:10E840008091C00085FFFCCF8AE08093C6008EEFE8
:10E8500090E10E9490CF0E94A81A1F9108951F93E3
:10E86000182F0E948B730E94011A882309F036C06A
:10E87000ECEAF0E1949108C08091C00085FFFCCFE4
:10E880009093C600319694919923B1F787E09AE06E
:10E89000612F70E04AE050E00E9488428091C00001
:10E8A00085FFFCCF8AE08093C600E5E4F1E1949116
:10E8B00008C08091C00085FFFCCF9093C6003196C0
:10E8C00094919923B1F78091C00085FFFCCF8AE035
:10E8D0008093C60088E391E10E9490CF0E94A81A1D
:10E8E0001F9108951F920F920FB60F920BB60F92C1
:10E8F00011242F933F934F935F936F937F938F9345
:10E900009F93AF93BF93EF93FF939091CF0399237E
:10E91000D9F48091D8118093E111882311F0749A71
:10E9200001C074988091D9118093E011882311F06F
:10E93000759A01C075988091CB118093DF1188235F
:10E9400011F0A59A01C0A5988091E111891708F4EA
:10E9500074988091E011891708F475988091DF11FF
:10E96000891708F4A5989F5F9F779093CF038091B4
:10E97000D003843009F471C0853050F4813021F126
:10E98000813098F08230F1F1833009F09FC049C0A6
:10E99000863009F48DC0863008F46EC0873009F4E3
:10E9A0008BC0883009F092C08FC088E080937B00D4
:10E9B00080E480937C0080917A00806480937A0068
:10E9C0000E94C69A81E01BC08091780090917900E6
:10E9D000A0E0B0E02091EE113091EF114091F011E4
:10E9E0005091F111280F391F4A1F5B1F2093EE1120
:10E9F0003093EF114093F0115093F11182E0809326
:10EA0000D00364C088E080937B0082E480937C0024
:10EA100080917A00806480937A000E94C69A83E095
:10EA2000EECF8091780090917900A0E0B0E0209145
:10EA3000E2113091E3114091E4115091E511280F5A
:10EA4000391F4A1F5B1F2093E2113093E31140935B
:10EA5000E4115093E51184E0D2CF88E080937B00ED
:10EA600081E480937C0080917A00806480937A00B6
:10EA70000E94C69A85E0C3CF80917800909179007A
:10EA8000A0E0B0E02091EA113091EB114091EC113F
:10EA90005091ED11280F391F4A1F5B1F2093EA1177
:10EAA0003093EB114093EC115093ED1186E0A7CF1A
:10EAB0000E94C69A87E0A3CF1092D0038091F211F2
:10EAC0008F5F8093F21102C01092D0038091F211F7
:10EAD000803108F48AC08091DA118823C1F48091D2
:10EAE000EE119091EF119093BA118093B91180912A
:10EAF000EA119091EB119093BC118093BB1180911E
:10EB0000E2119091E3119093C6118093C51181E0B9
:10EB10008093DA111092F2111092EE111092EF110F
:10EB20001092F0111092F1111092EA111092EB1163
:10EB30001092EC111092ED111092E6111092E71163
:10EB40001092E8111092E9111092E2111092E31163
:10EB50001092E4111092E5112091B9113091BA117F
:10EB60008091C9039091CA03281739071CF080E0EF
:10EB70000E942F742091B9113091BA118091DB114C
:10EB80009091DC11821793071CF080E00E94EC73D7
:10EB90002091BB113091BC118091CB039091CC039B
:10EBA000281739071CF081E00E942F742091BB11B7
:10EBB0003091BC118091DD119091DE118217930785
:10EBC0001CF081E00E94EC732091C5113091C611B8
:10EBD0008091CD039091CE032817390734F010921D
:10EBE000B8111092B7110E94BD73FF91EF91BF91C0
:10EBF000AF919F918F917F916F915F914F913F91D5
:10EC00002F910F900BBE0F900FBE0F901F90189575
:10EC1000EF92FF920F931F93E090BD11F090BE1101
:10EC20000091BF111091C0116091B3117091B41196
:10EC3000882777FD8095982F0E945FDC20E030E0E8
:10EC400040EA51E40E94E3DA9B01AC01C801B7013C
:10EC50000E94BDDB882394F4C801B7010E942CDC1C
:10EC60007093CD116093CC110E94CD146093D0119C
:10EC70007093D1118093D2119093D311E090C11170
:10EC8000F090C2110091C3111091C4116091B5119F
:10EC90007091B611882777FD8095982F0E945FDCD0
:10ECA00020E030E040EA51E40E94E3DA9B01AC014D
:10ECB000C801B7010E94BDDB882394F4C801B701E5
:10ECC0000E942CDC7093CF116093CE110E94CD1462
:10ECD0006093D4117093D5118093D6119093D7116E
:10ECE0001F910F91FF90EF9008952F926F927F9256
:10ECF0008F929F92AF92BF92CF92DF92EF92FF924C
:10ED00000F931F93DF93CF93CDB7DEB729970FB63D
:10ED1000F894DEBF0FBECDBF8C01E62E61E06E150C
:10ED200068F5ECEAF0E1949108C08091C00085FF9D
:10ED3000FCCF9093C600319694919923B1F787E068
:10ED40009AE06E2D70E04AE050E00E948842E2E7CF
:10ED5000F1E1949108C08091C00085FFFCCF9093B1
:10ED6000C600319694919923B1F78091C00085FF38
:10ED7000FCCF8AE08093C6000E94EA1AAE2DB0E074
:10ED8000FD01EE0FFF1FE65CFB4F808191819987AB
:10ED90008887892B09F49FC0A25CBB4F9C919B8301
:10EDA0002224239479C0222D30E0A901440F551F5D
:10EDB000440F551FE885F985E40FF51F859194915F
:10EDC000081719070CF067C0C9010197880F991F30
:10EDD000880F991FFC013296A885B985EA0FFB1FA1
:10EDE000C590D4908A0F9B1FFC01659174917A8322
:10EDF0006983FA013296EA0FFB1FE590F490FD015A
:10EE0000E40FF51FA590B490B601882777FD809593
:10EE1000982F0E945FDC6C837D838E839F83898122
:10EE20009A81081B190BB801882777FD8095982FC8
:10EE30000E945FDC3B014C01EC18FD080027F7FC49
:10EE40000095102FC801B7010E945FDC9B01AC0147
:10EE5000C401B3010E949DDE7B018C01A981BA81AE
:10EE6000AA1ABB0ACC24B7FCC094DC2CC601B5019D
:10EE70000E945FDC9B01AC01C801B7010E94C4DBAA
:10EE80009B01AC016C817D818E819F810E94E4DABF
:10EE9000E62F692F09C02394BB812B1608F483CF7A
:10EEA000E0E070E080E060E0FB812F1679F5E22D74
:10EEB000F0E0EE0FFF1FEE0FFF1F32976885798598
:10EEC000E60FF71F65917491882777FD8095982F3D
:10EED0000E945FDC19C0B801882777FD8095982FC4
:10EEE0000E945FDC20E030E04AEF5EE30E949DDE9E
:10EEF00020E030E040E85DE30E949DDE20E030E06D
:10EF000040E050E00E94E4DAE62F692F2E2F372FE1
:10EF1000482F562FB901CA0129960FB6F894DEBFC3
:10EF20000FBECDBFCF91DF911F910F91FF90EF905A
:10EF3000DF90CF90BF90AF909F908F907F906F9019
:10EF40002F900895CF92DF92EF92FF920F931F932D
:10EF5000CF93DF9360E070E08FE793E42091BD03EF
:10EF60003091BE034091BF035091C0030E94C4DBA7
:10EF7000E091D103F091D2030F2EF0E0EF2EF0E0FC
:10EF8000FF2EF0E00F2FF0E01F2FF02DE092F31195
:10EF9000F092F4110093F5111093F6119B01482F94
:10EFA000592F2093FB113093FC114093FD11509386
:10EFB000FE11F093D403E093D303E092F711F092A3
:10EFC000F8110093F9111093FA11CB01DA01809333
:10EFD000FF1190930012A0930112B09302126C9A49
:10EFE0006D9A9D9A8091010180618093010187E073
:10EFF00061E070E00E94041A87ED80937A0010921D
:10F000007E0010927D0080917D00816080937D0064
:10F0100080917D00826080937D0080917D0084607E
:10F0200080937D0080E888BD80916E00846080932D
:10F030006E006AEF70E080E090E00E94DB1485E0F3
:10F0400090E0909304128093031209C08091DB1129
:10F050009091DC1140969093DC118093DB118091AC
:10F06000DB119091DC1160E00E94757620E030E0C9
:10F0700040EA50E40E94BDDB87FDE8CF83E191E0E8
:10F080009093D2038093D10309C08091C9039091DA
:10F09000CA0340979093CA038093C9038091C90320
:10F0A0009091CA0360E00E94757620E030E849E85C
:10F0B00053E40E94CBDD181644F385E090E0909372
:10F0C00006128093051209C08091DD119091DE1126
:10F0D00040969093DE118093DD118091DD11909127
:10F0E000DE1161E00E94757620E030E040EA50E4F5
:10F0F0000E94BDDB87FDE8CF83E191E09093D403CC
:10F100008093D30309C08091CB039091CC034097A7
:10F110009093CC038093CB038091CB039091CC034D
:10F1200061E00E94757620E030E849E853E40E94EF
:10F13000CBDD181644F3C091CD03D091CE03EC2E55
:10F14000DD2ECE010E94DB72609720E030E046E1C8
:10F1500053E40E94CBDD181694F3E092CD03D092D5
:10F16000CE03DF91CF911F910F91FF90EF90DF9031
:10F17000CF9008958091B9119091BA1160E00E94EA
:10F1800075766093BD117093BE118093BF119093FB
:10F19000C0118091BB119091BC1161E00E94757605
:10F1A0006093C1117093C2118093C3119093C411E5
:10F1B0008091C5119091C6110E94DB726093C711B6
:10F1C0007093C8118093C9119093CA110E948D96B3
:10F1D0008FB7F8941092DA118FBF08952F923F9253
:10F1E0004F925F926F927F928F929F92AF92BF9257
:10F1F000CF92DF92EF92FF920F931F93DF93CF9303
:10F20000CDB7DEB765970FB6F894DEBF0FBECDBFA2
:10F210008091DA11882309F472C20E94BA788DEBCA
:10F2200091E19A8B898BA3EBB1E1B88BAF87E0EDCD
:10F23000F1E1FC87EB8788ED91E19A878987A9E264
:10F24000B2E1B887AF83EFE0F2E1FE83ED8381E1C5
:10F2500092E19C838B83A1E3B2E1BA83A9831D8AE7
:10F260001C8A1E861D86E3E5F2E1B491BB8BE98919
:10F27000FA896080718082809380AF85B889CD9053
:10F28000DC90B601882777FD8095982F0E945FDC7F
:10F29000A40193010E94E3DA7B018C01EC89FD89D2
:10F2A000E95FFD4E608371838283938320E030E0C9
:10F2B00040E251E40E94CBDD18162CF421E0ED81F0
:10F2C000FE812083E1C0C801B70120E030E040E2C8
:10F2D00051EC0E94BDDB87FD02C0CD2829F4E1E09E
:10F2E000AD81BE81EC93BBC0AD81BE818C91882382
:10F2F00069F080E090E0A0E0B0E0EB81FC818083E9
:10F300009183A283B383AD81BE811C92C801B701F2
:10F310002091B9033091BA034091BB035091BC03D3
:10F320000E949DDE1B012C01EC89FD89E75EFD4EEC
:10F330006083718382839383C801B701EB81FC8171
:10F3400020813181428153810E94E4DA5B016C01AA
:10F35000EC89FD89ED50FE4EE080F1800281138141
:10F36000A80197010E94BDDB87FD12C0EC89FD89D1
:10F37000E550FE4EE080F18002811381C601B501A7
:10F38000A80197010E94CBDD181614F086017501C3
:10F39000AB81BC81ED92FD920D931C931397C80134
:10F3A000B7012091BD033091BE034091BF0350913E
:10F3B000C0030E949DDE5B016C01EC89FD89EF5D5D
:10F3C000FD4E6083718382839383C401B301EF8117
:10F3D000F88520813181428153810E94E3DA2091B6
:10F3E000C1033091C2034091C3035091C4030E94F2
:10F3F0009DDE20ED3CEC4CE45DE30E949DDE7B0154
:10F400008C01A981BA816D917D918D919C9123E3AD
:10F4100033E343E75FE30E949DDE9B01AC01C8013B
:10F42000B7010E94E4DA7B018C01E981FA816083F3
:10F43000718382839383C201B101A60195010E9469
:10F44000E4DAA80197010E94E3DA7B018C0120E055
:10F4500030E040E050E00E94BDDB88235CF40F2EDA
:10F46000F0E0EF2EF0E0FF2EF0E00F2FF0E01F2F86
:10F47000F02D14C0C801B70120E030E04FE753E49D
:10F480000E94CBDD181654F40F2EF0E0EF2EF0E0C2
:10F49000FF2EFFE70F2FF3E41F2FF02DAF81B8856C
:10F4A0006D927D928D929C921397ED85FE85ED5F16
:10F4B000FD4E60817181882777FD8095982F0E948D
:10F4C0005FDC9B01AC01C401B3010E94CBDD1816C7
:10F4D000F4F4ED85FE85EF52FC4F60817181882741
:10F4E00077FD8095982F0E945FDC9B01AC01C401E1
:10F4F000B3010E94BDDB882354F4C801B7010E9408
:10F500002CDC75956795E985FA85608303C0A9852C
:10F51000BA851C92EB85FC8580819181A281B381A3
:10F520000097A105B10509F45DC00E94CD14AB851B
:10F53000BC852D913D914D915C91621B730B840BA9
:10F54000950B61547C498040904008F44BC0ED8598
:10F55000FE85E453FE4E60817181665F7F4F882790
:10F5600077FD8095982F0E945FDC9B01AC01E989B3
:10F57000FA8960817181828193810E94BDDB882339
:10F580005CF5AF85B8891D921C9289E592E10E94D5
:10F5900081CF9B89E3E5F2E108C08091C00085FF3F
:10F5A000FCCF9093C600319694919923B1F7E8E08F
:10F5B000F3E007C08091C00085FFFCCF31969093A7
:10F5C000C60090819923B1F78091C00085FFFCCFE0
:10F5D000BAE0B093C60006C0EB85FC8510821182AC
:10F5E0001282138289899A8904969A8B898BAC89B5
:10F5F000BD891496BD8BAC8BEF85F8893296F88B5C
:10F60000EF878D859E8502969E878D87AB85BC850D
:10F610001496BC87AB87E985FA853196FA87E98726
:10F620008F819885049698878F83AD81BE811196CE
:10F63000BE83AD83EB81FC813496FC83EB838981AF
:10F640009A8104969A838983AC89BD89189709F0B9
:10F650000ECE0E94CD142091391230913A12409171
:10F660003B1250913C12621B730B840B950B685834
:10F6700073418040904008F442C00E94CD146093D2
:10F68000391270933A1280933B1290933C12E0909F
:10F69000C711F090C8110091C9111091CA11C80189
:10F6A000B70120E030E040EA50E40E94CBDD1816BC
:10F6B0001CF5C801B70120E030E046E153E40E94A8
:10F6C000BDDB8823CCF46091B7117091B811882705
:10F6D00077FD8095982F0E945FDC9B01AC01C801EB
:10F6E000B7010E94CBDD88231CF01092CB1107C01C
:10F6F0008FE78093CB1103C01092CB11A59865962C
:10F700000FB6F894DEBF0FBECDBFCF91DF911F9132
:10F710000F91FF90EF90DF90CF90BF90AF909F90B0
:10F720008F907F906F905F904F903F902F900895B3
:10F730002F923F924F925F926F927F928F929F9201
:10F74000AF92BF92CF92DF92EF92FF920F931F93EF
:10F75000DF93CF93CDB7DEB7E6970FB6F894DEBF51
:10F760000FBECDBF6C8F7D8F8E8F9F8F5EAB4DABED
:10F7700039A328A30E94CD14698B7A8B8B8B9C8B29
:10F780002DA93EA9233031051CF4E7E1F3E019C0AF
:10F79000EAE2F3E007C08091C00085FFFCCF31961C
:10F7A0009093C60090819923B1F78091C00085FFA6
:10F7B000FCCF14C48091C00085FFFCCF319690939C
:10F7C000C60090819923B1F78091C00085FFFCCFDE
:10F7D0008AE08093C6000E948B734DA95EA957FFF3
:10F7E00074C08FE78093CB1189899A89AB89BC89D2
:10F7F0008D879E87AF87B88B89879A87AB87BC87B1
:10F8000019AA1AAA1BAA1CAA1F8A1E8A91E09D8BFC
:10F810001D821E821F8218868FE7A82EB12CC12C54
:10F82000D12C0FE7202E312C412C512C20E030E040
:10F8300040E050E029833A834B835C830F2EF0E055
:10F840006F2EF0E47F2EFCE18F2EF6E49F2EF02D3C
:10F850004DA95EA948525E4E5BA34AA3EAE5F3E1D7
:10F8600054915CA3E5E5F3E184918DA3EEE4F3E12B
:10F8700094919EA3E7E4F3E1A491AFA3E1E4F3E163
:10F88000B491B8A7EBE3F3E1249129A7EDE2F3E10A
:10F8900034913AA7E7E2F3E144914BA7E1E2F3E1C7
:10F8A00054915CA7EBE1F3E184918DA7ADA9BEA9CA
:10F8B000AA0FBB1FAA0FBB1FA354BE4EBFA7AEA764
:10F8C000E1EEF2E1B491B8AB07C0EDA9FEA9E852B0
:10F8D000FE4E8FE7808388CF8091DA11882309F468
:10F8E000A3C20E94BA78EDA9FEA9F7FF0DC0F0915E
:10F8F000C711F9AB2091C8112AAB3091C9113BABAC
:10F900004091CA114CAB11C0AEA5BFA5BC91B9AB1B
:10F91000EEA5FFA5F181FAABAEA5BFA51296BC91ED
:10F92000BBABEEA5FFA5F381FCAB69817A818B812E
:10F930009C8129A93AA94BA95CA90E94CBDD181684
:10F9400044F089A99AA9ABA9BCA989839A83AB83FE
:10F95000BC83C401B30129A93AA94BA95CA90E949F
:10F96000BDDB87FD06C089A99AA9ABA9BCA93C014A
:10F970004D012D89222309F451C069A97AA98BA9C7
:10F980009CA92C8D3D8D4E8D5F8D0E94CBDD181670
:10F990000CF04AC20E94CD1429853A854B855C85BE
:10F9A000621B730B840B950B695873418040904028
:10F9B00008F43AC2D601C50182199309A409B50910
:10F9C0004DA95EA957FF07C0B595A795979587954F
:10F9D0008093CB1107C0B595A79597958795EAA118
:10F9E000FBA180830E94CD146D877E878F87988BC3
:10F9F0009B01AC0189859A85AB85BC85281B390B99
:10FA00004A0B5B0B2D833E834F8358872C8D3D8D96
:10FA10004E8D5F8D29833A834B835C8369A97AA9D4
:10FA20008BA99CA92C8D3D8D4E8D5F8D0E94BDDBD9
:10FA300088230CF0F8C10E94CD142D853E854F859A
:10FA40005889621B730B840B950B69587341804076
:10FA5000904008F4E8C10E94CD1469877A878B87AB
:10FA60009C874E895F89452B09F4B8C1DC01CB0125
:10FA70002D853E854F855889821B930BA40BB50BB2
:10FA80002D813E814F815885280F391F4A1F5B1FEA
:10FA9000288F398F4A8F5B8F2D813E814F8158850A
:10FAA000281B390B4A0B5B0BCA01B901A20191015A
:10FAB0000E946FDF288D398D4A8D5B8D0E94D7DFC4
:10FAC0002A0D3B1D4C1D5D1D24313105410551059D
:10FAD0005CF474E1272E312C412C512C64E1A62ECC
:10FAE000B12CC12CD12C1FC059016A013CEEA316C8
:10FAF000B104C104D1042CF05BEEA52EB12CC12CB5
:10FB0000D12C40E8A416B104C104D1041CF41501A1
:10FB1000260109C04EEF242E312C412C512C2A18DD
:10FB20003B084C085D089CA1EAE5F3E108C0809120
:10FB3000C00085FFFCCF9093C60031969491992325
:10FB4000B1F787E09AE0B601A5012AE030E00E9413
:10FB500053429DA1E5E5F3E108C08091C00085FF17
:10FB6000FCCF9093C600319694919923B1F787E02A
:10FB70009AE0B201A1012AE030E00E9453429EA126
:10FB8000EEE4F3E108C08091C00085FFFCCF9093C4
:10FB9000C600319694919923B1F787E09AE0B401B9
:10FBA000A30122E030E00E9463439FA1E7E4F3E178
:10FBB00008C08091C00085FFFCCF9093C6003196AD
:10FBC00094919923B1F787E09AE049815A816B813A
:10FBD0007C8122E030E00E9463438091C00085FF79
:10FBE000FCCF8AE08093C6008E899F8903970CF42E
:10FBF000F5C0C201B1010E945FDC20E030E040E8C6
:10FC000050E40E949DDE7B018C0169817A818B81A9
:10FC10009C81A40193010E94E3DA20ED3FE049E4D6
:10FC200050E40E949DDE20E030E040E05FE30E946F
:10FC30009DDE9B01AC01C801B7010E94C4DB7B01C2
:10FC40008C01688D798D8A8D9B8D0E945FDC20E010
:10FC500030E04AE754E40E94C4DB3B014C0198A524
:10FC6000E1E4F3E108C08091C00085FFFCCF9093F0
:10FC7000C600319694919923B1F787E09AE0B801D4
:10FC8000A70122E030E00E94634399A5EBE3F3E192
:10FC900008C08091C00085FFFCCF9093C6003196CC
:10FCA00094919923B1F787E09AE0B401A30122E08F
:10FCB00030E00E9463438091C00085FFFCCF8AE062
:10FCC0008093C600C801B7012AE939E949E15FE339
:10FCD0000E949DDE7B018C019AA5EDE2F3E108C054
:10FCE0008091C00085FFFCCF9093C600319694911F
:10FCF0009923B1F78091C00085FFFCCF8AE0809303
:10FD0000C6009BA5E7E2F3E108C08091C00085FF33
:10FD1000FCCF9093C600319694919923B1F787E078
:10FD20009AE0B801A70122E030E00E94634380918D
:10FD3000C00085FFFCCF8AE08093C6009CA5E1E26D
:10FD4000F3E108C08091C00085FFFCCF9093C6000E
:10FD5000319694919923B1F7C801B701A801970191
:10FD60000E94E4DAA40193010E94C4DBAB01BC0150
:10FD700087E09AE022E030E00E9463438091C00077
:10FD800085FFFCCF8AE08093C6009DA5EBE1F3E1FF
:10FD900008C08091C00085FFFCCF9093C6003196CB
:10FDA00094919923B1F7C801B701A40193010E946E
:10FDB0009DDE20E030E040E05EE30E949DDEAB018E
:10FDC000BC0187E09AE022E030E00E94634380912A
:10FDD000C00085FFFCCF8AE08093C600D201C1013C
:10FDE0008A0D9B1DAC1DBD1DEDA9FEA9F7FF07C027
:10FDF000B595A795979587958093CB1107C0B59535
:10FE0000A79597958795EAA1FBA180832E893F89C5
:10FE10002F5F3F4F3F8B2E8B6C8C7D8C8E8C9F8CFD
:10FE200031E03D8B01C01D8A6C8D7D8D8E8D9F8D47
:10FE300020E030E040EA51E40E94E4DA9B01AC01AA
:10FE400069A97AA98BA99CA90E94CBDD18169CF4FC
:10FE5000E1EFF2E1949108C08091C00085FFFCCFF2
:10FE60009093C600319694919923B1F78091C00088
:10FE700085FFFCCFB3C00E94CD1429893A894B89F4
:10FE80005C89621B730B840B950B615D774080402E
:10FE9000904008F454C04DA95EA957FF11C060916D
:10FEA000CB11EBEEF2E1949108C08091C00085FF88
:10FEB000FCCF9093C600319694919923B1F711C06D
:10FEC000AAA1BBA16C91E5EEF2E1949108C08091EA
:10FED000C00085FFFCCF9093C60031969491992382
:10FEE000B1F7162F87E09AE049A95AA96BA97CA916
:10FEF00022E030E00E94634398A9E1EEF2E108C0FD
:10FF00008091C00085FFFCCF9093C60031969491FC
:10FF10009923B1F787E09AE0612F70E04AE050E062
:10FF20000E9488428091C00085FFFCCF8AE08093C8
:10FF3000C6000E94CD14698B7A8B8B8B9C8B0E94A0
:10FF4000CD147B018C010E94CD142D853E854F85FB
:10FF50005889E21AF30A040B150B29853A854B855B
:10FF60005C85E21AF30A040B150BE60EF71E081F58
:10FF7000191F31E8E3163FE4F30632E1030730E0EE
:10FF8000130798F0E4ECF2E1949108C08091C0006E
:10FF900085FFFCCF9093C600319694919923B1F7D9
:10FFA0008091C00085FFFCCF19C04E895F8988A170
:10FFB00099A18417950774F5E8E6F2E1949108C0D9
:10FFC0008091C00085FFFCCF9093C600319694913C
:10FFD0009923B1F78091C00085FFFCCF8AE0809320
:10FFE000C600E6960FB6F894DEBF0FBECDBFCF9128
:10FFF000DF911F910F91FF90EF90DF90CF90BF9016
:020000021000EC
:10000000AF909F908F907F906F905F904F903F90B8
:100010002F9008950E94B3CF5FCCFC01128213820F
:100020000895FC018381882311F081E08283089583
:10003000FC018281811112820895CF93DF93DC014C
:10004000FC01EB55FE4F808191810097C9F101972A
:1000500091838083ED01CC5ADF4FFD01ED58FF4FB6
:100060008BE1019009928150E1F7FD01EE5AFF4FBB
:10007000AF58BF4F8D919C911197A157B04091837C
:100080008083FD01ED58FF4F20E030E0AD014B557E
:100090005E4F10C02F5F3F4FEF01DF015F968BE196
:1000A0000D9009928150E1F7858D968D329791835D
:1000B0008083B196DA018D919C912817390750F30E
:1000C000DF91CF910895FC0186E394E091838083D2
:1000D0008781882321F0CF0104960E9480470895EC
:1000E000CF92DF92EF92FF920F931F93DF93CF9304
:1000F000CDB7DEB76F970FB6F894DEBF0FBECDBF9A
:100100008C016B01095A1F4FD8018C910755104083
:10011000882321F42FE2E22EF12C03C090E5E92E92
:10012000F12CE00EF11E86E394E09A8389831C8211
:100130001B8218861D82B7016C5F7F4FCE0105962A
:10014000A60121E00E948D4E882391F5EEE6F3E1B1
:10015000949108C08091C00085FFFCCF9093C600A9
:10016000319694919923B1F7E4E7F3E1949108C0B3
:100170008091C00085FFFCCF9093C600319694918A
:100180009923B1F709C08091C00085FFFCCF089486
:10019000C11CD11C9093C600F6019081992399F758
:1001A0008091C00085FFFCCF8AE08093C6005AC0D2
:1001B000F801EB55FE4F208131812A30310508F0DE
:1001C00040C02F5F3F4F3183208321503040F901E1
:1001D00085E0EE0FFF1F8A95E1F7E21BF30BED5868
:1001E000FF4FE00FF11F13C0AF01415E5F4FBF0132
:1001F0008BE1DB010D90BD01DA010D92AD01815063
:10020000C1F7929182913296968F858F7F97215078
:100210003040BFEF2E3F3B0739F7D801AD58BF4FF5
:10022000F70134968BE101900D928150E1F70F5860
:100230001F4FF70182819381D8018D939C930157C1
:100240001040D801AC5ABF4FFE0135968BE10190AA
:100250000D928150E1F70E5A1F4F8B819C81F8015E
:1002600091838083CE0101960E9463806F960FB6C2
:10027000F894DEBF0FBECDBFCF91DF911F910F91DC
:10028000FF90EF90DF90CF900895EF92FF920F9341
:100290001F938C013EECE32E31E0F32EE80EF91EA5
:1002A000C7010E943047C7010E948047F8011082B1
:1002B00011821F910F91FF90EF900895CF92DF92DE
:1002C000EF92FF920F931F93CF93DF937C016B010B
:1002D000DB010D900020E9F78D0101501040061B55
:1002E000170BEEECF1E0EE0EFF1ED7011C92E2E3DD
:1002F000FEEFEE0EFF1ECB016EE470E00E94B51122
:10030000EC01009731F4F8013197EC0DFD1D8601E9
:100310000EC060E270E00E94B5118C010F5F1F4FAC
:10032000CE016AE270E00E94B511FC0131978DE0C8
:1003300081838AE082831382C70186539E4FB8016E
:100340000E948F4F8EEC91E0E80EF91ED7018C9140
:10035000882319F1EEE9F3E1949108C08091C0007F
:1003600085FFFCCF9093C600319694919923B1F705
:10037000E5EAF3E1949108C08091C00085FFFCCFCD
:100380009093C600319694919923B1F78091C00063
:1003900085FFFCCF8AE08093C600DF91CF911F914B
:1003A0000F91FF90EF90DF90CF900895CF93DF9360
:1003B000EC018B81882309F43BC0EDECF3E19491CF
:1003C00008C08091C00085FFFCCF9093C600319695
:1003D00094919923B1F7CD57DD4F488159816A81B6
:1003E0007B81C358D24087E09AE02AE030E00E9447
:1003F0003442EBECF3E1949108C08091C00085FF9A
:10040000FCCF9093C600319694919923B1F7C558CB
:10041000DD4F488159816A817B8187E09AE02AE03B
:1004200030E00E9434428091C00085FFFCCF12C0B2
:10043000EBEBF3E1949108C08091C00085FFFCCF05
:100440009093C600319694919923B1F78091C000A2
:1004500085FFFCCF8AE08093C600DF91CF9108959D
:100460002F923F924F925F926F927F928F929F92C4
:10047000AF92BF92CF92DF92EF92FF920F931F93B2
:10048000DF93CF93CDB7DEB7AC970FB6F894DEBF4E
:100490000FBECDBF5C014B01FC018381882309F4B1
:1004A00038C1C50182539E4F0E948047F5011282D8
:1004B0001A8A1D8A198A188A86E394E09F878E8794
:1004C0005EE4C52ED12CCA0CDB1C2FE230E0A20E5C
:1004D000B31EF601B182A08221ED3FEFA20EB31E42
:1004E000F40180818F3209F090C0C4016FE270E0A6
:1004F0000E94B5117C010894E11CF11C3E01089496
:10050000611C711C260142E1242E312C2C0E3D1E53
:1005100077C0C7016FE270E00E94B5116C010097CF
:1005200009F481C0E816F90608F07DC08C010E19A7
:100530001F09C301B701A8010E94D511060D171D9F
:10054000F8011082F30107C08091C00085FFFCCF45
:1005500031969093C60090819923B1F78091C000A5
:1005600085FFFCCFFAE0F093C600F2016081718153
:100570006115710519F460E070E002C06C5F7F4F97
:10058000C101A30121E00E948D4E882371F5E9E0AD
:10059000F4E1949108C08091C00085FFFCCF909356
:1005A000C600319694919923B1F7FE01319607C0A8
:1005B0008091C00085FFFCCF31969093C60090815A
:1005C0009923B1F7E7E0F4E1949108C08091C0006D
:1005D00085FFFCCF9093C600319694919923B1F793
:1005E0008091C00085FFFCCF8DC02EE030E02C0F45
:1005F0003D1FF2013183208376010894E11CF11C38
:10060000E114F10409F085CF0BC080E590E0A80E5D
:10061000B91EF601B182A08220EB3FEFA20EB31EFD
:10062000D82C092D02C0DE2C0F2D8EE490E0A80EF0
:10063000B91EF5018081918122EB3FEFA20EB31E1E
:10064000009719F480E090E001C004966D2D702FA2
:100650000E945F4F882339F1E9EFF3E1949108C0DC
:100660008091C00085FFFCCF9093C6003196949195
:100670009923B1F78D2D902F9C01F90107C080912E
:10068000C00085FFFCCF31969093C60090819923DE
:10069000B1F783E892E0A80EB91EF501108211822D
:1006A0001282138232C0E1EEF3E1949108C080918E
:1006B000C00085FFFCCF9093C6003196949199239A
:1006C000B1F78D2D902F9C01F90107C08091C000DA
:1006D00085FFFCCF31969093C60090819923B1F7A6
:1006E000EFEDF3E1949108C08091C00085FFFCCF4D
:1006F0009093C600319694919923B1F78091C000F0
:1007000085FFFCCF8AE08093C600CE010E960E9442
:100710006380AC960FB6F894DEBF0FBECDBFCF910D
:10072000DF911F910F91FF90EF90DF90CF90BF90DE
:10073000AF909F908F907F906F905F904F903F9081
:100740002F900895BF92CF92DF92EF92FF920F9376
:100750001F93CF93DF938C01EB018FE28993EE24FB
:10076000E394FF2475EAC72E71E0D72EC00ED11E88
:100770006FE1B62E14C0FB9CC00111248D589F4F11
:10078000800F911FBE010E94924702C02196E39400
:100790008881882319F08CE88E15C0F7F3942F2DEB
:1007A00030E0F601808191812817390720F3E7FCBA
:1007B00007C0C80182539E4FBE010E94924701C0EC
:1007C0001882DF91CF911F910F91FF90EF90DF90F2
:1007D000CF90BF9008952F923F924F925F926F9269
:1007E0007F928F929F92AF92BF92CF92DF92EF92C1
:1007F000FF920F931F93DF93CF93CDB7DEB7AD97E3
:100800000FB6F894DEBF0FBECDBF6C014B014DA7F4
:10081000DC0113968C91882309F44AC3E1EDF1E0E1
:10082000CE0EDF1ED6018C91EFE2FEEFCE0EDF1E64
:10083000882309F419C1222309F0E1C029EE31E02F
:10084000C20ED31ED6018C91E7E1FEEFCE0EDF1E65
:10085000882371F1EEE9F3E1949108C08091C00022
:1008600085FFFCCF9093C600319694919923B1F700
:10087000E1EEF4E1949108C08091C00085FFFCCFC7
:100880009093C600319694919923B1F787E09AE04E
:1008900061E070E04AE050E00E9488428091C00030
:1008A00085FFFCCF8AE08093C6000E94EA1A00C34D
:1008B000EEE6F3E1949108C08091C00085FFFCCF83
:1008C0009093C600319694919923B1F7E8ECF4E146
:1008D000949108C08091C00085FFFCCF9093C60022
:1008E000319694919923B1F7F40107C08091C0002B
:1008F00085FFFCCF31969093C60090819923B1F784
:10090000EDEBF4E1949108C08091C00085FFFCCF2D
:100910009093C600319694919923B1F7C6012EEEBB
:1009200031E0C20ED31EB6010E94A2834BEF5FEFEF
:10093000C40ED51ED6019C91E7E1FEEFCE0EDF1E60
:100940008DE8989FF0011124E251FE4FEC0DFD1D42
:1009500007C08091C00085FFFCCF31969093C60000
:1009600090819923B1F7E7EBF4E1949108C080916D
:10097000C00085FFFCCF9093C600319694919923D7
:10098000B1F723E832E0C20ED31ED6014D915D913E
:100990006D917C91EDE7FDEFCE0EDF1E87E09AE0D2
:1009A0002AE030E00E9434428091C00085FFFCCFF5
:1009B0008AE08093C600A60147515E4FDA012C9170
:1009C000E22FF0E0EE0FFF1FEE0FFF1FEC0DFD1DFD
:1009D000E651FE4F83E892E0C80ED91ED6014D9035
:1009E0005D906D907C908DE79DEFC80ED91E408282
:1009F0005182628273822F5FDA012C932FC0EEE660
:100A0000F3E1949108C08091C00085FFFCCF9093E2
:100A1000C600319694919923B1F7E6EAF4E19491F6
:100A200008C08091C00085FFFCCF9093C60031962E
:100A300094919923B1F7F40107C08091C00085FF1C
:100A4000FCCF31969093C60090819923B1F78091A5
:100A5000C00085FFFCCF8AE08093C600C6018253A8
:100A60009E4F0E94804739C0E9EEF1E0CE0EDF1EB6
:100A7000D6011C92E7E1FEEFCE0EDF1EEEE6F3E1BB
:100A8000949108C08091C00085FFFCCF9093C60070
:100A9000319694919923B1F7E5E9F4E1949108C076
:100AA0008091C00085FFFCCF9093C6003196949151
:100AB0009923B1F7F40107C08091C00085FFFCCFF6
:100AC00031969093C60090819923B1F78091C00030
:100AD00085FFFCCF8AE08093C600D60112961C9257
:100AE0001A8A1D8A198A188A86E394E09F878E875E
:100AF000FEE4AF2EB12CAC0CBD1CEFE2F0E0CE0E4C
:100B0000DF1ED501CD92DC92E1EDFFEFCE0EDF1EB0
:100B1000D4018C918F3209F090C0C4016FE270E073
:100B20000E94B5117C010894E11CF11C3E0108945F
:100B3000611C711C2501E2E12E2E312C2C0E3D1E74
:100B400077C0C7016FE270E00E94B5115C010097A9
:100B500009F481C0E816F90608F07DC08C010E1971
:100B60001F09C301B701A8010E94D511060D171D69
:100B7000F8011082F30107C08091C00085FFFCCF0F
:100B800031969093C60090819923B1F78091C0006F
:100B900085FFFCCFFAE0F093C600D2016D917C9105
:100BA0006115710519F460E070E002C06C5F7F4F61
:100BB000C101A30121E00E948D4E882371F5E1E877
:100BC000F4E1949108C08091C00085FFFCCF909320
:100BD000C600319694919923B1F7FE01319607C072
:100BE0008091C00085FFFCCF31969093C600908124
:100BF0009923B1F7EFE7F4E1949108C08091C00028
:100C000085FFFCCF9093C600319694919923B1F75C
:100C10008091C00085FFFCCF1BC12EE030E02C0F7F
:100C20003D1FF2013183208375010894E11CF11C02
:100C3000E114F10409F085CF0BC040E550E0C40E8B
:100C4000D51ED501CD92DC92E0EBFFEFCE0EDF1E7C
:100C5000082DF92C01C00E2DF601E25BFF4F2DA5EA
:100C6000222309F4B1C0608171816115710519F405
:100C700060E070E002C06C5F7F4FC60182539E4F00
:100C8000402F5F2D21E00E948D4E882309F46CC017
:100C90004FED51E0C40ED51ED6014D915D916D9181
:100CA0007C91ECE9F0E0CE0EDF1ED6014D935D9312
:100CB0006D937C931397E5E8FDEFCE0EDF1EE1E721
:100CC000F4E1949108C08091C00085FFFCCF90931F
:100CD000C600319694919923B1F7802F9F2D9C01E6
:100CE000F90107C08091C00085FFFCCF3196909339
:100CF000C60090819923B1F7E9E6F4E1949108C028
:100D00008091C00085FFFCCF9093C60031969491EE
:100D10009923B1F787E09AE02AE030E00E9434425C
:100D20008091C00085FFFCCF8AE08093C60023E855
:100D300032E0C20ED31ED6011D921D921D921C924E
:100D40001397EBE5F4E1949108C08091C00085FF12
:100D5000FCCF9093C600319694919923B1F780917E
:100D6000C00085FFFCCF99C0E7E4F4E1949108C08E
:100D70008091C00085FFFCCF9093C600319694917E
:100D80009923B1F7802F9F2D9C01F90107C0809115
:100D9000C00085FFFCCF31969093C60090819923C7
:100DA000B1F7E5E4F4E1949108C08091C00085FFBB
:100DB000FCCF9093C600319694919923B1F780911E
:100DC000C00085FFFCCF44C0608171816115710551
:100DD00019F460E070E002C06C5F7F4FC60182537F
:100DE0009E4F402F5F2D26E50E948D4E882309F0EF
:100DF00033C0E1E3F4E1949108C08091C00085FF25
:100E0000FCCF9093C600319694919923B1F7802F2F
:100E10009F2D9C01F90107C08091C00085FFFCCF88
:100E200031969093C60090819923B1F7EFE2F4E1F7
:100E3000949108C08091C00085FFFCCF9093C600BC
:100E4000319694919923B1F78091C00085FFFCCF32
:100E50008AE08093C60028C081E0F6018083EDE13E
:100E6000F4E1949108C08091C00085FFFCCF90937D
:100E7000C600319694919923B1F7F40107C080918F
:100E8000C00085FFFCCF31969093C60090819923D6
:100E9000B1F78091C00085FFFCCF8AE08093C60047
:100EA000802F9F2D0E94A4CFCE010E960E946380BA
:100EB000AD960FB6F894DEBF0FBECDBFCF91DF91D8
:100EC0001F910F91FF90EF90DF90CF90BF90AF9068
:100ED0009F908F907F906F905F904F903F902F905A
:100EE0000895EF92FF920F931F93CF93DF93EC013E
:100EF0000E94576B8E0107511E4FD8018C919EECBA
:100F0000E92E91E0F92EEC0EFD1E8823A1F1C70118
:100F10000E948047F8016081615060838DE8689F7E
:100F2000B001112462517E4F6C0F7D1FCE0141E054
:100F300021E00E94EB83D801EC91F0E0EE0FFF1F5F
:100F4000EE0FFF1FEC0FFD1FE651FE4F4081518158
:100F500062817381CD57DD4F488359836A837B83D8
:100F6000C358D240C7010E9466468B81882369F02E
:100F700081E08A830AC00E94406AC7010E948047BC
:100F80001A8282E693E10E941540DF91CF911F9172
:100F90000F91FF90EF900895FC0181E08183CF01D4
:100FA00040E021E00E94EB830895EF92FF920F93BF
:100FB0001F93CF93DF938C01FC01138286A98823B2
:100FC00021F0C801C3960E94804727EAE22E21E063
:100FD000F22EE00EF11EC70160E045E30E942A45B3
:100FE000882309F5EEE6F3E1949108C08091C000F2
:100FF00085FFFCCF9093C600319694919923B1F769
:10100000E2E5F5E1949108C08091C00085FFFCCF36
:101010009093C600319694919923B1F78091C000C6
:1010200085FFFCCF7DC0E801C455DE4FCE01B7017E
:1010300041E00E942450882341F5CE01B70140E0F1
:101040000E942450882309F5EEE9F3E1949108C049
:101050008091C00085FFFCCF9093C600319694919B
:101060009923B1F7EFE3F5E1949108C08091C000B6
:1010700085FFFCCF9093C600319694919923B1F7E8
:101080008091C00085FFFCCF4BC0C801C396BE0154
:101090000E94814A882309F5EEE9F3E1949108C0A2
:1010A0008091C00085FFFCCF9093C600319694914B
:1010B0009923B1F7EFE2F5E1949108C08091C00067
:1010C00085FFFCCF9093C600319694919923B1F798
:1010D0008091C00085FFFCCF23C081E0F8018383AD
:1010E000EEE6F3E1949108C08091C00085FFFCCF4B
:1010F0009093C600319694919923B1F7E4E2F5E11B
:10110000949108C08091C00085FFFCCF9093C600E9
:10111000319694919923B1F78091C00085FFFCCF5F
:101120008AE08093C600D801AC5ABF4FF801F3960D
:101130008BE101900D928150E1F7F80181A992A90C
:101140000E5A1F4FF8019183808302551040C80149
:101150008F96025B1F4FF80191838083DF91CF91BF
:101160001F910F91FF90EF9008952F923F924F9211
:101170005F926F927F929F92AF92BF92CF92DF92D7
:10118000EF92FF920F931F93DF93CF93CDB7DEB70C
:10119000CC55D0400FB6F894DEBF0FBECDBF6C016A
:1011A000662311F527E832E0C20ED31ED6018C91DA
:1011B000E9E7FDEFCE0EDF1E882309F4E2C02FE73A
:1011C00032E0C20ED31ED601ED90FD900D911C9120
:1011D000E1E8FDEFCE0EDF1E0E94CD14E616F70605
:1011E0000807190708F4CDC027E832E0C20ED31E65
:1011F000D6011C92E9E7FDEFCE0EDF1ED601139655
:101200008C91882341F4C6010E94D587F601838121
:10121000882309F4B6C000D000D0EDB7FEB73196F0
:101220007E010894E11CF11CADB7BEB71296FC928A
:10123000EE92119785E993E193838283D6019D967F
:101240008D919C919E97958384830E94E4118701E0
:10125000EDB7FEB736960FB6F894FEBF0FBEEDBFE2
:10126000570108C0D8018C9190E00E9400E0F8017D
:1012700081938F01F50101900020E9F73197EA1978
:10128000FB09802F8E198E176CF363E3A62EB12C09
:10129000AC0CBD1CC50140E050E060E070E00E9475
:1012A000664699245DE3E52EF12CEC0EFD1E2E0121
:1012B0000894411C511C4FE1642E712C6C0E7D1E54
:1012C0003EE8232E33E1332E42C0D8018C9190E0CA
:1012D0000E9400E0F80181938F01F7010190002046
:1012E000E9F73197EE19FF09802F8E198E176CF3ED
:1012F00027968FAD27978E3751F1C701B20145E090
:1013000050E00E94C711009711F500D000D0EDB752
:10131000FEB73196ADB7BEB712967C926E9211971A
:1013200033822282558244820E94E411EDB7FEB7D7
:1013300036960FB6F894FEBF0FBEEDBFC3010E94F4
:101340008E408AE893E10E94154099249394C50148
:10135000B70140E050E00E949D49181614F487013F
:10136000BCCF992041F48FEF9FEFD6019E969C93BE
:101370008E939D9706C0F60185A596A5019696A722
:1013800085A7C45ADF4F0FB6F894DEBF0FBECDBF9E
:10139000CF91DF911F910F91FF90EF90DF90CF9051
:1013A000BF90AF909F907F906F905F904F903F90D5
:1013B0002F9008952F923F924F925F926F927F925B
:1013C0008F929F92AF92BF92CF92DF92EF92FF9255
:1013D0000F931F93DF93CF93CDB7DEB7CF58D04095
:1013E0000FB6F894DEBF0FBECDBF8C013B016A0182
:1013F00084E090E0C80ED91EF8017196C757DF4F00
:10140000F983E883C958D040C8010496CA57DF4F12
:1014100099838883C658D040C857DF4F1882C85870
:10142000D040B6E6EB2EF12CEC0EFD1EF7013B96FC
:10143000C557DF4FF983E883CB58D040A8E88A2E00
:10144000A2E09A2E800E911EF9E8AF2EF2E0BF2E98
:10145000A00EB11EEEE02E2E312C2C0E3D1E77E498
:10146000472E512C4C0E5D1EC2010496C357DF4F10
:1014700099838883CD58D040EEE6F3E19491C1572B
:10148000DF4F9883CF58D04049C1F7018385282F7B
:1014900030E0A901487150704031510509F04CC14C
:1014A000F4019081913009F447C1923009F444C1AC
:1014B000F701DE0111969081903239F08E2F8E194E
:1014C000883011F48EE28D939D933196C557DF4F8E
:1014D00088819981CB58D040E817F90761F71C92B1
:1014E0001E86F3018081882329F4C10164E573E03D
:1014F0000E94AA11C101B3010E94AA11C101BE013B
:101500006F5F7F4F0E94AA11C10164E573E00E94E2
:10151000AA111CA61FA61BA61AA686E394E099A7EB
:1015200088A7CE018C96B601AE014F5F5F4F21E0D8
:101530000E948D4E882309F03EC0F40180818823EB
:10154000D1F5C157DF4F9881CF58D040EEE6F3E197
:1015500008C08091C00085FFFCCF9093C6003196F3
:1015600094919923B1F7E6E5F3E007C08091C000BC
:1015700085FFFCCF31969093C60090819923B1F7F7
:101580008091C00085FFFCCFFAE0F093C600FE0119
:10159000319607C08091C00085FFFCCF31969093B3
:1015A000C60090819923B1F78091C00085FFFCCFE0
:1015B0008AE08093C600C357DF4FA881B981CD5818
:1015C000D040FE01BC968BE101900D928150E1F775
:1015D0008AA59BA5F2019383828386E394E091839D
:1015E0008083C801B101A2010E94DA89C2010E9470
:1015F0006380CE0188960E94638090C0953E09F476
:101600008DC09E3209F48AC09F3509F487C0F80165
:101610009189992331F09E3209F480C09F3509F4F5
:101620007DC023FD7BC080E04031510509F481E09D
:10163000F80184A7882349F4F7018085873409F0ED
:101640006DC081858E3709F469C0CA57DF4FA88104
:10165000B981C658D040F7018081803241F08E2F89
:101660008E19883011F48EE28D9380818D9331969E
:10167000C557DF4F88819981CB58D040E817F907CB
:1016800059F71C92F4018081882329F5F30107C0E2
:101690008091C00085FFFCCF31969093C600908169
:1016A0009923B1F7CA57DF4FE881F981C658D04076
:1016B00007C08091C00085FFFCCF31969093C60093
:1016C00090819923B1F78091C00085FFFCCFFAE0AB
:1016D000F093C60023C0813039F4F50180819181F7
:1016E0000196918380831AC08230C1F4C857DF4FBE
:1016F000F881C858D0402F2F30E0F50180819181CA
:1017000028173907F1F0C857DF4FF881C858D04083
:10171000FF5FC857DF4FF883C858D040C601B701F4
:10172000C757DF4F48815981C958D0400E949D4911
:1017300018160CF4AACE05C0F7019081992309F080
:101740005DCFC157DF4F0FB6F894DEBF0FBECDBFE0
:10175000CF91DF911F910F91FF90EF90DF90CF908D
:10176000BF90AF909F908F907F906F905F904F90C1
:101770003F902F900895EF92FF920F931F93DF9366
:10178000CF93CDB7DEB76F970FB6F894DEBF0FBE1D
:10179000CDBF7C018C01025B1F4F805B9F4FF80126
:1017A0009183808328E832E0E20EF31E21E0F70106
:1017B00021937F011182108227E73DEFE20EF31E95
:1017C000049640E050E060E070E00E946646F80158
:1017D00020813181DE011596F90134968BE101906B
:1017E0000D928150E1F7F901828193819C838B8373
:1017F00086E394E09A838983C70169E673E08E01EA
:101800000F5F1F4FA8010E94DA89C8010E94638000
:10181000F701E757FD4F808191816F960FB6F894DD
:10182000DEBF0FBECDBFCF91DF911F910F91FF9013
:10183000EF900895EF92FF920F931F93DF93CF9352
:10184000CDB7DEB76F970FB6F894DEBF0FBECDBF32
:101850007C018C01025B1F4F805B9F4FF8019183DD
:10186000808328E832E0E20EF31E22E0F7012083B5
:1018700028E73DEFE20EF31EF701E757FD4F6083C7
:101880001182049640E050E060E070E00E946646FD
:10189000F80120813181DE011596F90134968BE142
:1018A00001900D928150E1F7F901828193819C832F
:1018B0008B8386E394E09A838983C70169E673E0AA
:1018C0008E010F5F1F4FA8010E94DA89C8010E9494
:1018D00063806F960FB6F894DEBF0FBECDBFCF9179
:1018E000DF911F910F91FF90EF900895EF92FF927B
:1018F0000F931F93DF93CF93CDB7DEB76F970FB6DC
:10190000F894DEBF0FBECDBF7C0188E892E0E80E00
:10191000F91EF701108288E79DEFE80EF91E870196
:101920000D5C1F4FC80140E050E060E070E00E9495
:101930006646DE011596F8018BE101900D9281500B
:10194000E1F7F70181A992A99C838B8386E394E058
:101950009A838983C70169E673E08E010F5F1F4F89
:10196000A8010E94DA89C8010E9463806F960FB6B1
:10197000F894DEBF0FBECDBFCF91DF911F910F91C5
:10198000FF90EF9008950F931F93CF93DF93DC01A7
:10199000D3961C92D397D6961C92D697D2961C9229
:1019A0001E92D19786E394E0D0969C938E939F9756
:1019B000AC5ABF4F1C9213961C92A755B040FD0124
:1019C000E05BFF4FAE5ABF4F11961C921E92A2557C
:1019D000B04091838083ED01C159DF4FFE0120E0CB
:1019E00030E0482F14821782138212824083918341
:1019F000215E3F4F7F9681E02633380799F7A8553F
:101A0000BE4F89E18C9313961C9258961C921B969C
:101A10001C9213961C92A15DB140FD01E653FE4F4E
:101A2000A453BE4F11961C921E9240839183A155E0
:101A3000BF4F1D921D921D921C92139718961D92D6
:101A40001D921D921C921397A358B24012961C929D
:101A5000129713961C9213971C9211961C92119731
:101A60008D0101581D4FF8011082118212821382DC
:101A7000AB55BE4F11961C921E92AC5BBF4F1C9291
:101A8000FE01C90111920197E9F7A256BF4F81E00B
:101A90008C93A758B2409E961C921E929D970E94CE
:101AA000CD1468577C4E8F4F9F4FF8016083718330
:101AB00082839383DF91CF911F910F910895DF93DC
:101AC000CF93CDB7DEB72A970FB6F894DEBF0FBE1F
:101AD000CDBF80916A0390916B03A0916C03B0918C
:101AE0006D038B839C83AD83BE83FE01339624E616
:101AF00030E08081F999FECF1FBA32BD21BD80BD93
:101B00000FB6F894FA9AF99A0FBE2F5F3F4F283616
:101B1000310511F03196EDCFE9E2FCE08081F999D1
:101B2000FECF1FBA32BD21BD80BD0FB6F894FA9A20
:101B3000F99A0FBE2F5F3F4F2837310511F03196CC
:101B4000EDCFE9E1FCE08081F999FECF1FBA32BD0B
:101B500021BD80BD0FB6F894FA9AF99A0FBE2F5F97
:101B60003F4F2838310511F03196EDCFE9E3FCE025
:101B70008081F999FECF1FBA32BD21BD80BD0FB65D
:101B8000F894FA9AF99A0FBE2F5F3F4F2839310522
:101B900011F03196EDCFEDE4FCE08081F999FECFB4
:101BA0001FBA32BD21BD80BD0FB6F894FA9AF99ADA
:101BB0000FBE2F5F3F4F2C39310511F03196EDCF1D
:101BC000E1E5FCE08081F999FECF1FBA32BD21BD6D
:101BD00080BD0FB6F894FA9AF99A0FBE2F5F3F4F67
:101BE000203A310511F03196EDCFE9E4FCE0808137
:101BF000F999FECF1FBA32BD21BD80BD0FB6F89452
:101C0000FA9AF99A0FBE2F5F3F4F243A310511F02F
